:020000040000fa
:080000000002040000000000f2
:020000040000fa
:100400000f7223000e7f24000e0188000000000000
:100410000c00070000a820000100200011000700c8
:10042000000020000000e000020032000000020096
:1004300000000000647c0200000000000040da00c0
:100440000000fe004440a900c0c421000000e000fc
:100450000300320000002000a00188004440a800f2
:100460000000060091018800800078000000eb0089
:1004700015003700e280400032a0b4009101ba00bc
:10048000e280400032a0b4009102ba00e280400055
:1004900032a0b4000002eb00472bde00f507b200eb
:1004a000602ce10004003a000059eb008301e900f0
:1004b000fdff3e00040037006128e100010032002a
:1004c0000082eb00040007001101ba000200e00006
:1004d000e8ff3a00000006003159ba008301e90044
:1004e0000c0032002159ba008301e90008003200f3
:1004f0000400e00003003a00e280400032a0b400b3
:10050000f5ff370011d9ba008301e900faff3a007c
:100510008100e800e180400032a0b4000000060045
:1005200000000000000000000000000000000000cb
:1005300000000000000000000000000000000000bb
:1005400000000000000000000040da000000fe0093
:10055000839f68000100e00002003d006000100081
:10056000e08018000300e00002003d00600111007f
:10057000e0811900050007004f00e00002003b0089
:1005800060001000e0801800000006006022b80043
:10059000060220000000d0008180d2000482d20038
:1005a0008582d2000000a0000202520083825a001d
:1005b000030031000202420083824a000000a100d1
:1005c0000603e900f3ff3a0000000600020ab90042
:1005d000001bb9000200b800810042008100430006
:1005e00000000600800178000001780031407800aa
:1005f000005978000004e000fcff3a000300780096
:1006000000000600889fbe008a9fbe008c9fbe002f
:100610000001780061ef20001100e0000b003a00bb
:10062000a0ef2000b077880090778800d17788000d
:10063000a1778800214090000004a000a04098000d
:10064000614090000004a000e0409800e7004100f5
:10065000c208de00c20cdd00a47780000d0121007d
:10066000007223000d05500022002000811f780039
:10067000110009000205d80000067800cf007800bc
:10068000c308dd00e48540008001eb000601210085
:1006900065ef20000100370001027800244090003f
:1006a0000008a300020032000a003700110a780097
:1006b00094007800214090000008a300fbff320066
:1006c00009014200828f500002003900840f51005e
:1006d0004600310094007800848f5000eeff3e0009
:1006e000868f500002003900858f5000eaff3900e4
:1006f00090778000800f52004f003a00858f5000a5
:100700004d003a008301e800e18f5100e2ff36001e
:100710008c8f5400040036008a8f54000200310090
:100720000b04780012003700614ab8006151b9002b
:10073000b0ff2f000100200002005000838058000d
:10074000800f5200818f5a000200350009047800a2
:10075000070037000d805400327223000200400071
:10076000110009000a80d8000a80b900000478004e
:10077000080078006f00070080017800e10f40005a
:100780002d00320090778000030878009277800077
:1007900064004100a2409000808f510002003200ae
:1007a0000104a000010037000104a10021419800cc
:1007b000088041006400500080097800907788002c
:1007c00062ef2000020878009177800021409000bd
:1007d0000004a000a0409800234090000004a10065
:1007e000a041980002027800a7ff3700a277880096
:1007f000828f5000090036009200780000ef200040
:10080000a2419000034878007177880014097800ad
:100810008040eb00a077800021409800a077800006
:10082000000a7800244090000004a00020429800b4
:1008300064004200010037000000eb004f06be00dc
:100840004f05be004f04be000000060064005000cb
:10085000a0778800a04090000104a10021409800ea
:1008600000000600889fbe008a9fbe000005780039
:10087000e401500013001000c285de002340900008
:100880000008a30004003200a377880023409000f2
:100890000004a100a04198000100780059ff070062
:1008a000000478000000e000170032008a0f5000ba
:1008b0001500320060b8970008005000c284de00c6
:1008c000898f550001003600890578004259dd0006
:1008d0008a007800080078000f0007008a0f540093
:1008e000090031004248dd00000044008a0f50003a
:1008f000050036000a0050000000440072778000b6
:10090000837780000288be00080078004f05be0093
:100910004f04be00000006008001eb00020037001b
:1009200061f079008301e800828f5100fcff3a00fa
:1009300000000600889fbe0080047800f0778000e9
:100940000000e00003003a00100007000000e00093
:100950000a003500f07780000900e00002003a004c
:100960000004780006003700000478000900400009
:10097000060007000000e00001003d000084eb00dd
:10098000080078004f04be000000060080007800d8
:100990000000e00004003a0000012100f077880028
:1009a00001017800060037000081eb00007223008f
:1009b000808f500002003e00f17788000001eb00bc
:0809c0000200780000000600af
:020000040000fa
:020000040001f9
:0457f800fe4300006c
:020000040000fa
:020000040001f9
:0457fc007f3e0000ec
:020000040000fa
:10000800a4020000a4020000a27f0000c67f000036
:10001800ea7f0000a4020000a4020000a40200007d
:10002800a4020000a4020000a4020000a402000030
:10003800a4020000a4020000a4020000a402000020
:1000480060410000a4020000047f0000a402000038
:10005800a4020000a4020000a4020000a402000000
:10006800a4020000a4020000a4020000a4020000f0
:100078006a7f0000a4020000a4020000a40200009d
:10008800a4020000a4020000a40200009a7e00005e
:10009800a4020000a4020000a4020000a4020000c0
:1000a800a4020000a4020000a4020000a4020000b0
:1000b800a4020000a4020000a4020000a4020000a0
:1000c800a4020000a4020000a4020000a402000090
:1000d800a4020000a4020000a4020000a402000080
:1000e800a4020000a4020000a4020000a402000070
:1000f800a4020000a4020000a4020000a402000060
:10010800a4020000a4020000a4020000a40200004f
:10011800a4020000a4020000a4020000a40200003f
:10012800a4020000a4020000a4020000a40200002f
:10013800a4020000a4020000a4020000a40200001f
:10014800a4020000a4020000a4020000a40200000f
:10015800a4020000a4020000a4020000a4020000ff
:10016800a4020000a4020000a4020000a4020000ef
:10017800a4020000a40200001a660000a402000005
:10018800a4020000a4020000a4020000a4020000cf
:10019800a4020000a4020000a4020000a4020000bf
:1001a800a4020000a4020000a4020000a4020000af
:1001b800a4020000a4020000a4020000a40200009f
:1001c800a4020000a4020000a4020000a40200008f
:1001d800a4020000a4020000a4020000a40200007f
:1001e800a4020000a4020000a4020000a40200006f
:0801f800a4020000a4020000b3
:020000040000fa
:10020800a4020000a4020000a27f0000c67f000034
:10021800ea7f0000a4020000a4020000a40200007b
:10022800a4020000a4020000a4020000a40200002e
:10023800a4020000a4020000a4020000a40200001e
:1002480060410000a4020000047f0000a402000036
:10025800a4020000a4020000a4020000a4020000fe
:10026800a4020000a4020000a4020000a4020000ee
:100278006a7f0000a4020000a4020000a40200009b
:10028800a4020000a4020000a40200009a7e00005c
:10029800a4020000a4020000a4020000a4020000be
:1002a800a4020000a4020000a4020000a4020000ae
:1002b800a4020000a4020000a4020000a40200009e
:1002c800a4020000a4020000a4020000a40200008e
:1002d800a4020000a4020000a4020000a40200007e
:1002e800a4020000a4020000a4020000a40200006e
:1002f800a4020000a4020000a4020000a40200005e
:10030800a4020000a4020000a4020000a40200004d
:10031800a4020000a4020000a4020000a40200003d
:10032800a4020000a4020000a4020000a40200002d
:10033800a4020000a4020000a4020000a40200001d
:10034800a4020000a4020000a4020000a40200000d
:10035800a4020000a4020000a4020000a4020000fd
:10036800a4020000a4020000a4020000a4020000ed
:10037800a4020000a40200001a660000a402000003
:10038800a4020000a4020000a4020000a4020000cd
:10039800a4020000a4020000a4020000a4020000bd
:1003a800a4020000a4020000a4020000a4020000ad
:1003b800a4020000a4020000a4020000a40200009d
:1003c800a4020000a4020000a4020000a40200008d
:1003d800a4020000a4020000a4020000a40200007d
:1003e800a4020000a4020000a4020000a40200006d
:0803f800a4020000a4020000b1
:020000040000fa
:1028000096010000a0010000aa010000b401000030
:10281000be010000c8010000d2010000dc01000080
:10282000e6010000aa0a0000a40a00009e0a0000b7
:10283000940100009e010000a8010000b201000008
:10284000bc010000c6010000d0010000da01000058
:10285000e4010000a80a0000a20a00009c0a00008f
:10286000900100009a010000a4010000ae010000e8
:10287000b8010000c2010000cc010000d601000038
:10288000e0010000a60a0000a00a00009a0a000069
:10289000530000002d0000003a200000000a000054
:1028a0000d00000042000000505000004d3a0000b2
:1028b0000020000045450000505200004f4d000030
:1028c000207700006f720000647300002075000024
:1028d00073650000642e00000a0d0000004c00002b
:1028e0006f610000646900006e67000020730000e3
:1028f00061760000656400002073000065740000cc
:10290000746900006e670000732e00002e2e000018
:102910000a0d0000004400006f6e0000650a000010
:102920000d00000053610000766900006e67000032
:102930002053000065740000746900006e67000099
:10294000732e00002e2e0000004400006f6e000069
:10295000652e00000a0d0000002a00002a2a00004f
:102960005265000073650000742000004f75000080
:102970007470000075740000732e00002a2a000095
:102980002a0a00000d0000004c2d000053740000c6
:10299000696300006b200000582d00006178000082
:1029a00069730000004c00002d53000074690000a2
:1029b000636b0000205900002d6100007869000061
:1029c00073000000522d0000537400006963000082
:1029d0006b200000582d0000617800006973000032
:1029e000005200002d53000074690000636b00006a
:1029f000205900002d61000078690000730000007c
:102a00004c2d000054720000696700002061000036
:102a10006e6100006c6f000067000000522d000026
:102a20005472000069670000206100006e610000c0
:102a30006c6f000067000000546f000075630000b9
:102a40006870000061640000204c000065660000b2
:102a500074200000205800002d61000078690000fb
:102a600073000000546f0000756300006870000080
:102a700061640000204c00006566000074200000c6
:102a8000205900002d6100007869000073000000eb
:102a9000546f0000756300006870000061640000fe
:102aa0002052000069670000687400002058000090
:102ab0002d6100007869000073000000546f000071
:102ac000756300006870000061640000205200001f
:102ad0006967000068740000205900002d61000043
:102ae0007869000073000000582d00005469000050
:102af0006c740000005900002d540000696c000047
:102b0000740000005368000061720000652000003e
:102b100062750000747400006f6e0000004c0000cd
:102b20002d53000074690000636b000020620000f8
:102b300075740000746f00006e000000522d0000dc
:102b400053740000696300006b2000006275000090
:102b5000747400006f6e0000004f0000707400007d
:102b6000696f00006e730000206200007574000041
:102b7000746f00006e000000442d000050610000e2
:102b80006420000055700000004400002d5000003b
:102b90006164000020520000696700006874000052
:102ba000004400002d50000061640000204400003b
:102bb0006f7700006e000000442d0000506100009f
:102bc000642000004c65000066740000004c0000aa
:102bd0002d5400007269000067200000627500003b
:102be000747400006f6e0000005200002d5400004d
:102bf00072690000672000006275000074740000b4
:102c00006f6e0000004c00002d420000756d00004a
:102c10007065000072000000522d00004275000037
:102c20006d700000657200000054000072690000c1
:102c3000616e0000676c0000652000006275000096
:102c4000747400006f6e00000043000069720000a1
:102c5000636c000065200000627500007474000061
:102c60006f6e000000430000726f0000737300007d
:102c70002062000075740000746f00006e00000098
:102c80005371000075610000726500002062000051
:102c900075740000746f00006e0000005053000057
:102ca0002062000075740000746f00006e00000068
:102cb000546f0000756300006870000061640000dc
:102cc0002062000075740000746f00006e00000048
:102cd000c4940000d3940000e2940000f19400003a
:102ce000009500000e9500001c9500003295000034
:102cf000489500005e950000749500007b950000eb
:102d0000829500008f9500009e950000ad95000013
:102d1000bc950000c5950000d1950000dc95000031
:102d2000e7950000f5950000039600000c96000062
:102d3000159600002596000033960000409600008e
:102d40004e9600005896000045720000726f000019
:102d5000723a0000204900006e64000065780000af
:102d6000206f000075740000206f000066200000d6
:102d7000726100006e670000652e0000200a0000ee
:102d80000d00000043680000616e00006e650000e9
:102d90006c200000004c00006f61000064690000be
:102da0006e67000020640000656600006175000029
:102db0006c740000207300006574000074690000ea
:102dc0006e67000073200000666f00007220000034
:102dd000004c00006f610000646900006e67000035
:102de000206100006c6c000020640000656600003b
:102df000617500006c7400002073000065740000b1
:102e0000746900006e670000732e00002e2e000013
:102e10000045000045500000524f00004d200000ca
:102e20007772000069740000652000006572000080
:102e3000726f0000723a0000200000003d3d00006b
:102e40003d4500006e74000065720000696e000070
:102e500067200000436f00006e6600006967000095
:102e6000204d00006f640000653a00000a0d00006c
:102e70000a0d00002a500000726500007373000004
:102e80002027000045730000632700002074000025
:102e90006f20000064690000737000006c61000026
:102ea00079200000636f00006e6600006967000013
:102eb0002067000075690000646500003d3d00006a
:102ec0003d0a00000d0a00000d00000045780000da
:102ed00069740000696e000067200000436f000005
:102ee0006e66000069670000204d00006f640000fe
:102ef000652e00000a0d000000530000504900003c
:102f00002042000075730000204d00006f64000037
:102f100065200000300a00000d0000005350000042
:102f20004920000042750000732000004d6f000032
:102f300064650000203100000a0d0000005300000d
:102f4000504900002042000075730000204d000031
:102f50006f64000065200000320a00000d000000d0
:102f6000535000004920000042750000732000000b
:102f70004d6f000064650000203300000a0d000062
:102f800000450000525200004f5200002053000044
:102f9000504900002042000055530000204d000021
:102fa0004f440000450a00000d0000004964000085
:102fb0006c65000020610000757400006f2d00003a
:102fc0006f6600006620000073650000742000003a
:102fd000746f000020310000302000006d69000097
:102fe0006e2e00000a0d000000490000646c000015
:102ff0006520000061750000746f00002d6f0000f7
:1030000066660000206400006973000061620000d1
:103010006c650000642e00000a0d000000540000e2
:103020006f670000676c000065640000206f00009f
:103030007574000070750000747300002072000049
:103040006573000065740000206f00006e200000b2
:1030500064690000736300006f6e00006e6500001d
:10306000637400002e0a00000d000000546f000081
:10307000676700006c650000642000006f75000049
:1030800074700000757400007320000070720000fe
:103090006573000065720000766500006420000022
:1030a0006f6e00002064000069730000636f000011
:1030b0006e6e000065630000742e00000a0d0000b3
:1030c000004c0000454400002042000072690000ee
:1030d00067680000746e000065730000733a0000ba
:1030e000200000004c45000044200000436f000019
:1030f0006c6f0000722000005365000074740000c3
:10310000696e0000673a000020000000426c000079
:10311000756500000052000065640000004f00006b
:10312000726100006e6700006500000059650000d4
:103130006c6c00006f770000004c0000696d0000af
:103140006500000047720000656500006e00000029
:103150005475000072710000756f00006973000003
:103160006500000050750000727000006c65000082
:1031700000500000696e00006b00000057680000fe
:103180006974000065000000414400004300000035
:103190004261000074740000657200007900000054
:1031a00045720000726f0000720000005050000075
:1031b0004d2000004f750000747000007574000011
:1031c000204d00006f640000652000003d200000dd
:1031d00000540000726900006d2000003d200000d6
:1031e000005400006f75000063680000706100000b
:1031f000642000004d6f000064650000203d000069
:10320000205600006972000074750000616c0000b7
:10321000204a00006f7900007374000069630000a9
:103220006b0a00000d000000546f00007563000081
:103230006870000061640000204d00006f640000b1
:10324000652000003d200000546f00007563000001
:1032500068700000616400000a0d00000054000066
:103260006f7500006368000070610000642000005a
:10327000537000006c690000742000003d200000c5
:103280004f6e00000a0d0000005400006f75000032
:10329000636800007061000064200000537000004b
:1032a0006c690000742000003d2000004f660000a3
:1032b000660a00000d0000005365000072760000f1
:1032c0006f2f00004d6f0000746f0000722000002f
:1032d000466f00007277000061720000642e0000eb
:1032e0000a0d00000053000065720000766f0000b8
:1032f0002f4d00006f7400006f720000205200001c
:103300006576000065720000736500002e0a0000fb
:103310000d000000506f0000736900007469000028
:103320006f6e0000206900006e7000007574000070
:10333000206d00006f640000652e00000a0d000083
:10334000004900006e630000726500006d650000ba
:103350006e740000616c0000206900006e70000057
:1033600075740000206d00006f640000652e000081
:103370000a0d00000053000065720000766f000027
:10338000206e00006f74000020720000656d000068
:103390006170000070650000642e00000a0d0000de
:1033a0000053000065720000766f0000207200007c
:1033b000656d000061700000706500006420000011
:1033c000746f0000204400002d7000006164000054
:1033d000206c000065660000742f00007269000018
:1033e00067680000742e00000a0d00000053000002
:1033f00065720000766f000020720000656d0000ad
:10340000617000007065000064200000746f0000af
:10341000204400002d700000616400002075000051
:10342000702f0000646f0000776e00002e0a00000d
:103430000d00000053650000727600006f20000050
:10344000726500006d61000070700000656400002e
:10345000207400006f20000073710000756100008f
:10346000726500002f63000069720000636c000049
:10347000652e00000a0d0000005300006572000078
:10348000766f000020720000656d00006170000022
:103490007065000064200000746f0000204400008c
:1034a0002d7000006164000020740000726900004b
:1034b000616e0000676c0000652f00006372000001
:1034c0006f730000732e00000a0d0000005300000f
:1034d00065720000766f000020720000656d0000cc
:1034e000617000007065000064200000746f0000cf
:1034f000204400002d70000061640000206c00007a
:1035000065660000742f00007269000067680000a3
:1035100074200000627500006d700000657200008c
:10352000732e00000a0d00000053000065720000b9
:10353000766f000020720000656d00006170000071
:103540007065000064200000746f0000206c0000b3
:1035500065660000742f0000726900006768000053
:10356000742000006a6f0000797300007469000025
:10357000636b00002070000075730000686200003b
:1035800075740000746f00006e7300002e0a000056
:103590000d00000053650000727600006f200000ef
:1035a000726500006d6100007070000065640000cd
:1035b000207400006f20000073680000617200003a
:1035c000652f00006f700000746900006f6e0000ce
:1035d000732e00000a0d000000450000727200000a
:1035e0006f7200002e0a00000d00000054720000ef
:1035f0006967000067650000722000004c690000e8
:103600006e6b0000204f00006e2e00000a0d0000bf
:1036100000540000726900006767000065720000d6
:10362000204c0000696e00006b2000004f66000017
:10363000662e00000a0d0000004c000065660000c8
:103640007420000053740000696300006b200000c8
:10365000446900006666000065720000656e000047
:1036600074690000616c0000204d00006978000062
:10367000204f00006e2e00000a0d0000004c0000dc
:103680006566000074200000537400006963000048
:103690006b2000004469000066660000657200004f
:1036a000656e000074690000616c0000204d000030
:1036b00069780000204f0000666600002e0a0000b6
:1036c0000d000000526900006768000074200000cf
:1036d00053740000696300006b200000446900001f
:1036e0006666000065720000656e00007469000087
:1036f000616c0000204d000069780000204f000040
:103700006e2e00000a0d00000052000069670000e4
:10371000687400002053000074690000636b0000af
:1037200020440000696600006665000072650000c4
:103730006e740000696100006c2000004d6900009b
:10374000782000004f660000662e00000a0d000081
:10375000004d000065630000616e0000756d0000a3
:10376000205300007465000065720000696e00005f
:10377000672000004d690000782000004f660000bf
:10378000662e00000a0d0000004d00006563000079
:10379000616e0000756d000020530000746500002c
:1037a00065720000696e0000672000004d6900002e
:1037b000782000004f6e00002e0a00000d0000006f
:1037c0004d650000636100006e7500006d20000013
:1037d0005374000065650000726900006e670000a8
:1037e000204d000069780000204f00006e2c000082
:1037f00020720000656d0000617000002072000002
:10380000696700006874000020730000746900009c
:10381000636b0000207900002d61000078690000d2
:1038200073200000746f000020000000537400003b
:10383000696300006b200000486f00006c640000aa
:103840002f52000065630000616c00006c200000d6
:103850006469000073610000626c00006564000030
:103860002e0a00000d000000537400006963000080
:103870006b200000486f00006c6400002f520000b5
:1038800065630000616c00006c200000746900003a
:1038900065640000207400006f2000004c2d0000c3
:1038a00053740000696300006b2000004275000043
:1038b000747400006f6e00002e0a00000d000000fe
:1038c00053740000696300006b200000486f000023
:1038d0006c6400002f52000065630000616c000002
:1038e0006c20000074690000656400002074000012
:1038f0006f200000522d0000537400006963000027
:103900006b20000042750000747400006f6e0000b0
:103910002e0a00000d000000526100006e670000da
:10392000652000004f6600006673000065740000ab
:10393000203d000020000000526100006e67000082
:10394000652000003d20000000440000656100008b
:1039500064620000616e0000642000003d200000f1
:1039600000530000656e0000736900007469000078
:103970007669000074790000203d000020000000fe
:10398000486f00006d650000205000006f7300005c
:1039900069740000696f00006e2000003d20000087
:1039a00000430000616c0000696200007261000069
:1039b000746900006e670000204100006c6c00001c
:1039c000204800006f6d000065200000506f00006f
:1039d00073690000746900006f6e0000732e0000b0
:1039e0002e2e0000004f000075740000707500005e
:1039f00074200000496e00007665000072740000bb
:103a0000656400002e0a00000d0000004f750000e4
:103a10007470000075740000204e00006f7200008a
:103a20006d6100006c2e00000a0d0000004f0000c8
:103a3000757400007075000074200000546f000061
:103a4000676700006c6500002e0a00000d00000092
:103a50004f75000074700000757400002053000062
:103a6000696e0000676c000065200000536800006c
:103a70006f7400002e0a00000d0000004f7500005a
:103a8000747000007574000020410000757400001f
:103a90006f66000069720000652e00000a0d0000cc
:103aa000004f000075740000707500007420000065
:103ab000546f0000676700006c6500002041000043
:103ac000757400006f66000069720000652e0000ca
:103ad0000a0d0000004f00007574000070750000b2
:103ae00074200000507500007368000062750000cb
:103af000747400006f6e00002e0a00000d000000bc
:103b000045520000524f0000522000004f55000067
:103b10005450000055540000204d00004f44000058
:103b2000452e00000a0d000000500000756c0000da
:103b3000736500005769000064740000682000008d
:103b40003d20000000300000206d0000730a0000de
:103b50000d00000041750000746f000066690000f0
:103b6000726500002050000065720000696f00005f
:103b7000642000003d200000000a00000d3d000010
:103b80003d3d0000476500006e6500007261000069
:103b90006c2000005365000074740000696e000022
:103ba000677300003d3d00003d0a00000d0000006d
:103bb000456e00007465000072200000636f000015
:103bc0006e66000069670000206d00006f640000f1
:103bd000653a0000204800006f6c0000642000007f
:103be000505300002042000075740000746f000004
:103bf0006e2000002b20000053680000617200005e
:103c0000652000003320000073650000636f000032
:103c10006e640000730a00000d0000005361000094
:103c200076650000206100006e64000020650000e1
:103c300078690000743a0000204800006f6c0000b2
:103c4000642000004f700000746900006f6e000077
:103c5000730a00000d0000004c6f0000616400005a
:103c60002064000065660000617500006c7400004f
:103c7000733a0000204800006f6c000064200000d0
:103c800053680000617200006520000031200000d0
:103c900073650000636f00006e6400002028000060
:103ca0006375000072720000656e000074200000f1
:103cb00063680000616e00006e6500006c29000002
:103cc0002f33000020730000656300006f6e00005a
:103cd0006473000020280000616c00006c2000006c
:103ce00063680000616e00006e6500006c73000088
:103cf000290a00000d00000043790000636c0000f9
:103d000065200000746f0000206e000065780000e0
:103d1000742f00007072000065760000696f00006b
:103d20007573000020630000686100006e6e000083
:103d3000656c0000203a0000205200002f4c00006b
:103d400020420000756d000070650000720a0000de
:103d50000d00000043790000636c00006520000046
:103d600053500000492000006275000073200000dd
:103d70006d6f000064650000733a0000205200007f
:103d80002d53000074690000636b0000202b0000bd
:103d90002054000072690000616e0000676c000032
:103da000650a00000d000000456e00006162000021
:103db0006c6500002f440000697300006162000020
:103dc0006c65000020690000646c00006520000044
:103dd00061750000746f00002d64000069730000bd
:103de000636f00006e6e000065630000743a0000af
:103df000205200002d53000074690000636b000026
:103e0000202b000020430000726f0000737300003d
:103e10000d0a00000050000072650000736500008c
:103e200072760000652f0000526500007365000087
:103e3000742000006f75000074700000757400003d
:103e4000732000006f6e0000206300006f6e0000a2
:103e5000747200006f6c00006c650000722000003e
:103e600064690000736300006f6e00006e650000ff
:103e7000637400003a200000522d000053740000cb
:103e8000696300006b2000002b20000050530000ed
:103e90002042000075740000746f00006e0a00007c
:103ea0000d00000043680000616e000067650000bf
:103eb000206c000069670000687400006261000007
:103ec00072200000627200006967000068740000e0
:103ed0006e650000737300003a2000004c2d000056
:103ee00053740000696300006b2000002b20000069
:103ef000442d000050610000642000004c6500006b
:103f0000667400002f5200006967000068740000aa
:103f10000a0d000000430000686100006e670000a9
:103f2000652000006c690000676800007462000092
:103f300061720000206300006f6c00006f7200006f
:103f40003a2000004c2d000053740000696300000b
:103f50006b2000002b2000005368000061720000fd
:103f6000650a00000d000000546f00006767000044
:103f70006c650000205200004320000050500000fb
:103f80004d2000004d6f000064650000206f0000b0
:103f90006e20000063680000313100003a2000000c
:103fa0004c2d000053740000696300006b2000007a
:103fb0002b2000004f700000746900006f6e00003d
:103fc000730a00000d0000000a0d00003d3d0000d6
:103fd0003d53000065720000766f00002041000034
:103fe000646a000075730000746d0000656e000067
:103ff000747300003d3d00003d0a00000d0000000c
:10400000546f0000676700006c65000020610000cd
:10401000627300006f6c0000757400006520000082
:10402000706f000073690000746900006f6e00001b
:104030002f6900006e630000726500006d6500006e
:104040006e740000616c0000206d00006f64000061
:10405000653a0000205200002d53000074690000f2
:10406000636b0000202b0000205200002d42000056
:10407000756d000070650000720a00000d00000000
:10408000496e000076650000727400002064000034
:104090006972000065630000746900006f6e0000c3
:1040a0003a200000522d00005374000069630000a4
:1040b0006b2000002b2000004c2d000042750000fa
:1040c0006d700000657200000a0d000000530000d2
:1040d000656e000073690000746900007669000075
:1040e000747900003a2000005472000069610000f9
:1040f0006e6700006c6500002f430000726f0000c7
:10410000737300000a0d00000044000065610000a8
:1041100064620000616e0000643a000020530000f9
:104120007175000061720000652f00004369000096
:10413000726300006c6500000a0d00000052000070
:10414000616e000067650000206f000066200000bf
:104150006d6f0000746900006f6e00003a2000006f
:10416000442d0000506100006420000055700000e4
:104170002f4400006f7700006e0a00000d00000061
:1041800054720000696d0000202800007261000078
:104190006e670000652000006f660000206d000063
:1041a0006f740000696f00006e2000006c690000f1
:1041b0006d69000074730000206d00006f760000d0
:1041c000652000007769000074680000207400001a
:1041d000726900006d2900003a200000442d0000a3
:1041e00050610000642000004c650000667400000f
:1041f0002f52000069670000687400000a0d00007b
:1042000000430000656e000074650000722000002d
:104210006f66000066730000657400002074000083
:10422000726900006d20000028720000616e0000bd
:1042300067650000206f0000662000006d6f0000c1
:10424000746900006f6e0000206c0000696d000052
:104250006974000073200000646f0000206e00008d
:104260006f740000206d00006f760000652900006b
:104270003a200000522d00005374000069630000d2
:104280006b2000002b200000442d00005061000036
:10429000642000004c650000667400002f5200008e
:1042a00069670000687400000a0d0000004a000001
:1042b0006f79000073740000696300006b200000d8
:1042c0007a650000726f000020630000616c0000de
:1042d0006962000072610000746900006f6e000086
:1042e0003a200000486f00006c640000205000007d
:1042f0005320000042750000747400006f6e0000cf
:104300002031000020730000656300006f6e000024
:1043100064200000286300007572000072650000d0
:104320006e74000020630000686100006e6e000083
:10433000656c0000292f0000332000007365000029
:10434000636f00006e6400007320000028610000ad
:104350006c6c000020630000686100006e6e00005d
:10436000656c0000732900000a0d00000053000076
:1043700065720000766f0000206800006f6c00001e
:10438000642f000072650000636100006c6c000027
:10439000207000006f73000069740000696f0000f6
:1043a0006e2000006d6f0000646500002065000055
:1043b0006e610000626c0000653a0000204c000055
:1043c0002d53000074690000636b0000202b000077
:1043d0002043000069720000636c0000650a000061
:1043e0000d0000005472000069670000676500005e
:1043f000722000006c6900006e6b00003a20000023
:104400004c2d000053740000696300006b20000015
:104410002b200000437200006f730000730a00003d
:104420000d000000546f000075630000687000000c
:1044300061640000206d00006f64000065200000d2
:1044400028610000627300006f6c0000757400004a
:1044500065200000706f000073690000746900003f
:104460006f6e000020760000732000007669000067
:1044700072740000756100006c2000006a6f00001b
:104480007973000074690000636b0000293a000032
:10449000205200002d53000074690000636b00007f
:1044a000202b0000204400002d500000616400001b
:1044b00020550000700a00000d000000546f00003d
:1044c00075630000687000006164000020730000e4
:1044d000706c0000697400002076000073200000fa
:1044e000776800006f6c0000653a00002052000001
:1044f0002d53000074690000636b0000202b000046
:10450000204400002d5000006164000020440000a1
:104510006f7700006e0a00000d0000004a6f000077
:104520007973000074690000636b00002064000070
:104530006966000066650000726500006e74000028
:10454000696100006c200000647200006976000060
:10455000652000006d690000786500007220000091
:104560003a2000004c2d00005374000069630000e5
:104570006b2000002b200000437200006f730000ce
:10458000730a00000d0000004a6f000079730000fc
:1045900074690000636b0000206d0000656300001b
:1045a000616e0000756d00002077000068650000f6
:1045b000656c0000206d00006978000065720000e5
:1045c0003a2000004c2d0000537400006963000085
:1045d0006b2000002b20000053710000756100006b
:1045e000726500000a0d000000520000656d0000b9
:1045f0006170000020630000686100006e6e0000c2
:10460000656c0000207400006f20000062750000df
:10461000747400006f6e000020700000616900007b
:10462000723a0000205200002d530000746900000f
:10463000636b0000202b0000205300007175000008
:1046400061720000650a00000d0000000a0d000004
:104650003d3d00003d42000075740000746f000095
:104660006e200000416400006a7500007374000051
:104670006d6500006e740000733d00003d3d00005c
:104680000a0d000000540000657300007420000053
:104690006f750000747000007574000020770000d2
:1046a000686900006c650000206300006f6e000008
:1046b0006669000067750000726900006e6700009f
:1046c0003a200000522d000053740000696300007e
:1046d0006b0a00000d000000496e000076650000c6
:1046e00072740000204f00007574000070750000a7
:1046f000743a000020430000726f000073730000e2
:104700000a0d000000430000686100006e670000b1
:104710006520000062750000747400006f6e000078
:10472000206d00006f64000065200000287000000c
:10473000757300006862000075740000746f0000fb
:104740006e2c0000207400006f670000676c000092
:10475000652c000020650000746300002e29000015
:104760003a20000054720000696100006e6700008a
:104770006c6500000a0d000000530000696e000027
:10478000676c0000652d0000536800006f74000026
:104790002f410000757400006f6600006972000010
:1047a00065200000707500006c730000652000003b
:1047b0007769000064740000683a0000204400003b
:1047c0002d50000061640000204c00006566000070
:1047d000742f00005269000067680000740a00002e
:1047e0000d000000416400006a7500007374000051
:1047f00020610000757400006f660000697200009f
:104800006520000070650000726900006f640000a0
:104810003a200000442d0000506100006420000098
:10482000557000002f4400006f7700006e0a0000f2
:104830000d0a00000d000000720000007100000071
:10484000700000002a2a00002a5200006573000050
:10485000657400002053000074610000746500005e
:10486000732e00002a2a00002a0a00000d00000012
:104870005541000052540000204900006e690000bc
:1048800074690000616c0000697a000065640000d2
:104890002f2e00000a0d0000004300004d440000d0
:1048a000206300006f6d0000706c000065740000f4
:1048b000653a0000200000005265000073650000aa
:1048c000742e00000a0d0000005200006561000017
:1048d0006420000041640000647200006573000001
:1048e000732e0000204c00006f630000616c00001c
:1048f00020420000445f0000414400004452000098
:104900003a200000002e000020530000746f0000c9
:10491000726900006e67000020610000646400009e
:1049200072650000737300002e0a00000d00000085
:104930000a0d0000004c00006f630000616c000075
:10494000204e0000616d0000652e00000a0d000081
:1049500000570000726900007465000020430000e9
:104960006c610000737300002e0a00000d0000004f
:104970005772000069740000652000005363000056
:10498000616e0000204500006e610000626c000056
:10499000652f00004469000073610000626c000034
:1049a000652e00000a0d0000004c0000696e00003a
:1049b0006b2000004b65000079200000526500006c
:1049c000706c0000792e00000a0d0000004f0000fe
:1049d00074680000657200002e0a00000d000000df
:1049e000526f00006c650000204300006861000009
:1049f0006e670000652000005375000063630000cf
:104a00006573000073660000756c00002e0a0000dc
:104a10000d000000526f00006c6500002043000094
:104a2000686100006e6700006520000046610000bc
:104a3000696c0000656400002e2000002045000025
:104a4000727200006f7200003a20000000490000fe
:104a50006e7100007569000072790000204300004b
:104a60006f6d0000706c000065740000650a000046
:104a70000d000000496e00007175000069720000b1
:104a80007920000052650000737500006c7400000e
:104a90002c200000726500006d6f0000746500003e
:104aa00020420000445f00004144000044520000e6
:104ab0003a200000004300006f6e00006e650000a9
:104ac00063740000696f00006e2000004163000005
:104ad00063650000707400006564000020450000fc
:104ae000766500006e7400003a200000005300005c
:104af0007563000063650000737300002e200000e2
:104b0000486100006e6400006c650000203d0000fc
:104b10002000000045720000726f0000723a000031
:104b200020000000496e0000636f00006d69000006
:104b30006e670000204300006f6e00006e6500008d
:104b400063740000696f00006e3a0000205200009c
:104b5000656d00006f740000655f00004264000036
:104b60005f41000064640000722000003d200000ee
:104b70000044000069730000636f00006e6e000067
:104b8000656300007420000045760000656e00003b
:104b9000743a0000200000005375000063630000b9
:104ba00065730000732e0000004500007272000063
:104bb0006f7200002e000000456e0000637200005e
:104bc00079700000746900006f6e000020630000bf
:104bd000686100006e670000653a00000043000055
:104be000686100006e6e0000656c000020450000ea
:104bf0006e6300007279000070740000696f00003d
:104c00006e2000004f6e00002e2000004861000062
:104c10006e6400006c6500003d000000436f000002
:104c20006d6d0000616e0000642000005374000090
:104c30006174000075730000204500007665000077
:104c40006e7400003a20000000500000656e000005
:104c5000646900006e6700002e00000045720000cd
:104c6000726f0000722000003078000030320000c7
:104c70003a200000556e00006b6e00006f77000058
:104c80006e200000436f00006e6e00006563000040
:104c9000746900006f6e000020490000442e00007f
:104ca00000450000727200006f7200002043000097
:104cb0006f640000653a0000004c0000696e00005f
:104cc0006b2000004b650000792000005265000059
:104cd0007175000065730000742e00002020000034
:104ce000424400005f41000044440000523a00008a
:104cf000004d000061780000205300006c6f000040
:104d00007473000020430000686100006e670000bb
:104d1000652e00000a0d0000004300006f640000d3
:104d2000653d000030780000303100002e2000008a
:104d3000436f00006d6d0000616e00006420000094
:104d4000526500006a65000063740000656400003d
:104d50002e0a00000d000000436f00006465000093
:104d60003d30000078300000322e00002843000063
:104d70006f6e00006e65000063740000696f0000d4
:104d80006e20000052650000712900002e00000016
:104d9000505300004d3d00003078000030300000de
:104da000303100002028000053440000502900004a
:104db0002e20000053430000494400003d00000045
:104dc000505300004d3d00003078000030300000ae
:104dd000313100002028000048490000445f0000f5
:104de00043540000524c0000292e000020530000c4
:104df00043490000443d000000500000534d0000b6
:104e00003d3000007830000030310000332e0000cb
:104e10002053000043490000443d000000210000f1
:104e20002121000045720000726f0000723a0000fc
:104e300020500000534d0000206e00006f740000f1
:104e40002073000075700000706f00007274000025
:104e5000656400002e0a00000d000000436f000092
:104e60006e6e000065630000746900006f6e0000e4
:104e7000204300006f6d0000706c0000657400003e
:104e8000653a000000530000756300006365000090
:104e9000737300002e200000004800004944000009
:104ea00020430000545200004c2000002850000015
:104eb000534d0000203000007831000031290000ff
:104ec0000a0d000000480000494400002044000092
:104ed000415400004120000028500000534d0000c4
:104ee0002030000078310000332900000a0d000056
:104ef000005500006e6b00006e6f0000776e0000c2
:104f00000a0d000000500000656e0000646900009a
:104f10006e6700002e2e00002e0a00000d0000001b
:104f200046610000696c000075720000652e00008b
:104f300020450000727200006f7200003a0000000d
:104f4000436f0000646500003d30000078300000d1
:104f500034280000436f00006e660000696700009f
:104f60002052000065710000293a0000004800004e
:104f700049440000204300006f6e0000747200007e
:104f80006f6c000020430000686100006e6e00003e
:104f9000656c00002e0a00000d000000484900006a
:104fa00044200000446100007461000020430000c0
:104fb000686100006e6e0000656c00002e0a000043
:104fc0000d00000053440000502000004368000022
:104fd000616e00006e6500006c2e00000a0d00007e
:104fe000002100002121000045720000726f0000c6
:104ff000723a0000205500006e6b00006e6f0000da
:10500000776e000020430000686100006e6e0000b3
:10501000656c000020490000442e00000a0d0000cd
:10502000004300006f640000653d00003078000020
:1050300030350000284300006f6e000066690000f4
:10504000672000005265000073700000292e0000e8
:1050500020000000537500006363000065730000ca
:10506000730a00000d00000046610000696c00003a
:105070002e0a00000d000000446900007363000068
:105080006f6e00006e650000637400002072000007
:105090006571000075650000737400003a0000003f
:1050a0002044000041540000412e00000a0d000081
:1050b0000020000043540000524c00002e0a000063
:1050c0000d00000020530000445000002e0a000094
:1050d0000d000000205500006e6b00006e6f000098
:1050e000776e000020430000686100006e6e0000d3
:1050f000656c00002e0a00000d00000044690000ed
:10510000736300006f6e00006e6500006374000042
:105110002052000065730000706f00006e73000085
:10512000653a000000430000683a00005344000064
:10513000502e00000a0d00000053000044500000f3
:105140002041000074740000726900006275000064
:105150007465000020520000657100007565000054
:10516000737400002e0a00000d000000577200004a
:105170006974000065200000436c0000617300004a
:105180007320000045720000726f0000723a000048
:1051900020000000202d000020410000434c0000b2
:1051a00020630000616e00006e6f0000742000003c
:1051b00062650000207700007269000074740000ce
:1051c000656e00002000000042540000204f0000e7
:1051d0007574000070750000743a00002000000033
:1051e00045720000726f0000723a00002043000018
:1051f000616e00006e6f00007420000066690000a0
:105200006e640000206300006f7200007265000091
:10521000637400002074000079700000652e0000a7
:105220000a0d0000004900004e490000540a000029
:105230000d00000048430000495f0000434d00009e
:10524000445f00005245000053450000543a0000fe
:105250002000000048430000495f0000434d00006b
:10526000445f000052450000414400005f420000de
:10527000445f000041440000445200003a20000016
:1052800000480000434900005f4300004d44000017
:105290005f4c00004f430000414c00005f4e000097
:1052a000414d0000453a0000200000004843000046
:1052b000495f0000434d0000445f0000434c000084
:1052c00041530000535f0000444500005649000070
:1052d000434500003a200000004800004349000018
:1052e0005f4300004d4400005f5300004341000055
:1052f0004e5f0000454e0000414200004c4500005a
:105300003a20000000480000434900005f430000cd
:105310004d4400005f4900004e5100005549000017
:10532000525900003a2000000048000043490000a4
:105330005f4300004d4400005f4300005245000001
:1053400041540000455f0000434f00004e4e0000f6
:1053500045430000544900004f4e00003a20000031
:1053600000480000434900005f4300004d44000036
:105370005f4100004343000045500000545f0000bf
:10538000494e0000434f00004d4900004e470000c9
:105390002e200000524f00004c450000204300002a
:1053a000484100004e4700004520000052450000e3
:1053b000515500004553000054450000443a000098
:1053c0002000000048430000495f0000434d0000fa
:1053d000445f000053430000414e00005f44000062
:1053e00049530000414200004c4500003a200000b3
:1053f000004c0000494e00004b5f00004b45000090
:10540000595f000052450000504c0000593a00001e
:1054100020000000534300004944000020430000e6
:10542000545200004c2000003d200000004c0000c1
:1054300032430000415000005f4300004f4e000027
:105440004e450000435400005f52000045530000e9
:1054500050300000313a0000200000004c320000c3
:1054600043410000505f0000434f00004e460000e3
:10547000494700005f5200004551000030310000f4
:105480003a200000004c0000324300004150000070
:105490005f4300004f4e000046490000475f000098
:1054a0005245000053500000303100003a20000007
:1054b000004c000032430000415000005f440000f7
:1054c00049530000434f00004e4e0000454300008a
:1054d000545f000053440000505f0000524500003c
:1054e000513a0000200000004c320000434100000f
:1054f000505f000044490000534300004f4e00003d
:105500004e450000435400005f5200004553000028
:1055100050300000313a0000200000004c32000002
:1055200043410000505f0000434f00004e4e00001a
:1055300045430000545f0000524500005131000017
:10554000313a0000200000004c32000043410000ce
:10555000505f0000434f00004e4e000045430000e6
:10556000545f0000524500005350000031310000ec
:105570003a200000004c000032430000415000007f
:105580005f4300004f4e000046490000475f0000a7
:105590005245000051310000313a00002000000067
:1055a0004c32000043410000505f0000434f0000b8
:1055b0004e460000494700005f520000455300007e
:1055c00050310000313a0000200000005343000039
:1055d00049440000204400004154000041200000e4
:1055e0003d200000004c000032430000415000000c
:1055f0005f4300004f4e00004e4500004354000042
:105600005f5200004553000050310000333a000063
:10561000200000004c32000043410000505f0000b9
:10562000434f00004e460000494700005f52000013
:1056300045510000313300003a200000004c0000ca
:1056400032430000415000005f4300004f4e000015
:1056500046490000475f00005245000053500000db
:10566000313300003a20000000470000455400009c
:1056700020460000454100005455000052450000fe
:105680002030000078300000322000002850000058
:10569000533400005f420000545f0000494e000098
:1056a00049540000293a0000200000004c3200005c
:1056b00043410000505f0000444900005343000094
:1056c0004f4e00004e450000435400005f44000070
:1056d00041540000415f000052450000535000005b
:1056e0003a200000004c000032430000415000000e
:1056f0005f44000049530000434f00004e4e00003d
:1057000045430000545f000043540000524c000029
:105710005f52000045530000503a00002000000096
:105720004c32000043410000505f0000444900003b
:10573000534300004f4e00004e450000435400000c
:105740005f44000041540000413a00002000000086
:1057500048430000495f00004449000053430000f3
:105760004f4e00004e450000435400003a20000018
:10577000005500006e6b00006e6f0000776e000039
:1057800020440000656d00006f200000537400008d
:1057900061740000652e00000a0d00000052000038
:1057a000656100006420000042610000636b00003e
:1057b0002041000044440000522e00000a0d000069
:1057c0000057000061690000746900006e67000006
:1057d000206600006f72000020720000656100000a
:1057e00064200000746f0000206300006f6d0000f3
:1057f000706c000065740000652e00002e2e000005
:10580000005000006169000072200000436f00003a
:105810006e740000726f00006c6c00006572000016
:105820002077000069740000682000006c610000af
:1058300073740000204200006c7500006574000065
:105840006f6f000074680000206400006f6e00003d
:10585000676c0000652e00002e2e00000a0d00006f
:105860000057000061690000746900006e67000065
:10587000206600006f72000020770000726900004f
:1058800074650000207400006f200000636f00004a
:105890006d7000006c650000746500002e2e000025
:1058a0002e000000446f00006e6500002e200000f6
:1058b0000044000065760000696300006520000078
:1058c00057720000697400006520000045720000f6
:1058d000726f000072200000210d00000a0000001d
:1058e000536500007420000052650000706f0000d6
:1058f000727400002030000078310000343a00005b
:1059000000530000756300006365000073730000be
:105910002e0a00000d000000496e000069740000ae
:10592000696100006c6900007a6500002043000096
:105930006f6e0000747200006f6c00006c650000f8
:10594000722e00000a0d0000002000002d20000033
:105950004465000076690000636500002052000085
:10596000656100006420000045720000726f000055
:1059700072200000210d00000a00000047650000b1
:105980006e6500007269000063200000646500001d
:105990006d6f000020640000657600006963000000
:1059a00065200000617400007461000063680000fd
:1059b00065640000202d0000206500007665000071
:1059c0006e7400002c200000646500007669000001
:1059d00063650000416400006472000065730000ac
:1059e000733d0000000d00000a0000004765000044
:1059f0006e650000726900006320000064650000ad
:105a00006d6f00002064000065760000696300008f
:105a10006520000064650000746100006368000098
:105a200065640000202d0000206500007665000000
:105a30006e7400000d0a0000000d00000a2a00002c
:105a40002a2a00002a2a00002055000053420000a4
:105a500020450000727200006f720000202d0000cf
:105a60002068000075620000732000006172000071
:105a7000652000006e6f0000742000007375000048
:105a8000707000006f7200007465000064200000f8
:105a90002a2a00002a2a00002a0d00000a0000001d
:105aa0000d0a00002a2a00002a2a00002a200000ed
:105ab000555300004220000045720000726f000044
:105ac000722000002d20000064650000766900004f
:105ad0006365000020690000732000006e6f000005
:105ae0007420000073750000707000006f72000079
:105af00074650000642000002a2a00002a2a0000a1
:105b00002a0d00000a0000000d0a00002a2a0000e9
:105b10002a2a00002a2000005553000042200000dd
:105b200045720000726f0000722000002d200000fe
:105b3000636100006e6e00006f740000206500005d
:105b40006e7500006d6500007261000074650000f4
:105b50002064000065760000696300006520000095
:105b60002a2a00002a2a00002a0d00000a0000004c
:105b70000d0a00002a2a00002a2a00002a2000001c
:105b8000555300004220000045720000726f000073
:105b9000722000002d200000636c00006965000089
:105ba0006e740000206400007269000076650000d9
:105bb00072200000696e00006974000069610000d5
:105bc0006c6900007a610000746900006f6e00006b
:105bd00020650000727200006f720000202a000031
:105be0002a2a00002a2a00000d0a0000000d0000e9
:105bf0000a2a00002a2a00002a2a00002055000054
:105c00005342000020450000727200006f720000d5
:105c1000202d0000206f000075740000206f000030
:105c2000662000006865000061700000206d0000c3
:105c3000656d00006f720000792000002a2a0000c4
:105c40002a2a00002a0d00000a0000000d0a0000a8
:105c50002a2a00002a2a00002a20000055530000aa
:105c60004220000045720000726f000072200000a8
:105c70002d200000756e0000737000006563000049
:105c80006966000069650000642000002a2a00009f
:105c90002a2a00002a0d00000a000000332e00000e
:105ca00030310000003a0000204300006f75000012
:105cb0006c640000206e00006f740000206900001a
:105cc0006e69000074690000616c0000697a000070
:105cd000652000007379000073740000656d00009a
:105ce0002e20000020480000616c00007469000054
:105cf0006e6700002e0000000d0a00000d0a000073
:105d00002a20000053650000727600006f530000e7
:105d1000686f0000636b0000203200002046000026
:105d2000697200006d77000061720000652000005c
:105d30005265000076200000002000002a0d0000bf
:105d40000a0000003d5000007265000073730000ff
:105d50002027000045730000632700002069000031
:105d60006e200000636f00006e7300006f6c000017
:105d700065200000746f000020640000697300005b
:105d8000706c0000617900002071000075690000ee
:105d9000636b000020720000656600006572000001
:105da000656e0000636500002067000075690000f3
:105db000646500003d0a00000d0a00000d000000af
:105dc000204300006f7500006c640000206e00002e
:105dd0006f740000206900006e69000074690000a3
:105de000616c0000697a00006520000055530000d6
:105df000422e000020200000486100006c7400006a
:105e0000696e0000672e0000004300006972000008
:105e10006375000069740000205400006573000081
:105e2000742000004d6f0000646500002e0a000021
:105e30000d00000046690000726d000077610000ef
:105e400072650000204300006f640000653a0000a6
:105e5000200000004e65000077200000465700003b
:105e60002044000065740000656300007465000054
:105e7000642e00000a0d0000004c00006f6100005d
:105e80006465000064200000536100007665000036
:105e9000642000005365000074740000696e000007
:105ea000677300002e2000000a0d0000004400006f
:105eb00069730000636f00006e6e00006563000090
:105ec000746900006e6700002e2e00002e0a00008c
:105ed0000d000000496400006c65000020540000c3
:105ee000696d0000656f0000757400002e0a0000e7
:105ef0000d00000053740000616300006b4500005a
:105f0000727200006f720000004d000061740000aa
:105f10006820000045720000726f000072000000ef
:105f2000535000004920000042750000732000001b
:105f30004d6f000064650000203000000a0d000075
:105f4000005300005049000020420000757300001b
:105f5000204d00006f64000065200000310a000041
:105f60000d00000053500000492000004275000061
:105f7000732000004d6f00006465000020320000b7
:105f80000a0d0000005300005049000020420000ac
:105f900075730000204d00006f6400006520000054
:105fa000330a00000d00000045520000524f00006f
:105fb00052200000535000004920000042550000cc
:105fc000532000004d4f0000444500000a0d000022
:105fd00000000000496e00006974000020330000da
:105fe000442000004d6f000075730000650a00003a
:105ff0000d000000496e000069740000205400008c
:106000006872000075730000746d00006173000019
:1060100074650000720a00000d0000005465000065
:10602000737400002043000061730000653a0000b3
:10603000200000000a0d0000005500006e6b0000fb
:106040006e6f0000776e0000204300006173000057
:10605000650a00000d0000003031000032330000fe
:106060003435000036370000383900004142000066
:1060700043440000454600004144000044520000f3
:10608000204e00006f740000206600006f75000055
:086090006e6400002e00000008
:020000040000fa
:10609800881f78000000eb008008880011a1a90083
:1060a80010c1a9000111200091407800f2ccb30082
:1060b80082c060000144a0008000fd0010e1b7002c
:1060c8008000fd001061a9001021a9003008880097
:1060d80080007800074329006600200085412900d8
:1060e800140020000340290082bb200061807b004f
:1060f8000608780061807a000408780061807900d9
:10610800020878008180e800f88f5000f7ff3a0015
:10611800a0002000400d8800f0032000900c8800ab
:10612800e00c8800300d8800800d8800d00d8800b4
:10613800200e8800700e8800c00e8800100f88009e
:1061480011e1a80000a02600810120008aed0700c7
:1061580008c42900a80c880000d0270001002000ee
:1061680085ed0700f80c880000d02700010020000a
:1061780081ed0700480d880000d0270001002000ad
:106188007ded0700980d880000d027000100200051
:1061980079ed0700e80d880000d0270001002000f5
:1061a80075ed0700380e880000d027000100200098
:1061b80071ed0700880e880000d02700010020003c
:1061c8006ded0700d80e880000d0270001002000e0
:1061d80069ed0700280f8800d5c6bf0008ccb300ba
:1061e800084060002041b300d5e6b70092a1a9009d
:1061f80000a02600810120005fed0700dac6bf007d
:10620800084060003041b300dae6b7009ca1a9005d
:1062180000a026008101200057ed0700d3c6bf006b
:10622800084060004041b300d3e6b700a6a1a9002a
:1062380000a02600810120004fed0700dbc6bf004b
:10624800084060005041b300dbe6b700b0a1a900e8
:1062580000a026008101200047ed0700d2c6bf003c
:10626800084060006041b300d2e6b700baa1a900b7
:1062780000a02600810120003fed0700dcc6bf001a
:10628800084060007041b300dce6b700c4a1a90073
:1062980000a026008101200037ed0700cdc6bf0011
:1062a800084060008041b300cde6b700cea1a90048
:1062b80000a02600810120002fed0700c1c6bf0005
:1062c800084060009041b300c1e6b700d8a1a9001a
:1062d80000a026008101200027ed0700c0c6bf00ee
:1062e800084060003042b300c0e6b700e2a1a90050
:1062f8000001eb009208880013a1a90012c1a900af
:1063080012c1bf00f1ccb300014060000044a000fe
:1063180012e1b7001221a9005208880013e1a80071
:106328009500a80070c0b300a860b7004f047800bb
:1063380000000600889fbe008a9fbe008c9fbe009a
:10634800800578000006eb000d0120007860b90098
:10635800a2972000000441008d0478000005eb009e
:106368000b00e0000900320089007800180078006e
:10637800d7eb07008080fb000004e0000600320035
:1063880001007800e93007000300370009007800b1
:106398001cea0700000c780009007800e3300700c9
:1063a80080442900a43007000c007800df30070083
:1063b800a0442900a03007000a007800db3007005d
:1063c800c04429009c300700380078004f3107008e
:1063d800f0442900983007008904e8000a05e8001d
:1063e800ec0f5500deff3a000c06e800ec8646008c
:1063f800ec0f5600d5ff3a008006eb00c368dd00bd
:10640800a08e200000854000090478000006eb00fb
:106418000b00e00004003200880078001a007800c1
:10642800abeb07000300370008007800f5e9070028
:10643800000d780008007800bc30070020452900ce
:106448007d3007000d007800b8300700a04429000f
:10645800793007000c007800b4300700c0442900e8
:10646800753007003a00780028310700f044290009
:10647800713007008800e8000c06e800e40f5600b9
:106488000200320001047800e1ff37008d06e800c1
:10649800e4844400f28f5600d8ff3a000b00e00075
:1064a800030032004047800089eb070003003700f3
:1064b80001007800d3e90700404788008880e80099
:1064c8000b00e000030032001046800080eb07005c
:1064d8000300370001007800cae907001046880069
:1064e800e30044000b00e000030032000046800097
:1064f80077eb07000300370001007800c1e90700c7
:1065080000468800e40044000b00e000030032006d
:10651800f04580006eeb07000300370001007800ab
:10652800b8e90700f0458800e50044000b00e000ea
:1065380003003200e045800065eb070003003700e8
:1065480001007800afe90700e0458800e600440054
:106558000b00e00003003200d04580005ceb070030
:106568000300370001007800a6e90700d04588003d
:10657800e70044000b00e0000300320010408000f8
:1065880053eb070003003700010078009de907007e
:1065980010408800e80044000b00e00003003200cf
:1065a800c04580004aeb070003003700010078006f
:1065b80094e90700c0458800e90044000b00e000aa
:1065c80003003200b045800041eb070003003700ac
:1065d800010078008be90700b0458800ea00440014
:1065e8000b00e000030032000040800038eb070099
:1065f800030037000100780082e9070000408800a6
:10660800404529000c30070000408000bf300700db
:10661800f0442900083007006b00440043300700ad
:1066280090452900043007004f06be004f05be0004
:106638004f04be0000000600f0462900fe2f0700a8
:106648000000eb003bff0700b0482900fa2f370095
:1066580020492900f82f07001000200035ff070007
:10666800504a2900f42f3700a097200000000600a8
:10667800a08e200000000600f04580000000060003
:10668800889fbe008a9fbe008c1f78008005780016
:10669800010678000005eb00e18f550004003a0080
:1066a8000c0478002a012000290020000a00370085
:1066b800e28f550006003a000a004500418c200090
:1066c800010040000048eb008040eb0011409800ba
:1066d8000a0478008a0478004340dd000080e8005e
:1066e800a18e200060807800e20f50003800320050
:1066f80005003e000000e00008003200e10f5000f5
:10670800bc003a0010003700e30f5000630032006d
:10671800e40f5000b7003a006a003700912b0700d9
:1067280008014400c184200001014100898044001f
:10673800808040009181fb00114090004800dd00fe
:10674800030070001e0037008a2b07008980440070
:10675800808040001181fb00114090004800dd005e
:10676800020070000d00320088004400408c2000b8
:10677800008140008001eb009280fb0012409000f5
:106788004800dd000100700001003a0013002000fd
:10679800034978004818de001041980008004400ba
:1067a800c284200002014000418c2000010040000a
:1067b8009080fb00104090004800dd000100700050
:1067c800004978004800de00104198008900370031
:1067d800682b070089804400808040001181fb00fd
:1067e800114090004800dd00020070000b003200ec
:1067f8000801440081822000810041000040eb0034
:10680800e14870008041780090409800c0842000e2
:106818000001410011497800134198000802440022
:1068280080822000800142009380fb00134090008a
:106838004800dd0001017000100032004340dd0017
:1068480064004000a18e200060807800800f510015
:106858000a003e00c0842000000042008040eb0097
:1068680061c87000114098000200e8008049780073
:106878004800de00904198005e003700080144009f
:1068880080822000000041000048eb008040eb00bf
:1068980011409800c084200053003700312b0700b6
:1068a80089804400808040001181fb0011409000e5
:1068b8004800dd00020070004400320088024400f5
:1068c8001d0037002b2b0700898044008080400082
:1068d8001181fb00114090004800dd0002007000ab
:1068e8000d00320088004400408c200000814000e8
:1068f8008001eb009280fb00124090004800dd0010
:106908000100700001003a001300200003497800dc
:106918004818de001041980088024400408c20008e
:10692800008042009080fb00104090004800dd008d
:1069380001007000250032008082200000804200a3
:106948009080fb00104090004800dd0001027000bc
:106958004340dd00e6004000a38e200061817900fd
:10696800801f7800110009000282d8004f007800cb
:106978006400400060807900808f5000050031007d
:10698800c0842000008042008040eb0061c8700095
:106998000500370008004400c184200001004000c1
:1069a8000048eb008040eb0011409800880044004c
:1069b80080822000808040000400e8008048780041
:1069c8004800de00904098000a00370008014400a3
:1069d800c0842000000041000048eb008040eb002c
:1069e8001140980080822000000141000149780090
:1069f80011419800c340dd00a08e2000610278009c
:106a0800e10f52000d003a0088004400c0842000c5
:106a1800008140008001eb009280fb001240900052
:106a28004800dd000100700001003a008401780090
:106a3800034978004818de00104198000a05e8006c
:106a4800f10f550014ff36008001eb004480200050
:106a5800c5842000f80f2000038041000401400095
:106a6800050040009080fb00104090004800dd00c9
:106a780001007000084960004800de0010419800dd
:106a88008301e800f28f5100f3ff3a000400780018
:106a9800b82d0700bc2e0700104890000048a3003e
:106aa80006003200b82e07004060900061006000c8
:106ab800080060000ce8b7000d68ef00b22e070070
:106ac800104890000058a30006003200ae2e0700c0
:106ad800406090000000d100610060000ee8b7003f
:106ae8000f68ef00a82e0700104890000068a30068
:106af80006003200a42e0700406090004200de002d
:106b08006100600010e8b7001168ef009e2e0700d2
:106b1800104890000004e00006003d009a2e07008f
:106b2800406090004300de006100600012e8b7009a
:106b38001368ef00942e0700204890000008a30077
:106b480006003200902e0700406090004400de00ee
:106b5800610060001ce8b7001d68ef008a2e07007e
:106b6800204890000018a30006003200862e070077
:106b7800406090004500de00610060001ee8b7003c
:106b88001f68ef00802e0700204890000028a3000f
:106b9800060032007c2e0700406090004600de00b0
:106ba8006100600020e8b7002168ef00762e07003a
:106bb800204890000038a30006003200722e07001b
:106bc800406090000080fb004700de0022e8b7002c
:106bd8002368ef006c2e0700204890000048a300af
:106be80005003200682e07005060900061006000c8
:106bf80018e8b7001968ef00632e070020489000d6
:106c08000058a300060032005f2e07005060900075
:106c18000000d100610060001ae8b7001b68ef00af
:106c2800592e0700204890000068a3000600320093
:106c3800552e0700506090004200de0061006000a1
:106c480014e8b7001568ef004f2e070020489000a1
:106c58000004e00006003d004b2e07005060900045
:106c68004300de006100600016e8b7001768ef0017
:106c7800452e0700304890000008a30006003200a7
:106c8800412e0700506090004400de006100600063
:106c980006e8b7000768ef003b2e07003048900071
:106ca8000018a30006003200372e0700506090003d
:106cb8004500de006100600008e8b7000968ef00e1
:106cc800312e0700304890000028a300060032004b
:106cd8002d2e0700506090004600de006100600025
:106ce80004e8b7000568ef00272e07003048900039
:106cf8000038a30006003200232e070050609000e1
:106d08000080fb004700de000ae8b7000b68ef00d0
:106d18001d2e0700304890000048a30005003200ef
:106d2800192e0700606090006100600026e8b70037
:106d38002768ef00142e0700304890000058a30081
:106d480006003200102e0700606090000000d1009d
:106d58006100600024e8b7002568ef00c1802000ca
:106d6800914078008180fb000dc8bf004800dd001d
:106d78000100700002003200dc42a8000100370068
:106d8800dc42a900e1802000914078008180fb006e
:106d98000fc8bf004800dd0001007000020032008b
:106da800dc62a80001003700dc62a9000181200034
:106db800914078008180fb0011c8bf004800dd00c9
:106dc8000100700002003200dc82a80001003700d8
:106dd800dc82a90021812000914078008180fb009d
:106de80013c8bf004800dd00010070000200320037
:106df800dca2a80001003700dca2a900c1812000a4
:106e0800914078008180fb001dc8bf004800dd006c
:106e18000100700002003200e402a80001003700ff
:106e2800e402a900e1812000914078008180fb0004
:106e38001fc8bf004800dd000100700002003200da
:106e4800e422a80001003700e422a9000182200002
:106e5800914078008180fb0021c8bf004800dd0018
:106e68000100700002003200e442a800010037006f
:106e7800e442a90021822000914078008180fb0033
:106e880023c8bf004800dd00010070000200320086
:106e9800e462a80001003700e462a90081812000b3
:106ea800914078008180fb0019c8bf004800dd00d0
:106eb8000100700002003200ec02a8000100370057
:106ec800ec02a900a1812000914078008180fb009c
:106ed8001bc8bf004800dd0001007000020032003e
:106ee800ec22a80001003700ec22a9004181200013
:106ef800914078008180fb0015c8bf004800dd0084
:106f08000100700002003200dcc2a8000100370056
:106f1800dcc2a90061812000914078008180fb00db
:106f280017c8bf004800dd000100700002003200f1
:106f3800dce2a80001003700dce2a9006180200043
:106f4800914078008180fb0007c8bf004800dd0041
:106f58000100700002003200d5a2a800010037002d
:106f6800d5a2a90081802000914078008180fb0093
:106f780009c8bf004800dd000100700002003200af
:106f8800d5c2a80001003700d5c2a9004180200061
:106f9800914078008180fb0005c8bf004800dd00f3
:106fa8000100700002003200ec62a8000100370006
:106fb800ec62a900a1802000914078008180fb004c
:106fc8000bc8bf004800dd0001007000020032005d
:106fd800dc22a80001003700dc22a9006182200021
:106fe800914078008180fb0027c8bf004800dd0081
:106ff8000100700002003200cc62a80001003700d6
:10700800cc62a90041822000914078008180fb0079
:1070180025c8bf004800dd000100700002003200f2
:10702800e482a80001003700e482a9004f06780036
:107038004f05be004f04be00000006008f0ab000d6
:10704800889fbe008a9fbe008c9fbe008e1f78005e
:107058008004eb000b8720002a98200047290700ae
:1070680089804400808040001181fb00114090001d
:107078004800dd000b047800820d70006680540023
:10708800e30f5000cc003e002a0090000000e00012
:1070980040003a00e68f540002003200e88f5400a6
:1070a8001a003a001a0090000000e0000e003a00b2
:1070b8001a0078000000e00004003a0031290700b7
:1070c8009080fb00104090000d003700e10f500049
:1070d800b9003a002b290700504990000281fb00b3
:1070e800604890001e003700e10f5000b2003a00df
:1070f80024290700c04090008180fb005040900088
:107108004800dd00010c7000ab003700e78f540029
:1071180002003200e98f5400a7003a001a009000dc
:107128000000e00014003a001a0078000000e000b7
:1071380005003a0013290700a04090008180fb0059
:1071480030409000eeff3700e10f50009a003a00ff
:107158000c290700704990000281fb000050900044
:107168004800dd0002007000620420000280b900bf
:10717800000c780090003700e10f50008e003a00b4
:1071880000290700e04090008180fb0070409000db
:10719800dbff3700e10f500087003a00e68f54000c
:1071a80020003a00a05080000000e00014003a00df
:1071b800905080000000e00005003a00f128070028
:1071c800b05090008180fb004050900012003700c2
:1071d800e10f500078003a00ea28070000619000ab
:1071e8000281fb00106090004800dd000200700082
:1071f800620420000280b900e04388006e00370076
:10720800e10f50006c003a00de280700f0509000b3
:107218008180fb00005890004800dd0001007000ec
:10722800f5ff3700e78f540020003a0060518000d6
:107238000000e00014003a00505180000000e00017
:1072480005003a00cf280700d05090008180fb004d
:107258006050900012003700e10f500056003a00cd
:10726800c8280700206190000281fb003060900070
:107278004800dd0002007000620420000280b900ae
:10728800f04388004c003700e10f50004a003a00f4
:10729800bc280700905890008180fb00205890007f
:1072a8004800dd0001007000f5ff3700e88f54004a
:1072b80020003a00205280000000e00013003a004d
:1072c800105280000000e00005003a00ad280700d9
:1072d800e06090008180fb00706090001100370032
:1072e800e10f500034003a00a628070030719000e2
:1072f8000281fb00407090004800dd000200700031
:10730800620420000280b90008003700e10f500035
:1073180029003a009b280700a06890008180fb00a4
:10732800306890004800dd000100700000448800cb
:1073380021003700e98f54001f003a00e052800016
:107348000000e00013003a00d05280000000e00086
:1073580005003a008b280700806890008180fb00b8
:107368001068900011003700e10f500012003a0039
:1073780084280700507190000281fb006070900023
:107388004800dd0002007000620420000280b9009d
:1073980008003700e10f500007003a00792807007d
:1073a800c06890008180fb00506890004800dd00b4
:1073b80001007000104488008904e8008b85e8000b
:1073c80078054500ec8f540024ff3a00692807002f
:1073d800a04090008180fb00304090004800dd0014
:1073e80001007000e10f500005003a008000eb003a
:1073f800a208e20001003a008000780011458800e8
:107408005c280700c04090008180fb00504090003d
:107418004800dd0001007000e10f500005003a004f
:107428008000eb00a008e20001003a00800078002c
:107438000145880010408000e10f5000050036002b
:10744800000040006400400001872000b243800033
:1074580002b07800c3982000e3a79f000007eb0064
:107468000c872000aa98200044e32000d4a79f009e
:107478004d00200085882000c5a79f002b9820007c
:10748800bba79f00e48456006fa49700110020005a
:10749800988f10000e003a00322807008060900094
:1074a8008180fb00106090004800dd000100700042
:1074b800070032002f280700a04090008180fb00c1
:1074c800304090004800dd000100700011003a00d3
:1074d80022002000980f110019003a002128070007
:1074e800806090008180fb00106090004800dd0003
:1074f80001007000120032001e280700c0409000f2
:107508008180fb00504090004800dd0001007000c1
:107518000b003200dfa197001300be0042062000d6
:107528000300200008e407000001be0020059800c1
:107538008d0078000200780065e707003400370006
:10754800bfa59700150020009b8f12001f003a006e
:10755800988f120007003a0006280700a040900004
:107568008180fb00304090004800dd000100700081
:107578000d003a00100020009b0f100013003a0085
:1075880021002000988f100010003a00f92707000a
:10759800c04090008180fb00504090004800dd0012
:1075a80001007000090032000d00780095e5070021
:1075b8008000780020059800400620000008b800e8
:1075c8005fa197000089be00110037001b00e00092
:1075d8000d003a0018007800e20f500002003a004f
:1075e8000045800003003700e10f500006003a0014
:1075f80010458000e10f500003003a00cfa197002a
:10760800130e7800020037004fa297001c0a78007a
:107618007c2a0700e30f500003003200e40f5000fb
:10762800ca003a0032003700e78f54006a0032007f
:1076380005003e00e48f54002a003900e58f54000d
:107648000900360054003700e98f540084003200e6
:1076580071003900ea8f54000b003200eb8f5400a0
:1076680020003a00150037009c0278009a805200ea
:1076780044003700d0508000808050003d01370022
:1076880090518000fcff3700ecc2bf000008a30047
:1076980003003200ecc2bf000018a30088003200cb
:1076a800ecc2bf000008a30090003a00ecc2bf0083
:1076b8000018a3008a003a008c003700d5c2bf002a
:1076c8000058a30003003200d5c2bf000068a30021
:1076d8008e003200d5c2bf000058a30096003a00c1
:1076e8008f0037009c0578009a80550021013700eb
:1076f800e78f54003800320006003e00e58f540042
:107708001100320024003e00e48f54008c003a003f
:1077180008003700e98f5400510032003e0039005c
:10772800ea8f540060003200eb8f540084003a0066
:1077380070003700504f80007808b50001f82f001e
:10774800810040000b013700dcc2bf000068a300c5
:1077580005003200dc42e20003003500f10720009a
:1077680010508000c4ff3700dcc2bf000068a300cf
:1077780007003a00dc42e20005003d00020aee0084
:107788008000780000f82f0080804000f900370062
:1077980011508000f7003700dcc2bf000058a3007a
:1077a80004003200dcc2bf00f10720000038a3004b
:1077b800b0ff3200dcc2bf000058a30004003a004a
:1077c800dcc2bf0001f82f000038a300a9ff3a006f
:1077d800d1508000e7003700dcc2bf000028a300ba
:1077e80004003200dcc2bf00f10720000048a300fb
:1077f800a3ff3200dcc2bf000028a30004003a0047
:10780800dcc2bf0001f82f000048a3009cff3a002b
:1078180091518000d7003700e4c2bf000038a300b0
:1078280004003200e4c2bf00f10720000018a300e2
:1078380007003200e4c2bf000038a30006003a0087
:10784800e4c2bf000018a3000300320001f82f00b3
:107858005052800088ff370051528000c500370021
:10786800e4c2bf000008a30004003200e4c2bf0065
:10787800f10720000028a30007003200e4c2bf007f
:107888000008a30006003a00e4c2bf000028a300d5
:107898000300320001f82f001053800076ff3700f4
:1078a80011538000b3003700ecc2bf000008a300ea
:1078b80005003200d5c2bf000058a30002003a00fc
:1078c800f107200007003700ecc2bf000008a30042
:1078d80006003a00d5c2bf000058a30003003200da
:1078e80001f82f00d053800063ff3700d153800088
:1078f800a0003700ecc2bf000018a300050032004a
:10790800d5c2bf000068a30002003a00f1072000ba
:1079180007003700ecc2bf000018a30006003a00b9
:10792800d5c2bf000068a3000300320001f82f0091
:107938009054800050ff3700915480008d0037002c
:107948001c0178009a0051008a003700e48f540027
:107958001a003900e58f540003003600e98f5400ff
:1079680016003e000f00370040478000e10f50002e
:1079780007003a00c04380007a08b50022002000c2
:10798800110009000200d8008000fd000d0037003a
:107998009c0178009a80510000f82f0080804000f8
:1079a800080037001c0078002200200011000900a0
:1079b8000200d8009a005000020037001c0278002c
:1079c8009a0052003a009000e40f50003200320052
:1079d80006003e00e20f50001700320023003e0070
:1079e800e10f500063003a0006003700e60f500030
:1079f8004100320035003900e70f50005d003a00c1
:107a08004a003700dcc2bf000058a3000300320060
:107a1800dcc2bf000038a3004a003200dcc2bf004d
:107a28000058a30052003a00dcc2bf000038a3008f
:107a38004f0032004b003700dcc2bf000028a30013
:107a480003003200dcc2bf000048a3003d00320042
:107a5800dcc2bf000028a30045003a00dcc2bf001a
:107a68000048a300420032003e003700e4c2bf00d5
:107a78000038a30003003200e4c2bf000018a300ce
:107a880030003200e4c2bf000038a30038003a00da
:107a9800e4c2bf0031003700e4c2bf000008a30001
:107aa80003003200e4c2bf000028a3002500320012
:107ab800e4c2bf000008a3002d003a00e4c2bf00e2
:107ac8000028a3002a00320026003700ecc2bf00bd
:107ad8000008a30003003200ecc2bf000018a30096
:107ae80018003200ecc2bf000008a30020003a00d2
:107af800ecc2bf0019003700d5c2bf000058a30070
:107b080003003200d5c2bf000068a3000d00320098
:107b1800d5c2bf000058a30015003a00d5c2bf0067
:107b28000068a300120032000e003700ecc2bf004c
:107b38000038a30005003200dcc2bf000018a30013
:107b480002003a00f007200007003700ecc2bf002f
:107b58000038a30006003a00dcc2bf000018a300ea
:107b68000300320000f82f009a005000010037008f
:107b78009a00780015408000a5a79f00e18f520069
:107b8800050036000580e800808f540002003a00a6
:107b9800904e80009c0010008a0178000af097003f
:107ba8000082fb00848f50000200340004815000e2
:107bb800050037000400ea000001eb00808f500048
:107bc80001003d000481400013f097000080fb0095
:107bd80001002000cf91de007ae207007ab9970011
:107be8006a11b900cf91de00000041008180490090
:107bf80048f92f00088447000e0144000089be00a0
:107c08004bf62f008b8147000e8141000089be0092
:107c18006fa0970078004000e0a79f006407470026
:107c28000c86e80078054500dfa09700e480400056
:107c3800d1a79f008d06e8004fa197000281e800b8
:107c4800c2a79f003fa2970078024200b4a79f00f6
:107c580000032000800f57000afe3a00e545800027
:107c680085b79f00da458000baaf9f000f389700ac
:107c78009f3897006f339700ff3397000002430047
:107c880081824b00f4a79f0085af9f00060050003b
:107c98008780580090af9f00a1af9f004f3097009a
:107ca800df3097001301be000005410081854900bf
:107cb800caaf9f00dbaf9f000202500083825800ca
:107cc800e4af9f00f5af9f000002430081824b00a4
:107cd8000205520083855a009ab79f00abb79f00f0
:107ce8000402410085824900b4b79f00c5b79f00d0
:107cf8000600500087805800000241008182490038
:107d0800d4b79f00e5b79f00020050008380580059
:107d1800f0b79f0081bf9f008005eb004ee3200075
:107d280088067800cc972000afa297000500e000f5
:107d38001c003200e18f55000b00320005003900ad
:107d4800e28f55000d003200e38f550037003a00ee
:107d58000f0037007fb097008fb89700a08f9f0063
:107d6800b18f9f00310037005fb19700efb19700e6
:107d7800c28f9f00d38f9f002c0037003fb297001f
:107d8800cfb29700e48f9f00f58f9f002700370040
:107d98001fb09700afb0970080979f0091979f0002
:107da800220037008fb09700e18f50000e003a0094
:107db8000b00e00003003200e18f55000a003a0092
:107dc800050037006fa99700ffa99700a28f9f00b1
:107dd800b38f9f00040037004faa9700dfaa9700cf
:107de800c48f9f00d58f9f00bfaa9700e18f5200d4
:107df8000e003a00e28f550003003200e38f550071
:107e08000a003a00050037001fa89700afa897009e
:107e1800e08f9f00f18f9f00040037007fa197003b
:107e28008fa9970082979f0093979f002c0090003e
:107e3800160020000000e000010032000083eb0083
:107e48003c0090000000e0002d003a008c01780012
:107e58001c0090006a00b900cf80de000d01780098
:107e68001d02be00800f5200818f5a0002003400ac
:107e7800808ebe000600370060001000e080180009
:107e8800800f5200818f5a0001003d00808ebe0095
:107e9800130078006a00b90088bb20000004440081
:107ea800cfc4de006130b9001201be00c5e1070091
:107eb8000801400089814800c057210001002000c6
:107ec800800f5100818f5900020034000001be006c
:107ed80006003700341f2000840f5100e08f59003e
:107ee80002003c00421f2000030020000b804500d8
:107ef800c5f42f008f8242008232780036003700a6
:107f0800e10f500034003a000e0578006130b900e6
:107f18001d01be00abe107003e044000ae844800ee
:107f2800088fbe001c0178009c03900007004100e8
:107f3800863e20000680b900043e29004500200046
:107f48000000420081804a00070151000691b900f3
:107f58000201420083814a00800f5400818f5c0037
:107f680002003400008fbe0004003700820f540066
:107f7800838f5c0001003d00028fbe001a00be0026
:107f88000247260083002000820f5000838f58008c
:107f980002003400028dbe0007003700f2342c00c6
:107fa800820f5000e08f580003003c0000352c0081
:107fb80001002000008dbe000b8445001a00be00a1
:107fc80042062000030020005fe10700c3f42f00f1
:107fd8008f81410080317c008b05e80064074700f1
:107fe800e486460078064600ec8f55004eff3a00be
:107ff800017122000f309700810f500001003600f8
:1080080081379f00017122001f309700810f5000b7
:108018000100360091379f00017122002f30970030
:10802800810f500001003600a1379f00c0f42f00d7
:108038000f004000e9280700532907000048900076
:108048000008a300080032004f290700c04890002c
:108058008180fb00504890004800dd00010070005e
:1080680000004000e0279f004729070000489000d3
:108078000018a3000800320043290700e0489000d8
:108088008180fb00704890004800dd00010070000e
:1080980000004000f0279f003b290700004890009f
:1080a8000028a300080032003729070080509000fc
:1080b8008180fb00105090004800dd000100700036
:1080c80000004000802f9f002f29070000489000e3
:1080d8000038a300080032002b290700a0509000a8
:1080e8008180fb00305090004800dd0001007000e6
:1080f80000004000902f9f002329070000489000af
:108108000048a300080032001f290700c050900053
:108118008180fb00505090004800dd000100700095
:1081280000004000a02f9f0017290700004890007a
:108138000058a3000800320013290700e0509000ff
:108148008180fb00705090004800dd000100700045
:1081580000004000b02f9f000b2907000048900046
:108168000068a30008003200072907008058900023
:108178008180fb00105890004800dd00010070006d
:1081880000004000c02f9f00ff2807000048900013
:108198000004e00008003d00fb280700a0589000fc
:1081a8008180fb00305890004800dd00010070001d
:1081b80000004000d02f9f00f328070010489000cf
:1081c8000008a30008003200ef280700c0589000fc
:1081d8008180fb00505890004800dd0001007000cd
:1081e80000004000e02f9f00e7280700104890009b
:1081f8000018a30008003200e3280700e0589000a8
:108208008180fb00705890004800dd00010070007c
:1082180000004000f02f9f00db2807001048900066
:108228000028a30008003200d728070080609000cb
:108238008180fb00106090004800dd0001007000a4
:108248000000400080379f00cf28070010489000aa
:108258000038a30008003200cb280700a060900077
:108268008180fb00306090004800dd000100700054
:108278000000400090379f008000eb00024029007a
:1082880061007900c5f42f008f824200e5827800f2
:10829800050878008180e800f88f5000f8ff3a0060
:1082a8004f0778004f06be004f05be004f04be00c2
:1082b8008f0ab10000000600809fbe00821f780070
:1082c8003400f80000002000a00188000008e20047
:1082d80029003a00acc8bf00e14f50000c00320042
:1082e80005003900e24f500011003200e34f500002
:1082f8001f003a0015003700cd02a800aa0aed00b9
:10830800504588007008880010c0b3000600370088
:10831800cd02a900cd82a800a40aed00404588003e
:108328007008880020c0b300ace8b7002f00370001
:10833800cd82a900cda2a8009e0aed003045880094
:108348007008880030c0b300f7ff3700cda2a9003d
:1083580040458000aa08b400314580000100400073
:10836800c1c3290080805000214588007108880019
:10837800ac68ef001d00370040e6200011c0b300d4
:1083880090cf100014003a00cd02a800646eef00f0
:10839800c28a200012417800eb4f510009003e00cc
:1083a8000280fb000000400001402900e0807800c6
:1083b80060da2f0011004000700888000240e800d1
:1083c800d9ff37000071220070088800ac68ef0000
:1083d800cd82a90005003700cd02a9008025200024
:1083e8007008880010c0b30064eeb7008500a900cb
:1083f8003400f9004f0178004f00be00004006002d
:10840800881f780000047800d04a29008a280700cd
:1084180080c0b300504498000040eb0060449800ce
:1084280078409000c1cfb3000140600070449800cc
:108438008ac9bf0010449800a2c9bf002044980010
:10844800bac9bf0030449800d2c9bf004044980060
:10845800eac9bf00004c980002cabf00104c98003f
:108468007acabf00305498007bcabf0040549800b5
:1084780092cabf007054980093cabf00005c98006d
:108488003860900001c8b300014070003064980063
:1084980078609000014070007064980008007800cf
:1084a800dc1e07003924070046200700db230700ed
:1084b80000468000e10f500003003a008000eb0006
:1084c80020002000010037006000b8006cf80700a9
:1084d800dafa07004f047800000006001046800012
:1084e80000000600c045800000000600b04580007e
:1084f800000006003c00fa00881f7800000478009d
:1085080020fc2f000f004000816629001d00090093
:1085180031187800c003b100406a2900fd0f5400eb
:108528000e003e00206c2900432807000800780050
:108538007e280700a0c3b3003828070000c2b30094
:10854800362807000800440021fc2f0080804000e6
:1085580061807f0038280700f0442900362807008a
:108568004f0478000080fa0000000600889fbe00d3
:108578008a1f780000057800010478000000e000f8
:1085880006003a00b06c29002b2807000800780084
:10859800d8ff07008a44780012003700906e29003f
:1085a800252807008000eb00414788001146880015
:1085b8000146880000a62e00f0458800e1458800a5
:1085c800d14588001140880010002000c04588006f
:1085d800b0002000b0458800014088000104780000
:1085e80002003700eb0f540029003e007840b90024
:1085f8000081e800a19720008001eb0003b178001a
:1086080064024000d207200002b278000102400054
:10861800034a7800a2c0b3001242980066014000e5
:1086280003b178006801400003b178006a01400096
:1086380003b178006c0240001200200002b27800fa
:108648006e01400003b17800f002400083b2780068
:108658007201400003b178007402400082bb200020
:1086680002b278007600400003b07800e30f5400af
:1086780002003e000008200080b27800e4004400b8
:1086880080bb200012e30700804478000d0037000b
:108698006c0054004300dd00a28e20008001eb0036
:1086a800033079008080e80083307900e4014000dd
:1086b800510020008131790066004000410120000e
:1086c800013079000804e800fd0f540002003e0064
:1086d800e10f5500c3ff32000904e0000600320034
:1086e80090702900d427070009407800dd2707008b
:1086f800f0442900d0270700b0482900ce270700fa
:108708004f0578004f04be0000000600889fbe0099
:108718008a1f780000057800b408e2001e003a00bd
:10872800922307009080fb00104090004800dd0075
:108738000100700013003a008c230700806090004d
:108748008180fb00106090004800dd00010470008b
:108758000c003a00e0712900b7270700100020003c
:10876800a04588008845880098458800080078005a
:1087780060ff07008800780008007800c0f707004d
:1087880005003700b408e20003003a00200020008a
:108798002c240700d0053700b228ec00712307000d
:1087a800c04090008180fb00504090004800dd00f0
:1087b8000100700084003a006a230700a04090007e
:1087c8008180fb00304090004800dd00010070000f
:1087d8007d003a0067230700e05090008180fb008d
:1087e800705090004800dd00010070000800320061
:1087f800814580008100e800e201200011000900a5
:108808008280d8008000fd008045880039ff07007d
:1088180058230700c05090008180fb005050900002
:108828004800dd00010070000e0032008045800025
:108838000000e00002003a00d001200001003700eb
:108848000000e9008045880081458000e2012000a1
:10885800110009008280d8008000fd008045880052
:1088680024ff070084458000a600200011000900ad
:108878000682d80000027800010078006a21b90059
:108888007422b9008241780004417800864078005b
:1088980046230700352307009080fb001040900016
:1088a8004800dd000100700041062000810f5000e3
:1088b8000b003a002b230700e04090008180fb006a
:1088c800704090004800dd000100700004003a008c
:1088d8008145800025ff070050002000d9230700ac
:1088e800222307009080fb00104090004800dd0024
:1088f80001007000c1122000810f50000b003a00e7
:1089080018230700e04090008180fb007040900031
:108918004800dd008100700004003a0010002000cb
:1089280012ff0700a0002000c62307000f2307003e
:10893800e04090008180fb00704090004800dd001e
:108948000100700041062000810f50000c003a0021
:10895800042307009080fb00104090004800dd00d1
:108968000100700006003a0039f7070010002000e7
:108978007045880050002000b22307000701370027
:10898800f8220700e04090008180fb0070409000d2
:108998004800dd000100700003003a0070458000c7
:1089a800e10f5000020032000a00e000fb003a002c
:1089b80060762900202707000000eb00a04588000a
:1089c8007045880045053700e6220700c040900042
:1089d8008180fb00504090004800dd0001007000dd
:1089e80053003200df220700a04090008180fb0086
:1089f800304090004800dd00010070004c003a0053
:108a0800dc220700805890008180fb0010589000fd
:108a18004800dd000100700024003200c208ec00ac
:108a28006300600010468800e10f50000b00320020
:108a380005003900e20f50000f003200e30f50002c
:108a480018003a0012003700d0772900fa260700ec
:108a580041e2a90042c2a9000b003700e0782900d2
:108a6800f526070041e2a90042c2a9004302a90075
:108a780041e2a8000d003700f0792900ee26070032
:108a880041e2a90042c2a8004302a800f8ff37004b
:108a9800007b2900e826070041e2a90042c2a8009d
:108aa800f2ff3700107c2900e3260700b1220700f7
:108ab800c05890008180fb00505890004800dd00ad
:108ac8000100700009003200be08e20004003a000c
:108ad80000a62e00f0458800607d290002003700be
:108ae800be28ef00507f2900d3260700a1220700e7
:108af800806090008180fb00106090004800dd00dd
:108b080001007000a5003200c008ee00c008b700e0
:108b18004f00de00610010000046880002003200ad
:108b2800f08029009c003700608329009a003700f4
:108b38008c220700a04090008180fb00304090000c
:108b48004800dd0001007000940032008522070013
:108b5800c04090008180fb00504090004800dd003c
:108b6800010070008d003a0082220700a0489000a2
:108b78008180fb00304890004800dd000100700053
:108b88000b003a0079220700a04890008180fb0082
:108b9800304890004800dd000100700021032000eb
:108ba800810f500010003600b208ab000e003a00ea
:108bb800c0458000e90f500003003e000000e800b7
:108bc800c045880002003700200020001d23070050
:108bd8001086290098260700b8c8bf00a1260700fc
:108be800f04429009426070062220700e04890001c
:108bf8008180fb00704890004800dd000100700093
:108c08000b003a0059220700e04890008180fb00e1
:108c1800704890004800dd0001007000210320002a
:108c2800810f500010003600b208ab000e003a0069
:108c3800c04580000000e000030032000000e900a9
:108c4800c04588000200370020002000fd220700f0
:108c58001086290078260700b8c8bf0081260700bb
:108c6800f044290074260700422207009080fb0088
:108c7800104090004800dd0001007000350032000f
:108c8800b608ec00b0458800eb0f50000100360034
:108c9800b628ef002087290067260700b045800026
:108ca80001002000eb0f5000e08f580025003e0027
:108cb800006001000d0037000e0037000f0037007c
:108cc8001000370011003700120037000500370088
:108cd8001200370013003700140037001500370062
:108ce800160037006088290017003700b08829006f
:108cf80015003700f0882900130037006089290023
:108d080011003700d08929000f003700208a290078
:108d18000d003700808a29000b003700208b2900be
:108d280009003700908b290007003700e08b2900e5
:108d380005003700408c290003003700808c29008b
:108d480001003700008d29003b260700f044290068
:108d58003926070007220700e04090008180fb00c9
:108d6800704090004800dd00010070000b003200e8
:108d78000008ee000008b7004f00de006100100098
:108d880000408800608d29002b26070000408000e5
:108d980066260700f0442900272607008045800042
:108da800eb0f5000f5023e00ee210700c040900096
:108db8008180fb00504090004800dd0001007000f9
:108dc800ef003200e7210700a04090008180fb00ff
:108dd800304090004800dd0001007000e8003a00d3
:108de800e4210700a04890008180fb0030489000f3
:108df8004800dd00010070000b003a00db2107008d
:108e0800a04890008180fb00304890004800dd00b9
:108e18000100700021032000810f50001900360066
:108e2800b208ab0017003a00804580007800b9000e
:108e38006e014000a3972000e2807900700c2000aa
:108e4800808f500003003c000100e80000b1790069
:108e580002003700200020007a220700908e2900a7
:108e6800f5250700804580007800b9006e004000b5
:108e7800a29720006000790050260700f0442900de
:108e8800ed250700bb210700e04890008180fb002a
:108e9800704890004800dd00010070000b003a00a7
:108ea800b2210700e04890008180fb0070489000e4
:108eb8004800dd000100700021032000810f5000f0
:108ec80019003600b208ab0017003a008045800050
:108ed8007800b9006e014000a3972000e280790075
:108ee80080f32f00808f5000030034000100e90058
:108ef80000b179000200370020002000512207004d
:108f0800908e2900cc250700804580007800b900a4
:108f18006e004000a2972000600079002726070015
:108f2800f0442900c42507008045800066005000f1
:108f3800e30f500032003e008e2107008048900069
:108f48008180fb00104890004800dd00010070009f
:108f580012003200824580007810b900ea00400013
:108f6800a3972000618079000000e00004003a0027
:108f78001000200080b07900108f2900060037000b
:108f88007810b9006a0040008001eb00a297200029
:108f98000330790040912900a725070075210700b3
:108fa800c04890008180fb00504890004800dd00d8
:108fb8000100700012003200824580007810b9006c
:108fc800ec004000a3972000618079000000e000d9
:108fd80004003a001000200080b07900f0922900c7
:108fe800060037007810b9006c0040008001eb00e3
:108ff800a297200003307900509429008e2507009d
:109008005c210700c05090008180fb005050900008
:109018004800dd0001007000140032008445800023
:109028008001eb007820b90066004000a29720007c
:10903800600079000000e00001003a001300200001
:109048007820b90066004000a2972000033079001c
:10905800c09529000300e00003003200e18f5100b1
:1090680002003a00309729007325070041210700c4
:10907800e05090008180fb00705090004800dd00b7
:109088000100700014003200844580008001eb006c
:109098007820b90068004000a2972000600079009d
:1090a8000000e00001003a00130020007820b90019
:1090b80068004000a297200003307900a09829009a
:1090c8000300e00003003200e18f510002003a0083
:1090d800109a29005825070026210700e05890001b
:1090e8008180fb00705890004800dd00010070008e
:1090f80022023200804580007800b90076004000e6
:10910800a3972000608179000201e800e700610070
:1091180001b07900a0a12900e38f500014003200ab
:1091280006003e00109d2900e18f5000100032001b
:10913800709f29000e003e000c00370070a6290021
:10914800e58f50000a003200d0a32900080039003a
:1091580050a92900e68f500005003200d0ae290042
:10916800e78f500002003a0003003700b09b290047
:109178003125070001023700a0ac2900fcff3700a9
:10918800f8200700a04090008180fb00304090004c
:109198004800dd00010070007f003200f120070068
:1091a800c04090008180fb00504090004800dd00e6
:1091b8000104700078003a00804580006400500087
:1091c800e10f500012003e00ea200700c05890004e
:1091d8008180fb00505890004800dd0001007000bd
:1091e8000b00320008007800e808e20001003a00ad
:1091f8001000200040478800e10f500002003a00ac
:1092080060af29000100370090b029000a25070047
:1092180080458000e10f500012003e00d520070075
:10922800c05890008180fb00505890004800dd0035
:10923800010070000b003200bc08ee00bc08b7004b
:109248004f00de0061001000e0458800e10f50008b
:1092580002003a00d0b1290001003700f0b329001c
:10926800f5240700b088ed00e10f500012003e0021
:10927800c0200700c05890008180fb005058900023
:109288004800dd00010070000b003200ba08ee0053
:10929800ba08b7004f00de0061001000d045880012
:1092a800e10f500002003a0020b629000100370003
:1092b80050b82900e0240700ae200700e0589000cd
:1092c8008180fb00705890004800dd0001007000ac
:1092d800110032000208ec00a20020001100090071
:1092e8000280d8001140880090ba29000100e000ef
:1092f80003003200e18f500003003a0050bc2900ff
:10930800cd2407000400370000be2900ca24070046
:109318000288ec0077fc070096200700a058900010
:109328008180fb00305890004800dd00010070008b
:1093380017003200804580007800b90072004000b4
:10934800a497200060017a000201e80033002000a1
:10935800801f7800110009000381d8004f007800b1
:1093680001307a00e18f50000500320060c1290009
:1093780006003900e28f500005003a00020037006d
:1093880040c329000100370000c62900aa240700ad
:10939800782007007901370076200700a048900060
:1093a8008180fb00304890004800dd00010070001b
:1093b8000b003a006d200700a04890008180fb0058
:1093c800304890004800dd000100700021032000b3
:1093d800810f500019003600b208ab0017003a00a0
:1093e800804580007800b9000081e800a39720003c
:1093f800e2807900700c2000808f500003003c0050
:109408000100e80000b179000200370020002000c8
:109418000c210700c0c82900872407008045800068
:109428007800b9000080e800a29720006000790069
:10943800e2240700f04429007f2407004d2007009c
:10944800e04890008180fb00704890004800dd00f3
:10945800010070000b003a0044200700e04890002b
:109468008180fb00704890004800dd00010070001a
:1094780021032000810f500019003600b208ab000c
:1094880017003a00804580007800b9000081e800a4
:10949800a3972000e280790080f32f00808f50008e
:1094a800030034000100e90000b179000200370030
:1094b80020002000e3200700c0c829005e24070020
:1094c800804580007800b9000080e800a29720005d
:1094d80060007900b9240700f044290056240700e9
:1094e80024200700804890008180fb0010489000ed
:1094f8004800dd00010070000b003a001b20070047
:10950800804890008180fb00104890004800dd00f2
:109518000100700021032000810f5000190036005f
:10952800b208ab0017003a00804580007800b90007
:1095380064014000a3972000e2807900900f20008a
:10954800808f500003003c000100e80000b1790062
:109558000200370020002000ba200700c0c92900f7
:1095680035240700804580007800b9006400400079
:10957800a29720006000790090240700f044290099
:109588002d240700fb1f0700c04890008180fb00c6
:10959800504890004800dd00010070000b003a00c0
:1095a800f21f0700c04890008180fb0050489000df
:1095b8004800dd000100700021032000810f5000e9
:1095c80018003600b208ab0016003a00804580004b
:1095d8007800b900e4004000a297200061007900fb
:1095e8000000e000030034000000e900803079004a
:1095f800020037002000200092200700c0c929007f
:109608000d240700804580007800b9006400400000
:10961800a29720006000790068240700f044290020
:1096280005240700d31f0700a05890008180fb0085
:10963800305890004800dd00010070000b003a002f
:10964800ca1f0700a05890008180fb003058900086
:109658004800dd000100700021032000810f500048
:1096680017003600b208ab0015003a0080458000ac
:109678007800b900a29720000001410092407800cc
:10968800c0c7b30080cf500002003e000149e80087
:1096980002003700200020006a20070050ca290075
:1096a800e5230700804580007800b900a2972000d4
:1096b80062407800eb230700f0442900de2307000e
:1096c800ac1f0700e05890008180fb0070589000a4
:1096d8004800dd00010070000b003a00a31f0700de
:1096e800e05890008180fb00705890004800dd0031
:1096f8000100700021032000810f50001600360081
:10970800b208ab0014003a00804580007800b90028
:10971800a297200080004100114078000004e0007a
:10972800020032008048e9000200370020002000d3
:109738004420070050ca2900bf2307008045800045
:109748007800b900a297200062407800c52307007e
:10975800f0442900b8230700861f070080589000ae
:109768008180fb00105890004800dd000100700067
:109778000b003a007d1f0700805890008180fb0095
:10978800105890004800dd000100700021032000ff
:10979800810f500019003600b208ab0017003a00dc
:1097a800804580007800b900a297200000014100a0
:1097b8009240900070ccb30080cf500003003e0070
:1097c8000140e80010419800020037002000200006
:1097d8001c20070010cb2900972307008045800034
:1097e8007800b900a29720000001410012409000c3
:1097f8009c230700f04429008f2307005d1f070002
:10980800c05890008180fb00505890004800dd004f
:10981800010070000b003a00541f0700c058900068
:109828008180fb00505890004800dd000100700066
:1098380021032000810f500018003600b208ab0049
:1098480016003a00804580007800b900a2972000f1
:109858008000410011409000e14f500003003600a5
:109868000040e900904098000200370020002000e6
:10987800f41f070010cb29006f23070080458000e4
:109888007800b900a2972000000141001240900022
:1098980074230700f044290067230700351f0700d9
:1098a800806090008180fb00106090004800dd001f
:1098b8000100700015003200301f0700814580004c
:1098c8007809b90070014100a89720008180400004
:1098d800808040001182fb00114090004800dd00ac
:1098e8000400700000317c0000cc290052230700de
:1098f800804580007800b9007000400060007c005e
:109908008a230700f04429004b230700171f07008c
:10991800806090008180fb00106090004800dd00ae
:109928000100700041062000810f500013003a002a
:1099380010cd2900402307000004eb00a99820005f
:109948000e1f070088004400808040001181fb0042
:10995800114090004800dd00820c70000804e80007
:10996800f8844400ec0f5400f5ff3a00504a2900ef
:1099780031230700a0002000b21f070080458000a7
:109988006c04500010002000f10f540053013e00f9
:10999800f41e0700c04090008180fb0050409000fa
:1099a8004800dd000100700007003200ed1e0700ce
:1099b800a04090008180fb00304090004800dd000e
:1099c8000100700041013200e61e0700a04090002f
:1099d8008180fb00304090004800dd0001007000ed
:1099e80007003200df1e0700c04090008180fb00a6
:1099f800504090004800dd00010070003301320043
:109a0800dc1e0700c05890008180fb005058900071
:109a18004800dd00010070000f0032000001eb007b
:109a28004340dd00a18e2000608078000000e00047
:109a380001003a0012002000c340dd00a08e200083
:109a48008230780030cf2900e10f51000100320048
:109a580060d02900f8220700c61e07008058900031
:109a68008180fb00105890004800dd000100700064
:109a7800360032004340dd000080e800a18e20005f
:109a880060807800e20f50001900320005003e00a7
:109a98000000e00008003200e10f500029003a0001
:109aa8000c003700e30f500018003200e40f50009c
:109ab80024003a001c0037004340dd000080e80025
:109ac80012002000a18e200002b0780070d1290079
:109ad8001d0037004340dd000080e8002200200020
:109ae800a18e200002b0780080d22900160037002d
:109af8004340dd000080e80032002000a18e2000f5
:109b080002b07800e0d329000f0037004340dd00a1
:109b18000080e80042002000a18e200002b07800fa
:109b280010d52900080037004340dd000080e80018
:109b38000001eb00a18e200002b07800b0d6290009
:109b48000100370000d82900bb220700871e070044
:109b5800a04890008180fb00304890004800dd005c
:109b680001007000813e2000810f5000090036007e
:109b78004340dd0064014000a38e2000e2807900ac
:109b880050a52e00808f500002003e006a804000e1
:109b980000b17900771e0700a04890008180fb0083
:109ba800304890004800dd00010070000b003a00ca
:109bb8006e1e0700a04890008180fb00304890008e
:109bc8004800dd000100700021032000810f5000d3
:109bd80017003600b208ab0015003a004340dd001c
:109be80064014000a38e2000e2807900f0a52e00d9
:109bf800808f500003003e000100e80000b17900aa
:109c080002003700200020000e1f070050d929004d
:109c1800892207004340dd0064004000a18e200037
:109c280060807800c122070030da2900822207000c
:109c38004e1e0700e04890008180fb0070489000ad
:109c48004800dd0001007000813e2000810f5000b7
:109c5800080036004340dd00e4004000a28e2000ea
:109c680061007900eb0f5000020036006a005000d6
:109c7800803079003f1e0700e04890008180fb009b
:109c8800704890004800dd00010070000b003a00a9
:109c9800361e0700e04890008180fb007048900065
:109ca8004800dd000100700021032000810f5000f2
:109cb80016003600b208ab0014003a004340dd003d
:109cc800e4004000a28e200061007900e10f5000fe
:109cd800030036000000e9008030790002003700f8
:109ce80020002000d71e070050d929005222070063
:109cf8004340dd0064004000a18e200060807800b1
:109d08008a22070030da29004b220700171e0700b5
:109d1800804890008180fb00104890004800dd00da
:109d280001007000813e2000810f500009003600bc
:109d38004340dd0066014000a38e2000e2807900e8
:109d480050a52e00808f500002003e006a8040001f
:109d580000b17900071e0700804890008180fb0051
:109d6800104890004800dd00010070000b003a0028
:109d7800fe1d0700804890008180fb00104890007d
:109d88004800dd000100700021032000810f500011
:109d980017003600b208ab0015003a004340dd005a
:109da80066014000a38e2000e2807900f0a52e0015
:109db800808f500003003e000100e80000b17900e8
:109dc80002003700200020009e1e0700a0da2900ac
:109dd800192207004340dd0066004000a18e2000e4
:109de800608078005122070030da2900122207002b
:109df800de1d0700c04890008180fb00504890009d
:109e08004800dd0001007000813e2000810f5000f5
:109e1800080036004340dd00e6004000a28e200026
:109e280061007900ec0f5000020036006a00500013
:109e380080307900cf1d0700c04890008180fb006a
:109e4800504890004800dd00010070000b003a0007
:109e5800c61d0700c04890008180fb005048900054
:109e68004800dd000100700021032000810f500030
:109e780016003600b208ab0014003a004340dd007b
:109e8800e6004000a28e200061007900e20f500039
:109e9800030036000000e900803079000200370036
:109ea80020002000671e0700a0da2900e221070031
:109eb8004340dd0066004000a18e200060807800ed
:109ec8001a22070030da2900db2107008800780011
:109ed8000a007800eaf10700100020004f0578001a
:109ee8004f04be0000000600d0db2900d221070085
:109ef80080dd2900d0210700e0e02900ce210700fd
:109f0800c0e22900cc210700c0e72900ca210700c8
:109f1800a0ea2900c821070040ed2900c621070052
:109f2800b0f02900c421070020f52900c22107004c
:109f3800b0f82900c021070040fb2900be21070016
:109f480040fe2900bc21070000002a00ba210700b2
:109f580000042a00b821070070062a00b62107006d
:109f680050082a00b4210700f0092a00b22107008e
:109f7800000c2a00b021070010102a00ae210700ab
:109f880070152a00ac210700701b2a00aa210700bf
:109f9800201f2a00a821070020212a00a621070047
:109fa800e0252a00a4210700e0282a00a2210700b2
:109fb800402c2a00a0210700502f2a009e210700cc
:109fc80060322a009c21070030342a009a210700b9
:109fd800c0362a009821070030382a009621070049
:109fe800d03b2a0094210700203f2a009221370005
:109ff800804178000004e00002003a007176800099
:10a0080011003700627680000c00370022009000b3
:10a018000000e00008003200a000900004003700b3
:10a0280021589000834f50000700320091007800bb
:10a038000100e000faff3a00120178000200e00097
:10a04800f2ff3a0082007800010078000000060064
:10a058006200200053ec2000934178000304e100e3
:10a068000d003a0001407800e1ff07008000780009
:10a07800420120000000e00007003200204090006c
:10a088000054a100a0409800214090000064a10065
:10a09800a04098000001eb000200780000000600d4
:10a0a800d0cebf004600de00610060000000060060
:10a0b800b076800001f0200001006000120320004b
:10a0c80016003200b076800001f020000100600028
:10a0d80001402000810f500007003a00b076800050
:10a0e800000fb200a2032000f00f50000b00320056
:10a0f8000203200009003700b076800001f020003c
:10a10800010060002203200001502000810f500050
:10a1180002003a00c6cebf000081fb0002007800b2
:10a12800000006000004e00014003a006376800096
:10a138000f003700130190000a003700a2009000ba
:10a1480074cfb30004003700314090000440600031
:10a15800b0409800910078000100e000faff3a0052
:10a16800120178000200e000f4ff3a009301780041
:10a178000300e000efff3a00000006009cff070024
:10a18800800078000000e0000300320030409000ba
:10a198000034a100b040980000000600881f780035
:10a1a80000047800204090000054a100204498004a
:10a1b800284090000064a1002044980028409000a6
:10a1c8000074a10020449800384090000004a100c9
:10a1d800304498002840900005ceb3000540600048
:10a1e80020449800384090000044a1003044980072
:10a1f800330c98006033b800060c9800170c9800d0
:10a208006123b80056049800670498000000eb002a
:10a21800700c9800210c98007204980000c1b300db
:10a228000400e0000100320000c3b300005c9800a5
:10a23800384090000014a100304498004f04780082
:10a2480000000600a04290000554a1002540980097
:10a25800a04290000564a10025409800a04290000b
:10a268000574a10025409800b04290000504a100a3
:10a2780035409800a042900006ceb30086c2620026
:10a2880025409800b04290000544a1003540980050
:10a29800330898006033b80006089800170898003b
:10a2a8000500200054009800650098008001eb002c
:10a2b80073089800210898007200980001c2b30042
:10a2c80001589800b04090000114a1003140980056
:10a2d800000006008f87e800889fbe008a9fbe00a6
:10a2e8008c9fbe008e1f780001467800824578005a
:10a2f8000304780084047800050578008606780051
:10a30800074778006200200051ec20009140780057
:10a318000104e10054003a00b076800001f020000a
:10a32800010060001200200001402000810f500051
:10a338004d003a0070768000304090000201200005
:10a348000018a30048003200ebcf55001f003a0068
:10a358006276800001003700120178000200e000f8
:10a3680040003200624090000080fb00890f5000de
:10a37800f9ff3a00220090000000e00039003200a6
:10a38800a000900004003700314090000018a3009e
:10a3980034003200910078000100e000faff3a0032
:10a3a8009200900001003700910078000100e00061
:10a3b8002c003200214090000080fb00880f5000e4
:10a3c800f9ff3a002101980008003700e1cf550055
:10a3d80006003a000300e00004003a00e24f56008d
:10a3e80002003e00044078004eff07001174800010
:10a3f8008c4878009b409800a84098004840de00b0
:10a40800b0409800c94098004848de00d040980005
:10a41800ea4098004850de00f040980070768000ce
:10a428002fe99700125898000e04e00006003a0041
:10a43800707680000a0278008d0178008200200082
:10a4480056ff070005003700707680000a02780082
:10a458008d017800820020007aff07000001eb00e0
:10a468000100370032002000020078004f07780012
:10a478004f06be004f05be004f04be002f00b100be
:10a488000000060080017800020278002040900059
:10a498000074a100a0419800334090000004a1007e
:10a4a800b04198002340900002ceb3000240600003
:10a4b800a0419800334090000044a100b0419800aa
:10a4c800b10998006000b8008009980091099800c7
:10a4d8006120b800d0019800e10198000000eb006d
:10a4e800f0099800d30890000030200080806000b8
:10a4f800808f500002003a0000c4b3000a00370001
:10a5080000102000808f500006003a0000c6b300fb
:10a5180080599800b30890000040eb0090409800e4
:10a528000200370000c8b3008059980033409000fb
:10a538000014a100b041980000000600889fbe00ea
:10a548008a1f780081417800020578000404be0063
:10a558006200200051ec2000914078000104e100e5
:10a5680026003a00b076800001f02000010060006b
:10a578001200200001402000810f50001f003a0007
:10a58800034078009afe070080017800420120000d
:10a598000000e00019003200500890000030b200be
:10a5a800820120001500320023589000520120003b
:10a5b8000004e00011003d0023409000120120003b
:10a5c8000058a3000d003a0023409000220120000b
:10a5d8000068a30009003a003340900002012000ff
:10a5e8000018a30005003200080178008a007800ee
:10a5f80003007800a3ff07000001eb0002007800c9
:10a608004f0578004f04be000000060061002000de
:10a6180052ec2000124178000204e10008003a00e0
:10a62800b076800001f020000100600031002000b9
:10a63800030032000000eb00b0768800800078004c
:10a6480001007800000006006200200051ec2000a4
:10a65800914078000104e10007003a00b1768000db
:10a668003200200000412000808f500002003a0094
:10a67800d62eec000001eb00020078000000060076
:10a6880070768000304090000018a300140032005b
:10a69800637680000e003700130190000900370030
:10a6a800a200900004003700314090000018a30079
:10a6b8000b003200910078000100e000faff3a0038
:10a6c800120178000200e000f5ff3a0093017800db
:10a6d8000300e000f0ff3a000300780000000600e5
:10a6e80010000500881f78000144780062002000ef
:10a6f80051ec2000914078000104e10013003a0079
:10a70800b076800001f020000100600012002000f7
:10a7180001402000810f50000c003a00d8ff0700cc
:10a72800220020000000e00008003a00080078003d
:10a73800c2eeb70000c0eb00717680009058980018
:10a7480000332000b07688000001eb00020078009a
:10a758004f04780000000600889fbe000204be0077
:10a768006200200053ec2000934178000304e100cc
:10a778000e003a00014078001dfe070080017800b5
:10a78800420120000000e00008003200e1406400bf
:10a79800c508dd00304090000054a1000140700061
:10a7a800b0419800891198000001eb000200780080
:10a7b8004f04be0000000600889fbe008a9fbe00ae
:10a7c8008c1f780000467800810478000205be00de
:10a7d80020072000808f500003003200f0ff270080
:10a7e800808f50000e003a001a489000e14f400058
:10a7f8001b003200a2c0b3000440bc000281e80084
:10a80800c0d62000e2017800615ab8000a01780039
:10a81800890078000c407800030001001000370020
:10a82800687680000c00370078409000a2c0b30022
:10a838000440bc000281e800c0d62000e201780094
:10a84800615ab8000a017800890078000c40780045
:10a8580003000100180478000800e000f2ff3a0045
:10a868004f0678004f05be004f04be0000000600ea
:10a878006200200051ec2000914078000104e100c2
:10a8880009003a00b1768000320020000040200024
:10a89800808f500004003a009404a9000041200071
:10a8a800b07688000001eb00020078000000060086
:10a8b800c1768000214090000064a100a04098006b
:10a8c800214090000054a100a0409800dd4eed000a
:10a8d800ddeeb7000300320000ff2f00d62eb600d1
:10a8e80000000600dc4eed00dceeb700020032008e
:10a8f800001120000300370070c0b300c6eeb70097
:10a9080000502000b0768800000006000800fa0019
:10a91800889fbe008a9fbe0008778000d0cea9001d
:10a928008005eb0069d320004ad320004358dd009e
:10a93800a1d32000608078000018a3000b0032002b
:10a94800484090009a4f100038003a00f9f89700f4
:10a958005840900080cf500034003a006840900082
:10a96800994f100031003a002f0037009a01780003
:10a97800884890008180fb00184890004800dd005e
:10a9880001007000808f510008003a00a84890002c
:10a998008180fb00384890004800dd00010070000d
:10a9a800990f100001003a00d0cea800e18f4100b5
:10a9b8001e003a000080eb00990f10001b003a00bf
:10a9c800884890008180fb00184890004800dd000e
:10a9d8008100700081bf9f00a84890008180fb0023
:10a9e800384890004800dd000100700090bf9f00cb
:10a9f8001a407800c0f79f0079f89700d0f79f00b9
:10aa080019407800e0f79f0084002000050020002e
:10aa18007081570091072000034078002013070039
:10aa28000000e00001003a00d0cea800d0cebf0060
:10aa38000068a30012003200c359dd0042d3200091
:10aa48008300410051409000c7eeb7006680410086
:10aa580060007900110020000028a3000e003200d9
:10aa6800c358dd0080d32000801f78006140780043
:10aa7800c2eeb7004f007800110020000600370032
:10aa88008b05e800e884440068054500e78f550019
:10aa9800a6ff3a008000eb00010078004f05be00d9
:10aaa8004f04be000080fa0000000600889fbe0028
:10aab8008a9fbe001e0037009005780016003700f8
:10aac800110578000a003700190478000900780099
:10aad8005cd7070060768000900090000000eb00d3
:10aae800a000980060768000100090002800980070
:10aaf8006076800010009000a00490000900e0003b
:10ab0800f1ff3a004fd707006076800019009800df
:10ab1800607680001a0098006076800090009000af
:10ab28000100e000e6ff3a0046d707006b76880090
:10ab3800607680000000e000dfff3a007076800059
:10ab4800c07688004f05be004f04be000000060016
:10ab5800889fbe000800370019049000190078008b
:10ab680038d70700507680000008eb005076800048
:10ab780034d7070058768800597680000900e0002d
:10ab8800f5ff3a00007780000000e0000200320084
:10ab98002cd7070009778800107480000000e000b7
:10aba8000200320027d70700822eef00bfff070000
:10abb8004f04be0000000600ce0ee20007003a0077
:10abc800200220008dd60700707688000000e00083
:10abd800120032000008eb0001003700dcff07001c
:10abe80070768000c07688008000eb00b17688001f
:10abf80086aeef008000fd00c4eeb700c5eeb700da
:10ac08008000fd00880ea8004000200050748800d5
:10ac1800607488007174880010002000000006002d
:10ac28000200fa008000eb0041248800c5cebf0076
:10ac38000b003200e1ff9f002400200005002000e7
:10ac48000f81e900a106200095120700c5cebf00bc
:10ac58001300200052ec200011072000d6fe070048
:10ac68006000b800d4ff07000080fa00000006006a
:10ac780052ec2000124178000204e1000b003a0077
:10ac880001407800dafc0700800078000000e0004e
:10ac980006003200204090000074a000a0409800f8
:10aca800314090000014a000b04098000000060059
:10acb800889fbe000204be0052ec200012417800ba
:10acc8000204e1000500320060c0b300004c7800c7
:10acd8008009eb00b31178002100370001407800ab
:10ace800c3fc0700800078000000e0001a00320072
:10acf800304090000000d100614160003140900078
:10ad08000008a30005003200004ceb00010a900087
:10ad1800910a9000848cbe000d00370021409000fd
:10ad28000058a3000200320010c1b300070037002a
:10ad3800214090000068a30003003200c158900031
:10ad4800014c78000200370090c1b300004c780035
:10ad58000280fb000300370040c1b300004c7800bc
:10ad6800100020004f04be0000000600800178009b
:10ad7800e1cf40000d003a000204e0000b003a0069
:10ad880080062000808f510003003a00a4ff0700ce
:10ad9800880ea90004003700b0062000808f5100fb
:10ada80002003a00880ea8000000050030000500e7
:10adb8008001780002027800204090000074a10011
:10adc800a0419800334090000004a100b0419800d1
:10add8002340900002ceb30002406000a0419800da
:10ade800334090000044a100b0419800b109980098
:10adf8006000b80080099800910998006120b800a7
:10ae0800d0019800e10198000000eb00f0099800db
:10ae1800d30890000030200080806000808f5000b0
:10ae280002003a0000c5b3000a00370000102000f5
:10ae3800808f500006003a0000c7b3008059980080
:10ae4800b30890000040eb009040980002003700e3
:10ae580000c9b30080599800334090000014a10045
:10ae6800b041980000000600889fbe008a1f780045
:10ae780081417800020578000404be0062002000c9
:10ae880051ec2000914078000104e10026003a00ce
:10ae9800b076800001f02000010060001200200060
:10aea80001402000810f50001f003a000340780045
:10aeb8004ffc070080017800420120000000e000fc
:10aec80019003200500890000030b20082012000c2
:10aed8001500320023589000520120000004e000c1
:10aee8001100350023409000120120000058a300f3
:10aef8000d003a0023409000220120000068a300c2
:10af080009003a0033409000020120000018a30015
:10af180005003200080178008a00780003007800f4
:10af2800a3ff07000001eb00020078004f0578003e
:10af38004f04be0000000600ec874700889fbe0053
:10af48008a9fbe008c9fbe008e1f78000047780045
:10af5800814678000246780083bf9f00087780000a
:10af68000005eb0069d32000c355dd00668045006d
:10af780041d32000608078000018a300260032002a
:10af880069f897008e4f500023003a0079f897002f
:10af98008d4f500020003a00994f16001e003a00cd
:10afa800884890008180fb00184890004800dd0028
:10afb80081007000c1b79f00a84890008180fb0005
:10afc800384890004800dd0001007000d0b79f00ad
:10afd800ceef9f00ddef9f00ecef9f008400200084
:10afe80005002000788157009107200000c0eb0081
:10aff800ab1107000000e00007003a0041d3200031
:10b008000b804000504090008fb89700804878002f
:10b0180010002000050037000a05e800e884440015
:10b02800e70f5500d0ff3a000000eb004f0778000b
:10b038004f06be004f05be004f04be00cf00b10052
:10b0480000000600ec874700889fbe008a9fbe006c
:10b058008c9fbe008e1f7800127780006c7680006f
:10b06800d02ea900d04ea80012447800a24090002b
:10b078008180fb00324090004800dd008080400065
:10b08800e1b79f0052409000f0ef9f000249900006
:10b0980082f79f00778157008ff097001141980041
:10b0a8000049eb0024002000050020009106200044
:10b0b80000c0eb007a1107008002eb000000e000fe
:10b0c80003003a0080c2b300c6eeb70015002000a6
:10b0d8008880fb001077800080844000010578009c
:10b0e8000040eb00e0ef9f00ae00370015002000a5
:10b0f800b700370099467800994090000980e80029
:10b10800e9cf50000c003a00d02ea800104078007b
:10b11800c3eeb7000018a30005003200d0cebf0070
:10b128000038a30002003200d04ea900a00037006a
:10b13800d06ea9009e003700e4cf50009c003a0072
:10b148009045780039479000c940900091f79f00da
:10b1580059429000e940900079419000e884440009
:10b16800d0cebf000068a30003003200c7cebf00e6
:10b1780080ef9f0005003700f881570004407800f1
:10b188006dff07000000e000890032000c04780021
:10b1980001003700180478000800e00004003200bd
:10b1a800684090008b4f5000faff3a000d003700be
:10b1b8008000200011d50700000478000000e0009e
:10b1c800710032006b4098000fe8970070449800b7
:10b1d8000000eb0010049800200498000c0c780084
:10b1e800080678006000200004d507008005780074
:10b1f8000000e0009a003a00630037002b04980032
:10b208000d80fb0000054500107780008004450094
:10b218008040eb00e1ef9f0053003700994678002b
:10b228000984e80019409000e54f500005003200fd
:10b238000d80fb0000054500107780008004450064
:10b248004900370020022000ecd407008001780074
:10b258000000ea00030070004f02de0010c0b300d7
:10b26800044250008482fb0018447800a8599800d2
:10b2780039409000b0599800c94090008180fb0087
:10b28800c1019800594090004800dd0080804000ce
:10b29800c1019800694090000083fb00a601980056
:10b2a8000001eb0092019800334090000024a000b8
:10b2b800b0419800334090000014a000b0419800bd
:10b2c8006000b80080099800910998008259980098
:10b2d8008fe8970091599800530890000030b20009
:10b2e80001102000810f500011003a000600e00014
:10b2f80002003a0010002000a001980023009000ee
:10b30800f00f50000200360000012000a001980054
:10b31800230090000000e900110020008008dd00f3
:10b32800a1019800334090000024a100b04198008a
:10b3380023009000b0019800ab00900081097800cc
:10b34800a30598006fe897000040e800e0ef9f0031
:10b358000d80fb0000054500107780008004450043
:10b368000404e0000b003a00efb09700810f55008d
:10b37800070031006fe897009ff09700814f500059
:10b38800a6ff390002003700150020000100370031
:10b398008002eb006fe897009ff09700814f500004
:10b3a80052ff3a000500e0000600320008003700ae
:10b3b8000d80fb00000545001077800080044500e3
:10b3c8008002eb006fb09700800f550049ff3900ed
:10b3d8000c00e000200032000500e00016003200fa
:10b3e8009c0478000b00370098007800110698003c
:10b3f80003003700900078002104980011d5070059
:10b40800280090000000e000faff3a0008007800e9
:10b418000cd507001c0490000800e000f2ff3a0079
:10b428000c00780007d507000900e0000a00320088
:10b4380009067800eaff37007fe89700c2eeb700f8
:10b448008ff097000180fb00407688006c768800ba
:10b45800100020000b0037000000eb000900370047
:10b4680018009000800d7800ae4598000000eb00b1
:10b47800a00598001b0498000e04e0005fff32004e
:10b488005fff37004f0778004f06be004f05be002c
:10b498004f04be00cf00b100000006000200fa0011
:10b4a800889fbe001d0037006074800002e92000fc
:10b4b800e20f500003003c006c00b900c2e9200014
:10b4c800000141009200780020072000808f500082
:10b4d80003003200f0ff2700808f500004003a007c
:10b4e8000281e800c5cebf00a3002000b2fc07001f
:10b4f800612480008c24ef008e2eed0060748000a3
:10b50800e20f500003003c000000e800607488006f
:10b51800010037008c2eef00612488008e0ee200b7
:10b52800e1ff3a0030748000e10f40000300320070
:10b5380030748000b076880086aeef00b176800067
:10b5480000f020008080600000202000808f5000e4
:10b558004101320006003e000100e0000e0032000a
:10b5680000102000808f5000eb023a008000370066
:10b5780000402000808f5000980232000010b00078
:10b58800808f5000af02320000302000808f5000c2
:10b59800e1023a0050013700b8768000080fb20087
:10b5a800f00f54005100320009022000890f5400a6
:10b5b800510032000800e000d7023a0098fd070069
:10b5c800707680000808780070768000180098006f
:10b5d80071768000314090000024a000b0409800af
:10b5e80071768000314090000014a000b0409800af
:10b5f800717680003140900009407000b04098009a
:10b60800017d200070768000011098000104200060
:10b6180070768000410098006000b8007276800063
:10b628000009980011099800707680002858980041
:10b638007076800008589800727680005208900052
:10b64800f1cf2f00010060005009980080c0eb0086
:10b65800707680001158980030c0b300dceeb70057
:10b668000004fd00c2eeb700c3eeb700c4eeb70099
:10b678000004fd008876880068768800987688003f
:10b6880068248800f10f200051248800c008200099
:10b698008224b6006f0050000024880088248800a7
:10b6a80071248800000021004800de00c0248800c2
:10b6b80081002000a1248800a0002000a024880088
:10b6c800a1248800000320003024880020002000e6
:10b6d8003025880048258800b8248800aae4a900f5
:10b6e800a00420000025880086023700880eab00e1
:10b6f80089023200830237000041eb00a2ff9f005d
:10b7080020c3b300b0ff9f002400200005002000e4
:10b71800668157009106200000c0eb00e00f07008b
:10b728000000e0000f0032001000200040248800d4
:10b738008ec0a900f00f2f00ce20b60000602000b8
:10b74800ce20b7009ec0a800b076800001ff200080
:10b758000100600070004000b07688008cc4a8002a
:10b768006d023700880ea900000120006902370029
:10b77800b1768000010fb20000022000808f5000d7
:10b788005c00320005003e000100e0000a003200c3
:10b79800f08f500060023a001200370000032000ca
:10b7a800808f50008d00320070004000808f500064
:10b7b80059023a00a6003700b07680006f0060009a
:10b7c80003003200e20f500053023a004d023700e6
:10b7d80010002000502488008c04a800b00f20001e
:10b7e80010023700b07680006f046000e20f54004a
:10b7f80039003200e40f5400390032000800e0003c
:10b8080045023a00107480000000e0000200320097
:10b818000cd40700187488008000200077d3070034
:10b82800107488000000e000fc0032000040eb00cb
:10b83800c2eeb700c3eeb7000000eb0080768800c8
:10b8480031c0b3008000fd00ddeeb7008000fd00d0
:10b85800d1002000512588006025880070258800c7
:10b868008025880090258800a0258800b0258800bc
:10b87800c0258800d0258800e0258800f0258800ac
:10b888000026880010268800202688003026880098
:10b89800402688009444e20006003500d00ea80037
:10b8a80000c8b300c4eeb70000082000b024880028
:10b8b800aae4a8009424a8009424a900d08ea90082
:10b8c800d0aea9009484a80030032000d076880068
:10b8d8006d004000d50137009484a900cf013700de
:10b8e800f000200060248800f00f200080248800e9
:10b8f80004023700b07680006f006000e10f50004e
:10b908001300320003003900e20f500002023a002f
:10b918001c003700007780000000e00002003200c1
:10b92800c8d30700e02eef001174800000c8b300f0
:10b938008048780060c0b300904098000041eb0058
:10b94800a240980010c0b300b0409800960037009d
:10b9580071768000314090000018a300ee0132009b
:10b96800314090000008a300640132001074800088
:10b9780040409000e94f5000ae013a0050c3b30078
:10b988007b013700107480001080fb001bd3070078
:10b9980080007800007788000000e0009f003200f7
:10b9a8001074800090487800f04090008180fb007f
:10b9b8007276800041019800a2d30700822eef0022
:10b9c80070768000400090000cd307001074880047
:10b9d8000000e00091003200a3003700b07680003c
:10b9e8006f006000e10f50003d0132000300390094
:10b9f800e20f5000c8013a009b003700d2cebf00ca
:10ba080070416000c4013a001174800000c8b3009e
:10ba18008048780060c0b30090409800a240980029
:10ba280010c0b300b0409800c2409800d2409800bf
:10ba38000077800010407800e0409800f2409800bd
:10ba480003778000707680001382fb00ad0037001a
:10ba5800aefb07001b003700b0768000000fb20075
:10ba6800ad013a00b07680006f006000e10f500031
:10ba78001b01320003003900e20f5000a6013a0012
:10ba88000900370010c0b300c5eeb700117480007c
:10ba98000041eb008248780050c0b3009040980005
:10baa800c5cebf0002013700d0cebf0061006000e4
:10bab8004700dd00c54eb700c4eeb70030c0b30084
:10bac800ddeeb700b076800001f0200001006000d4
:10bad8000010b0008f013700b1768000010fb2006e
:10bae80000022000808f50006200320005003e00f6
:10baf8000100e0000a003200f08f500086013a0091
:10bb08001700370000032000808f500086003200a5
:10bb180070004000808f50007f013a00d400370049
:10bb28000077800010509000deeeb7000800370064
:10bb3800100490001000780042d30700507680006f
:10bb48000008eb00507680003ed307005876880046
:10bb5800507680000000e000f5ff3a0069013700e8
:10bb6800b07680006f006000e10f5000dc0032000a
:10bb780003003900e20f500067013a001500370052
:10bb88001174800000c8b3008048780060c0b3001a
:10bb980090409800de4eed00a040980020c0b30011
:10bba800b04098000041eb00c2409800d240980095
:10bbb80080c0b300e0409800f240980070768000a2
:10bbc8008400200081017800040178009df90700b5
:10bbd800180137006000200088d207000000e0004c
:10bbe8000e0032000004780011748000314090008b
:10bbf8004800dd00a14090008180fb00010040006a
:10bc08007ed2070000017800000c78000000e000f8
:10bc180004003a00080078000ad3070030c3b300d4
:10bc2800d300370010748000b0409000c808dd00d1
:10bc3800204090000080fb00808040002141980057
:10bc4800c808de003141980052768000120498003e
:10bc5800587688001800780010778800e2ed2000f8
:10bc6800124178004244980030c0b300ddeeb700be
:10bc780024013700b07680006f006000e10f5000ab
:10bc88009700320003003900e20f500022013a0009
:10bc98001e0037001174800000c8b3008048780087
:10bca80060c0b30090409800de4eed00a0409800c0
:10bcb80020c0b300b04098000040eb00c04098009e
:10bcc800d040980050768000100078002040900006
:10bcd800e0409800507680001000780030409000d6
:10bce800f040980050768000900178002341900041
:10bcf8000281fb00334290004822dd00707680000c
:10bd08000202720082002000b0ff370030c0b3008a
:10bd1800ddeeb700de4eed00deeeb700f9003200d2
:10bd280000312000fb003700b07680006f00600013
:10bd3800e10f50003200320005003900e20f5000d8
:10bd480067003200e30f5000f3003a00420037006a
:10bd580056fb070022ec2000124178000204e000a4
:10bd68000f003a0050768000080037001000780075
:10bd780010778800b3fc07000000e0001a003a00c2
:10bd88004afb07002074800010009000207488008f
:10bd9800207480000000e000f4ff3a001200370031
:10bda80051768000217488000100370091009000ce
:10bdb8000100e0000300320041409000824f500033
:10bdc800faff3a0021748800910078001177880002
:10bdd8009cfc0700000478000000e00002003a0024
:10bde80032fb070028748800d0cebf000028a300cb
:10bdf80090003200840ee2008e003a001a003700ec
:10be0800d0cebf0064406000be003a00d04ea8000b
:10be1800117480008048780032c0b30092409800c6
:10be2800d0cebf000038a30002003200a240980024
:10be38000200370040c0b300a04098000040eb006b
:10be4800b0409800c0409800d0409800e04098006a
:10be5800f04098001c00370030c0b300ddeeb7009a
:10be6800840ee20080ff3a0040c3b3004000370070
:10be7800b07680006f006000e10f500018003200bb
:10be880005003900e20f50001e003200e30f500099
:10be9800a1003a001e003700117480000041eb0039
:10bea8008248780090c0b30090409800c2cebf008e
:10beb800a0409800b2409800c2409800d240980034
:10bec800e2409800f2409800707680000002eb0093
:10bed8008401780082002000b0f807005500370080
:10bee80071768000314090000018a3008a0032006b
:10bef800314090000008a3004e003a006cfa070099
:10bf08008500370030c0b300ddeeb70049003700c8
:10bf1800b076800001f02000010060000010b00041
:10bf2800b0768800d0cebf000068a30013003200ae
:10bf380071ec20009140780001407800a2c0b30065
:10bf48000440bc0082017800c2d620000282410071
:10bf5800c5cebf00e302790034019000c40190000f
:10bf6800050001000000e0006b003a0090c3b30038
:10bf7800c6eeb700005020006600370068768000e3
:10bf880013003700f840900001407800a2c0b300c9
:10bf98000440bc0082017800c2d620000282410021
:10bfa800c5cebf00e302790034019000c4019000bf
:10bfb800050001000000e00004003a0090c3b3004f
:10bfc800c6eeb70000502000b0768800180478004c
:10bfd8000800e000ebff3a004f003700b076800021
:10bfe800000fb200f00f50004b003a00b07680000e
:10bff8006f006000e30f500007003200e50f5000ab
:10c008000e003200e10f500043003a009444a800ab
:10c0180050012000030037009444a9009404a800ac
:10c02800b0002000d076880000042000002488009a
:10c0380082c4a800d62eec0037003700004020004c
:10c0480034003700b2768000020fb20032003a00a6
:10c0580080002000a024880062248800f10f2000be
:10c0680051248800c00820008224b6006f005000c8
:10c078000024880082248800712488008c04a80089
:10c0880062ec20001241780040c3b300c1c6b3007f
:10c09800804f51001500320007003e008140e80043
:10c0a800e74f5100110032000040e900804f510075
:10c0b8000b003a000800370051c6b30050c3b30064
:10c0c800804f51000900320064404000804f510009
:10c0d80003003a0004003700f1c6b300030037003c
:10c0e80001c7b30001003700e1c6b3008180fb003f
:10c0f800c5cebf00140020000500200082ec2000ff
:10c10800670d0700b076800001ff20000100600085
:10c1180070004000b07688004f04be000080fa002e
:10c128000000060000427800717680008082fb00e3
:10c13800510890004800de0063006000850f500041
:10c1480005003a00314090000018a30002003a00b0
:10c15800c17688003a003700d56eef00637680001c
:10c168002b003700520890004800de006300600092
:10c17800850f500023003a00e24f520015003200ac
:10c18800e34f5200060032000404e0001d003a00ac
:10c19800324090000018a3001a003a002700370028
:10c1a800324090000018a3000600320032009000d0
:10c1b8000000e00013003a002200900030019800cf
:10c1c80010003700320090000000e0000d003a0037
:10c1d8001a003700324090000018a30009003a0006
:10c1e800324090000048a30006003a00d56eec00eb
:10c1f80051ed200091407800d4cebf0080cf500090
:10c208000c003e0012017800070037009301780007
:10c218000300e0000b003200230090000000e00063
:10c22800faff3200200190000200e000cdff3a0042
:10c23800f6ff3700d5cebf00d4eeb700c27688002f
:10c24800100005000000050000417800e94f50008b
:10c2580011003a00d0cebf00470021000048a300db
:10c2680001003a0007002100d0cebf004400de00e4
:10c27800610060000004a2004400dd0001ed200020
:10c28800914078000144a10080c07000010078004e
:10c29800d0eeb70025003700d0cebf00c700210080
:10c2a8000058a30001003a0087002100d0cebf004b
:10c2b8004500de00610060000004a2004500dd00ca
:10c2c80001ed2000914078000154a10080c0700069
:10c2d80001007800d0eeb700ed4f510013003a008e
:10c2e800c676800076009000060a9000960a9000b4
:10c2f800460190000100200004005000858058008d
:10c3080003002000820f5000838f5800020036007f
:10c31800c60190001d0037007601900006089000c5
:10c32800960890008001510018003700c6768000fa
:10c338003658900063406000e14f50000b00320017
:10c3480056009000e6009000060a9000960a9000b9
:10c35800460190000400500085805800030020002a
:10c36800820f5000838f580002003600c6019000eb
:10c378002e00370056019000e60190000608900054
:10c38800960890008001510028003700260b900085
:10c39800960398000e003700b60890003608900003
:10c3a8001040900062c0b3000440bc006601410028
:10c3b800e280780091039800050037003609900064
:10c3c800060890009608900000014100920398002a
:10c3d8000040eb009043980083007800f13fb200e2
:10c3e80000c02f00970b6000978b7000c17680000b
:10c3f800314090004300de00610060004e00dd0027
:10c4080017e0a100970b7000314090004200de0059
:10c41800610060004b00dd0017b0a100970b7000b1
:10c4280000002800970b70000000060036589000a6
:10c4380063406000e14f5000e0ff3a00d6ff37004c
:10c4480000427800d0cebf00d3cdb3000008a300cf
:10c4580001003a00d3c5b300c2768000325890007c
:10c468006340600001003a000344a1003258900084
:10c4780063406000e14f500001003a000304a1004e
:10c488000380fb0050258800c4cebf000080fb005d
:10c49800b02488000180fb004400dd00840078009f
:10c4a800f107b20001007000f0248800d28ea800c5
:10c4b80000000600881f7800b0768000d2cebf004a
:10c4c8000048a300bc013a00d2cebf000004eb0034
:10c4d8000008a300aa003a000040eb0011ff070083
:10c4e8000000e000a0003200c376800003589000ee
:10c4f80080007800010fb20000022000808f5000f9
:10c508001f00320070004000808f50002e00320063
:10c51800f08f5000a1013a00035890006f006000ae
:10c52800e10f50000700320003003c000000e0006b
:10c538003400320099013700e20f50004000320009
:10c548002d0037000308900093089000d001980050
:10c55800e1019800334090000034a000b0419800f9
:10c5680090c0b30038ff0700c076800020589000c4
:10c5780091c0b300b2ff0700d20ea8008e013700a9
:10c58800035890006f006000e20f50000600320070
:10c5980017003c000000e0001a003200e10f5000d4
:10c5a8007e013a00eeff37000308900093089000e0
:10c5b800d0019800e1019800334090000034a000b9
:10c5c800b041980018003700035890006f006000d1
:10c5d800e20f5000dbff320005003c000000e000e5
:10c5e80008003200e10f50006c013a000e003700dd
:10c5f800e30f500012003200ef0f500067013a00bd
:10c6080035003700334090000034a100b041980055
:10c61800d0c0b3000cff0700c076800020589000ff
:10c62800d1c0b300d3ff370010c0b30006ff070026
:10c63800c07680002058900011c0b300cdff3700ad
:10c648000040eb0080599800334090000014a0008f
:10c65800b041980070748000e30f500044003c0023
:10c668000000e8007074880050748000e20f5000e9
:10c6780003003c000000e800507488000100370007
:10c688008a2eef00507480006c00b90002e9200087
:10c6980000014100200720000009780003089000ed
:10c6a800930890001001980021019800b3089000a9
:10c6b800310198000040eb00104998002358900081
:10c6c80000499800b3589000214998009359900068
:10c6d80033499800280037000040eb008059980043
:10c6e800334090000014a000b0419800707480009e
:10c6f800e30f50001e003c000000e8007074880042
:10c7080050748000e20f500003003c000000e80075
:10c7180050748800010037008a2eef0050748000a2
:10c728006c00b90002e9200000014100f0ff270079
:10c73800000978006000b8001001980021019800f5
:10c748000000eb0030019800c35890001149980090
:10c75800a358900001499800b358900021499800c7
:10c76800935990003349980000047800030037007b
:10c7780080c0b300b05998000004eb00d20ea800a6
:10c78800d2cebf000018a3007f003a00790037001e
:10c79800c37680000358900080007800010fb20033
:10c7a80000042000808f5000040032007000400018
:10c7b800808f500067003a00090037000358900046
:10c7c8006f006000e10f50000e003200ef0f5000c4
:10c7d800340032000000e0005e003a0084003700b8
:10c7e800035890006f006000e10f50000500320010
:10c7f800ef0f50002b0032000000e00055003a0017
:10c808009e0037000040eb008059980023009000fc
:10c81800b0019800334090000014a000b041980087
:10c8280070748000e30f500045003c000000e800f1
:10c838007074880050748000e20f500003003c00c0
:10c848000000e80050748800010037008a2eef00cd
:10c85800507480006c00b90002e92000000141001a
:10c868002007200000097800030890009308900032
:10c878001001980021019800b30890003101980038
:10c888000040eb0010499800235890000049980098
:10c89800b3589000214998001358900030499800e7
:10c8a800290037000040eb0080599800a300900051
:10c8b800b1019800334090000014a000b0419800e6
:10c8c80070748000e30f50001d003c000000e80079
:10c8d8007074880050748000e20f500003003c0020
:10c8e8000000e80050748800010037008a2eef002d
:10c8f800507480006c00b90002e92000000141007a
:10c90800f0ff2700000978006000b80010019800c7
:10c91800210198000000eb00300198004358900076
:10c9280010499800a3589000014998003358900086
:10c938002049980093589000314998000200370028
:10c9480080c0b300b05998000800e00002003a0027
:10c9580008003700180020000040eb0080599800bc
:10c9680023009000b0019800334090000014a0000c
:10c97800b041980030c0b300eafd07000000e000b5
:10c9880083ff3a00d22ea800d2cebf000038a30001
:10c9980089003a0020c0b300e2fd07000000e00073
:10c9a80078003200c3768000035890008000780039
:10c9b800010fb20000082000808f500004003200f0
:10c9c80070004000808f500068003a002300370054
:10c9d800035890006f006000e10f50002e003200f5
:10c9e800ef0f50004c0032000000e0005f003a00fa
:10c9f80090c0b30014fe0700c07680002058900055
:10ca080091c0b300220037008a2eef0050748000d6
:10ca18006c00b90002e9200000014100f0ff270086
:10ca2800000978006000b800100198002101980002
:10ca38000000eb0030019800c3589000114998009d
:10ca48002358900000499800b35890002149980055
:10ca5800135890003049980041003700035890005f
:10ca68006f006000e10f50000b003200ef0f500024
:10ca7800290032000000e0003c003a0010c0b3007a
:10ca8800f1fd0700c07680002058900011c0b30067
:10ca98006bfe0700480037000040eb008059980003
:10caa800334090000014a000b041980070748000da
:10cab800e30f500028003c000000e8007074880074
:10cac80050748000e20f500003003c000000e800b2
:10cad80050748800010037008a2eef0050748000df
:10cae8006c00b90002e92000000141002007200085
:10caf800000978000308900093089000100198003e
:10cb080021019800b3089000310198000040eb0023
:10cb180010499800caff37000040eb008059980080
:10cb2800334090000014a000b04198007074800059
:10cb3800e30f500008003c000000e8007074880013
:10cb480050748000e20f5000afff3c000000e80086
:10cb580050748800adff370080c0b300b05998000a
:10cb68000800e00002003a00060037001800200024
:10cb78000040eb0080599800334090000014a0005a
:10cb8800b0419800d54ee20002003200d46eef00aa
:10cb98007dff3700d26ea800070037000040eb0089
:10cba80080599800334090000014a000b0419800cc
:10cbb80018002000f1fe37004f047800000006003e
:10cbc800889fbe008a9fbe008c1f780000467800b0
:10cbd8008105780002057800830478006876800073
:10cbe8000c00370078409000a2c0b3000440bc009d
:10cbf80064014100c0d62000e2017800614ab80013
:10cc08000a0178008b0078000c40780003000100ce
:10cc1800180478000800e000f2ff3a004f06780098
:10cc28004f05be004f04be00000006003600f800a5
:10cc3800809fbe00829fbe00849fbe00869fbe006c
:10cc48008ec0a90082c4bf000068a3001000320093
:10cc580080c4bf000068a3000d003200000420005b
:10cc680000248800da0ee20009003200da2eed0016
:10cc7800da0ee20006003a0082c4a900b07680000d
:10cc880001f020000100600001003200d62eec0007
:10cc98008cc4bf000068a3000c0032008ac4bf0027
:10cca8000068a300090032008cc4a9000004200019
:10ccb80050248800b176800070005000808f5000aa
:10ccc80002003a0000102000307488008cc4bf00b5
:10ccd8000008a300070032008ac4bf000008a300b0
:10cce8000400320010002000502488008c04a900a1
:10ccf800862eef008cc4bf000038a300ce0032009f
:10cd08008ac4bf000038a300cb0032008cc4bf0027
:10cd18000018a300080032008ac4bf000018a3004e
:10cd280005003200c07680003058900063406000f3
:10cd3800e14f5000c0003a00d28ea9009224800032
:10cd48008000200050248800c4768000a4589000f9
:10cd5800f0248000ef8060006f006000808f50003a
:10cd6800b4003a00020078000238a300050032003f
:10cd7800c20021000028a30006003a00820021001a
:10cd880004003700420021000028a30001003a00f7
:10cd98000200210000c023009200600000802000f3
:10cda800808f500037003a00f03f200012016000e9
:10cdb800040890009408900002004000e0804800b9
:10cdc800000a9800110a98000000eb00700a980009
:10cdd800344090004300de00610060000004a200bf
:10cde8004300dd00b44090000134a10080c0700011
:10cdf8003142980004589000f04f5000080032006b
:10ce08008458900000c2b30080cf50000400320064
:10ce1800845890007040400080cf500032003a00a3
:10ce2800040990009409900074009000010020000b
:10ce3800800f5100818f59007e0039006000b800d2
:10ce4800000a9800110a98000a00370004099000a7
:10ce58009409900054009000e4009000800f510065
:10ce6800818f590073003900344090000004a000fd
:10ce780030429800045890000040e800005a98009a
:10ce88006c00370000c02000808f50000300320083
:10ce980000c02200808f50001b003a00f03f2000a5
:10cea80012016000040890009408900002004000fd
:10ceb800e0804800000a9800110a98000000eb0082
:10cec800700a9800344090004300de006100600062
:10ced8000004a2004300dd00b44090000134a1002a
:10cee80080c0700031429800345890006340600060
:10cef800e14f5000dcff320044009000800f5100e9
:10cf0800d9ff3900d1ff370000802200808f500000
:10cf180021003a00344090000044a00030429800bc
:10cf2800740890000000e800700a980034589000d7
:10cf380063006000e10f5000cbff320003003c00ab
:10cf48000000e000080032003a003700e20f50000d
:10cf580005003200e30f500036003a0024589000d4
:10cf68000004e000c0ff3500344090000058a300e2
:10cf780030003200f408900004109000808f5000b8
:10cf88002c003600244090000064a0002042980045
:10cf980070c1b3000700370000802300808f500065
:10cfa8000a003a00244090000054a0002042980053
:10cfb80010c1b300405a98000458900001cfb30044
:10cfc80001406000f040b300acff3700a44090007f
:10cfd8008140e800ffc060002440900002ceb3000a
:10cfe80002406000014070002042980024409000f8
:10cff8007f006000f30f50000e00340024409000c2
:10d008000064a0002042980030c1b300405a980044
:10d018000458900001cfb30001406000f040b30015
:10d02800005a9800f00f200070248800200020008b
:10d03800502488001ffd07008cc4bf000028a300ef
:10d048002c0032008ac4bf000028a3002900320047
:10d058004000200050248800627680001b003700c2
:10d06800220090000000e00017003200a0009000ad
:10d078000330200005102000f4ceb3001000370064
:10d088005108900003006000830f50000200320036
:10d09800850f500006003a00310090000000e000c3
:10d0a80003003200310090000000e900b000980051
:10d0b8003140900004406000b04098009100780032
:10d0c8000100e000eeff3a00120178000200e000e3
:10d0d800e3ff3a00d20ea900d22ea900d24ea90031
:10d0e800d26ea9000001fd00d4eeb7000001fd00da
:10d0f800f0fc07008cc4bf000018a30043003200f6
:10d108008ac4bf000018a30040003200d28ea900d4
:10d11800c37680003358900063406000e14f5000b0
:10d1280036003200a34090008140e800ffc0600054
:10d138002340900002ceb30002406000014070001e
:10d14800a0419800234090007f006000f30f50003a
:10d158002a0034008e44e20002003d0000c2b30001
:10d16800c05998008ec4bf000058a30002003200c6
:10d1780010c2b300c05998008ec4bf000048a30075
:10d188000200320020c2b300c05998008ec4bf000c
:10d198000038a3000200320030c2b300c059980022
:10d1a8008ec4bf000028a3000200320040c2b300b2
:10d1b800c05998008ec4bf000018a30002003200b6
:10d1c80050c2b300c05998008ec4bf000008a30025
:10d1d8000200320060c2b300c0599800234090009a
:10d1e8000064a000a04198000358900001cfb3004c
:10d1f80001406000f040b30080599800f00f200013
:10d208007024880020002000502488004f03be00ae
:10d218004f02be004f01be004f00be003600f900ad
:10d228000040060020422a00031507000000eb001a
:10d238007069880060698800410020005169880091
:10d2480040698800507780006dec370000302f006f
:10d25800103a88008001eb00233a880053168800b2
:10d2680093168800d3168800131788005317880070
:10d278009317880000ec2c0040168800f0ff290066
:10d288008016880010f02f00c016880002fc2f00be
:10d298000217880040ff2f0040178800f0c32f00b6
:10d2a80080178800c8c2a800c8e2a800a9c6bf00a5
:10d2b800024060000014a000a9e6b700a8c6bf009d
:10d2c800024060000024a000a8e6b700aac6bf007c
:10d2d80002406000c040b300aae6b700c3c6bf0062
:10d2e800024060007040b300c3e6b700d802a8004f
:10d2f80081c6bf0002406000b040b30081e6b700bd
:10d30800aec0bf0081cfb300014060005040b30001
:10d31800aee0b7008220a9008680a9005700a800c7
:10d328005720a80057c0a80057e0a8005780a800b9
:10d3380057a0a8007300a800f30888001fa1a9003f
:10d348001ec1a9001ec1bf000044a1000054a000d6
:10d358001ee1b7001e61a9001e21a900a3088800cc
:10d36800409c2000d00888001fe1a800a6c6bf0086
:10d3780002406000a040b300a6e6b700d1c6bf00d7
:10d38800024060005040b300d1e6b7008f14070098
:10d3980080432a00a8140700f01f2f006019880096
:10d3a800601980000080ea008019880021c3bf004e
:10d3b800c1cfb3000140600021e3b70000ceb30045
:10d3c8002063b7002043a9002023a8002343a80016
:10d3d80023c3bf007f40600023e3b70022c3bf0020
:10d3e80031ccb300014060000034a00022e3b70054
:10d3f8002223a9002203a900f0f3210020198800a4
:10d4080021e3a80087ff070010000500881f7800a7
:10d418001000200070698800e3c62000934178005e
:10d42800f2c6200012417800c818dd000280fb0017
:10d43800008440006bccbf000080fb00010020008e
:10d4480061005000e0805800fa0f5000e08f58004b
:10d458002e013e000060010086003700870037007b
:10d46800a4003700b7003700d7003700270137007e
:10d4780026013700e2003700240137002301370076
:10d488002201370021013700200137000d00370045
:10d49800ef0037001d0137001c0137006500370019
:10d4a8001c01370019013700180137001701370030
:10d4b800ff0037001501370014013700130137004a
:10d4c8000e0137001000200070698800d0442a003f
:10d4d8005914070040b02000800f5400510032005a
:10d4e80007003e00c0302000800f54000e003200bc
:10d4f80000912000800f54004c003a000e003700c5
:10d50800c0a02100800f540044003200c040220017
:10d51800800f54003f003200c0302100800f5400bb
:10d5280042003a0039003700c0452a00421407007b
:10d53800100020004400370050462a003e1407001f
:10d54800262def000a003700e6004100b0c6200093
:10d5580061407800f1d1200000f178000080fb00e4
:10d56800de14070000c2b3002c140700262dec00bf
:10d5780032698000e50f5100f3ff340030482a007b
:10d588002d140700f1d12000914078008180fb0024
:10d5980020cdbf004800dd00010070001100200010
:10d5a8004bcf070011d22000914078008180fb000a
:10d5b80022cdbf004800dd000100700021002000de
:10d5c80043cf070031d22000914078008180fb00d2
:10d5d80024cdbf004800dd000100700031002000ac
:10d5e8003bcf07001000200086cd0700c7140700b6
:10d5f8002000200083cd0700c4140700300020005d
:10d6080080cd0700c1140700a6003700b0492a00e2
:10d61800a5003700904a2a00a3003700804b2a0053
:10d62800a1003700504d2a009f003700704e2a0095
:10d638009d0037006d4ce20005003a00004f2a00bb
:10d64800fd130700a000200060698800b1003700c2
:10d65800a0502a00f81307006dccbf000080fb0023
:10d668009e14070080492a00f31307002c2def00b1
:10d67800a800370070522a008b003700030078009a
:10d6880019edb700020078001aedb70070ccbf00a2
:10d698001bedb70071ccbf001cedb70072ccbf000a
:10d6a8001dedb70073ccbf001eedb700a0532a00d4
:10d6b800e1130700262def000700370090d1200066
:10d6c800614078000080fb008414070000c2b300aa
:10d6d800d2130700262dec0031698000e58f500039
:10d6e800f6ff340080492a00d31307007000200099
:10d6f800d5ff3700b0552a00cf130700a0582a00dd
:10d708006d4ce20062003a006eccbf0069ecb700d5
:10d718006fccbf006aecb70070572a00c613070029
:10d728006fccbf000080fb006c1407006eccbf00fc
:10d738000080fb006914070000022000606988006f
:10d748005800370060698000e60f500071003a0009
:10d7580020592a00b81307006dccbf0019edb70097
:10d768006eccbf001aedb7006fccbf001bedb70041
:10d7780070ccbf001cedb70071ccbf001dedb70029
:10d7880072ccbf001eedb700262def000700370052
:10d7980090d12000614078000080fb004f14070002
:10d7a80000c2b3009d130700262dec0031698000ec
:10d7b800e58f5000f6ff340080492a009e130700c9
:10d7c80080002000a0ff3700905b2a009a13070012
:10d7d8006d4ce20004003a00c05c2a009613070072
:10d7e8002c2def0002003700505d2a00921307002d
:10d7f80080492a00901307008afe07004500370079
:10d80800c05d2a008c1307006d4ce2000d003a0041
:10d8180000c7200011c0b30090cf100009003a00e3
:10d82800f05e2a00841307006eccbf000080fb0066
:10d838002a1407006fccbf000080fb0027140700e4
:10d8480018003700505d2a007b13070015003700c9
:10d85800e0602a00781307006dccbf000300320097
:10d86800e24f500009003a000500370050622a00d4
:10d878007113070020002000706988000900370034
:10d88800e0622a006c1307000500370010652a00c3
:10d89800691307006dccbf000080fb000f14070060
:10d8a8002c2def0080492a00631307001900370068
:10d8b800d0652a0060130700262def000800370006
:10d8c8008000e800b0c62000614078000080fb00be
:10d8d8000214070000c2b30050130700262dec0005
:10d8e80030698000e50f5000f5ff340080492a00b8
:10d8f80051130700c000200053ff370090672a002b
:10d908004d130700000220004fff370020002000c1
:10d91800706988004f04780000000600100020009d
:10d9280070698800b2cc20001241780002007800ab
:10d9380062ecb70081cc200091407800e1cf500024
:10d94800f7003a00caccbf00e44f50007a0032001a
:10d9580006003e00e24f50000c00320048003e0036
:10d96800e14f5000ec003a0006003700e64f500047
:10d978009900320091003900e74f5000e6003a0064
:10d98800bc003700d0682a00ee003700c06a2a00c1
:10d9980029130700ceccbf00e14f500012003a0017
:10d9a800cf4ce20034003a00806c2a0022130700b2
:10d9b800d1ccbf000080fb00c8130700d0ccbf004b
:10d9c8000080fb00c513070080492a001a130700ce
:10d9d800d0ccbf0063ecb700d1ccbf0064ecb7007b
:10d9e800d0002000ca003700f14f500010003a0064
:10d9f800cf4ce20020003a00006e2a000e13070008
:10da0800d1ccbf000080fb00b4130700d0ccbf000e
:10da18000080fb00b113070080492a0006130700a5
:10da2800d0ccbf0067ecb700d1ccbf0026003700d0
:10da3800f34f500010003a00cf4ce2000e003a00bd
:10da4800d06f2a00fc120700d1ccbf000080fb0079
:10da5800a2130700d0ccbf000080fb009f13070073
:10da680080492a00f4120700d0ccbf0065ecb7004b
:10da7800d1ccbf0021003700f0702a00b100370078
:10da8800e0722a00ec120700d2ccbf0020003a0056
:10da980030742a00e812070001cd20009140780078
:10daa80000c7b30080cf50000a003a00d14ce20012
:10dab80008003a00d0742a00df120700ceccbf005d
:10dac80067ecb700cfccbf0068ecb700200120009e
:10dad8008f00370010c7b30080cf50000a003a000b
:10dae800d14ce20008003a0030762a00d212070032
:10daf800ceccbf0065ecb700cfccbf0066ecb7005a
:10db0800600120008200370090772a008d003700de
:10db1800e14f500002003a0030782a0089003700af
:10db280000792a00c4120700d2ccbf000080fb0095
:10db38006a13070078003700007a2a00be1207002f
:10db4800e1cc20009140780000c7b30080cf50009e
:10db580006003a00cf4ce20004003a00707b2a002d
:10db6800b5120700500120006900370010c7b30044
:10db780080cf500006003a00cf4ce20004003a0083
:10db8800e07c2a00ac12070080012000600037000a
:10db980020c7b30080cf500006003a00cf4ce20007
:10dba80004003a00207e2a00a3120700f00020009b
:10dbb80057003700107f2a006200370010812a00c2
:10dbc8009d120700a0822a00d24ce2005d003200bc
:10dbd80040832a005b003700c0832a0096120700a2
:10dbe800e1cc20009140780010c7b30080cf5000ee
:10dbf80008003a00cf4ce20006003a001007200067
:10dc08003613070000852a008b120700b001200098
:10dc18003f00370000c7b30080cf500008003a002b
:10dc2800cf4ce20006003a00000720002b13070043
:10dc380090852a0080120700c001200034003700b8
:10dc480020c7b30080cf500008003a00cf4ce20054
:10dc580006003a00200720002013070020862a002b
:10dc6800751207001001200029003700a0862a003d
:10dc780034003700e0872a006f120700e1cc20004b
:10dc88009140780065ccbf00000ce10009003a0023
:10dc980066ccbf00cf4ce30006003a000180fb00d1
:10dca8000e13070000852a0063120700e001200018
:10dcb8001700370067ccbf00000ce10009003a00ec
:10dcc80068ccbf00cf4ce30006003a000180fb009f
:10dcd8000213070090852a0057120700f001200060
:10dce8000b00370063ccbf00000ce10022003a00b3
:10dcf80064ccbf00cf4ce3001f003a000180fb005a
:10dd0800f612070020862a004b12070000022000a6
:10dd1800606988000000060080492a000900370071
:10dd280020c7b30080cf500007003a0030892a008e
:10dd380041120700caccbf00e64f50000e003a005f
:10dd4800d0892a003c12370010c7b30080cf50009a
:10dd580009003a00a1cc20009140780010cab30015
:10dd680080cf500004003a00f14f510002003a0001
:10dd780050778000a708070000000600b0c6200002
:10dd880011c0b30090cf100001003a00a1080700ad
:10dd98000000060076cebf00304de30005003a00d3
:10dda800810eab000300320081e72000914078002b
:10ddb800010037008040eb00b0c620009d08370006
:10ddc800b0c6200011c0b30090cf100001003a0087
:10ddd800ee09070000000600881f780030cdbf005c
:10dde80011100700004478000004e000060032002b
:10ddf800608b2a00101207000880fb00b71207008a
:10de080080492a000c1207000880fb004f047800a4
:10de180000000600881f7800cf91de0030cdbf00db
:10de280027100700004478000004e00004003200d6
:10de38000080fb00a9120700a08c2a00fe11070031
:10de480000e82300010020004bce07000880fb00fb
:10de58004f047800000006001c6cec0069100700f5
:10de6800e10f500003003200e20f500011003a00a9
:10de780009003700418e2a0020c22000d7c90700b8
:10de8800c80d0700800078007205200020c220001d
:10de9800e0ff07000a003700c00d07008000780087
:10dea80030cdbf000202200003002000bd0f070094
:10deb80003003700008f2a00df11070030c0b300cd
:10dec8000080fb0000000600881f7800626cec00f0
:10ded80030cdbf0061e72000914078000104e100e7
:10dee80002003a00810eab0005003a000004e00091
:10def80003003200cbfc07000000eb00610e0700b6
:10df080070698000e10f50000a00320003003900f8
:10df1800e20f500082043a007604370030912a005c
:10df2800c511070010002000706988002c2def0033
:10df38007e04370060698000010020000202200092
:10df4800820f5000e08f580078043e000060010006
:10df580020003700370037004800370062003700dc
:10df68007700370083003700970037009c003700a0
:10df7800c300370064043700df003700e0003700d3
:10df8800eb003700240137005c01370088013700b7
:10df9800b6013700d901370029023700fb013700e5
:10dfa800600237008c023700b4023700ec023700f9
:10dfb80022033700500337004e0437009803370018
:10dfc800bb033700e8033700070437003304370082
:10dfd800480437000004eb00d860880050778000c0
:10dfe80007e9070000a0260081012000e2cd070014
:10dff80030c0b3006becb700c0c0b3006cecb70026
:10e00800080078006decb700a1912a0020c220001a
:10e0180072c9070032002000b1c6200020c22000cb
:10e028006dff07000004e00040043a0010002000e3
:10e038002a00370090c0b3006becb70000c1b300f2
:10e048006cecb7006d6cef00a1922a0020c2200092
:10e0580062c9070032002000b1c6200020c220009b
:10e068005dff07000004e00030043a0020002000b3
:10e0780060698800706988002c04370030c1b300db
:10e088006becb700c0c0b3006cecb70040c0b30085
:10e098006decb70031c4b300010078006eecb70036
:10e0a80000c5b3006fecb7000100780070ecb70052
:10e0b800716cef0011942a0020c2200047c90700a4
:10e0c80072002000b1c6200020c2200042ff0700d5
:10e0d8000004e00015043a00300020006069880060
:10e0e80020002000e3ff370040c2b3006becb7000c
:10e0f800c0c0b3006cecb70030c0b3006decb70023
:10e1080080c0b3006eecb70050c0b3006fecb7002e
:10e11800706cef0061952a0020c220002fc907000b
:10e1280062002000b1c6200020c220002aff07009c
:10e138000004e000fd033a0040002000e7ff37003c
:10e14800a0c1b3006becb700c0c0b3006cecb70063
:10e1580010c0b3006decb70030c0b3006eecb70070
:10e16800d1962a0020c220001cc9070042002000c6
:10e178003c00370010c0b3006becb70040c0b300e0
:10e188006cecb70050c0b3006decb70030c3b300ff
:10e198006eecb700b0c8b3006fecb7007340400036
:10e1a80070ecb70000c3b30071ecb700a0c0b300b7
:10e1b80072ecb70031982a0020c2200007c9070076
:10e1c800820020002700370030cdbf0072052000f4
:10e1d80003002000b1c62000ce0e0700c0ff3700a4
:10e1e80050c0b3006becb70040c0b3006cecb70094
:10e1f800d0c0b3006decb70019cdbf006eecb7000e
:10e208001acdbf006fecb7001bcdbf0070ecb70094
:10e218001ccdbf0071ecb7001dcdbf0072ecb7007c
:10e228001ecdbf0073ecb70080c1b30074ecb7001b
:10e23800c0ccb30075ecb70010c0b30076ecb700e3
:10e248000040eb0077ecb70078ecb70079ecb7004a
:10e258007aecb70051992a0020c22000dfc80700d5
:10e2680002012000b1c6200020c22000dafe07000b
:10e278000004e000ad033a006000200097ff37007b
:10e2880090c0b3006becb70040c0b3006cecb700b3
:10e2980070c0b3006decb70019cdbf006eecb700cd
:10e2a8001acdbf006fecb7001bcdbf0070ecb700f4
:10e2b8001ccdbf0071ecb7001dcdbf0072ecb700dc
:10e2c8001ecdbf0073ecb700746cef00119b2a00e1
:10e2d80020c22000c1c80700a2002000b1c620004b
:10e2e80020c22000bcfe07000004e0008f033a00b3
:10e2f8009000200079ff3700b00020001803370095
:10e30800a0c1b3006becb700c0c0b3006cecb700a1
:10e3180010c0b3006decb7006e6cef00219e2a00b0
:10e3280020c22000adc80700420020003600370098
:10e33800b0c0b3006becb70040c0b3006cecb700e2
:10e3480060c1b3006decb70019cdbf006eecb7002b
:10e358001acdbf006fecb7001bcdbf0070ecb70043
:10e368001ccdbf0071ecb7001dcdbf0072ecb7002b
:10e378001ecdbf0073ecb70060c5b30074ecb700e6
:10e3880080ceb30075ecb70010c8b30076ecb700c8
:10e3980080c3b30077ecb70080c0b30078ecb70057
:10e3a80060c0b30079ecb70010c5b3007aecb700d1
:10e3b800704050007becb70000ccb3007cecb70099
:10e3c800f0c7b3007decb70020c1b3007eecb70006
:10e3d800a0cab3007fecb70090cdb30080ecb700c3
:10e3e80060c6b30081ecb700c0c3b30082ecb700cd
:10e3f800e0ccb30083ecb700919f2a0020c2200034
:10e4080076c8070092012000b1c6200020c2200073
:10e4180071fe07000502370069ccbf00c2ecb700e7
:10e428006accbf000042b000c3ecb70000c1b30023
:10e43800c4ecb7008040eb0001007800c5ecb700e1
:10e44800c0c0b300c6ecb70001007800c7ecb70045
:10e4580010c0b300c8ecb70001007800c9ecb700e1
:10e4680030c0b300caecb70062ccbf00cbecb70039
:10e4780080c0b300ccecb70001007800cdecb70049
:10e4880020c7b300ceecb70001007800cfecb7008e
:10e4980063ccbf00d0ecb70064ccbf00d1ecb700b0
:10e4a8008000fd00d2ecb700d3ecb700d4ecb70085
:10e4b800d5ecb7008000fd00a0a02a005e10070080
:10e4c800000720000511070080492a005a1007009c
:10e4d80071a12a0020c2200040c807004201200084
:10e4e80021cc200020c220004afe07000004e000e2
:10e4f8000e033a00e00020009902370069ccbf0003
:10e50800c2ecb7006accbf000042b000c3ecb70051
:10e5180000c1b300c4ecb7008040eb0001007800f4
:10e52800c5ecb700c0c0b300c6ecb7000100780066
:10e53800c7ecb70012c0b30002007800c8ecb700ff
:10e5480001007800c9ecb70040c0b300caecb700be
:10e5580002007800cbecb70080c0b300ccecb70069
:10e5680001007800cdecb70063ccbf00ceecb7005b
:10e5780064ccbf00cfecb7008000fd00d0ecb70042
:10e58800d1ecb7008000fd0002007800d2ecb700a3
:10e5980020c0b300d3ecb70000c4b300d4ecb7007c
:10e5a80001007800d5ecb700e1a22a0099013700f4
:10e5b80069ccbf00c2ecb7006accbf000042b00013
:10e5c800c3ecb700e0c0b300c4ecb7008040eb0078
:10e5d80001007800c5ecb700a0c0b300c6ecb700d6
:10e5e80001007800c7ecb70010c0b300c8ecb70052
:10e5f80001007800c9ecb70050c0b300caecb700fe
:10e6080062ccbf00cbecb70060c0b300ccecb70065
:10e6180001007800cdecb70063ccbf00ceecb700aa
:10e6280064ccbf00cfecb7008000fd00d0ecb70091
:10e63800d1ecb700d2ecb700d3ecb7008000fd00f6
:10e6480031a42a0020c22000e4c7070022012000cc
:10e6580021cc200020c22000eefd07000004e000cd
:10e66800b2023a00000120009cfe370069ccbf00ce
:10e67800c2ecb7006accbf000042b000c3ecb700e0
:10e68800c0c0b300c4ecb7008040eb0001007800c4
:10e69800c5ecb70080c0b300c6ecb7000100780035
:10e6a800c7ecb70010c0b300c8ecb7000100780091
:10e6b800c9ecb70060c0b300caecb70062ccbf00b9
:10e6c800cbecb70040c0b300ccecb7000100780039
:10e6d800cdecb70063ccbf00ceecb70064ccbf0074
:10e6e800cfecb70020c7b300d0ecb700010078002a
:10e6f800d1ecb70091a52a004d00370069ccbf00c6
:10e70800c2ecb7006accbf000042b000c3ecb7004f
:10e71800c0c0b300c4ecb7008040eb000100780033
:10e72800c5ecb70080c0b300c6ecb70001007800a4
:10e73800c7ecb70010c0b300c8ecb7000100780000
:10e74800c9ecb70060c0b300caecb70062ccbf0028
:10e75800cbecb70040c0b300ccecb70001007800a8
:10e76800cdecb70020c7b300ceecb70001007800ad
:10e77800cfecb70063ccbf00d0ecb70064ccbf00cf
:10e78800d1ecb70041a72a00b800370069ccbf0018
:10e79800c2ecb7006accbf000042b000c3ecb700bf
:10e7a800c0c0b300c4ecb7008040eb0001007800a3
:10e7b800c5ecb70080c0b300c6ecb7000100780014
:10e7c800c7ecb70010c0b300c8ecb7000100780070
:10e7d800c9ecb70020c0b300caecb70062ccbf00d8
:10e7e800cbecb70040c0b300ccecb7000100780018
:10e7f800cdecb70010c1b300ceecb7000100780033
:10e80800cfecb70000c7b300d0ecb7000100780028
:10e81800d1ecb700a0a02a00870f0700000720004e
:10e828002e10070080492a00830f0700e1a82a005c
:10e8380020c2200069c7070002012000f800370045
:10e8480069ccbf00c2ecb7006accbf000042b00080
:10e85800c3ecb70000c1b300c4ecb7008040eb00c4
:10e8680001007800c5ecb700c0c0b300c6ecb70023
:10e8780001007800c7ecb70010c0b300c8ecb700bf
:10e8880001007800c9ecb70030c0b300caecb7008b
:10e8980062ccbf00cbecb70080c0b300ccecb700b3
:10e8a80001007800cdecb70000c7b300ceecb7008c
:10e8b80001007800cfecb70067ccbf00d0ecb70000
:10e8c80068ccbf00d1ecb7008000fd00d2ecb700e7
:10e8d800d3ecb700d4ecb700d5ecb7008000fd004e
:10e8e800a0a02a00540f070000072000fb0f070014
:10e8f80080492a00500f070041aa2a0020c22000a0
:10e9080036c707004201200021cc200020c2200089
:10e9180040fd07000004e00004023a004001200026
:10e928008f01370069ccbf00c2ecb7006accbf00ca
:10e938000042b000c3ecb70000c1b300c4ecb7009c
:10e948008040eb0001007800c5ecb700c0c0b30000
:10e95800c6ecb70001007800c7ecb70012c0b300de
:10e9680002007800c8ecb70001007800c9ecb700d5
:10e9780040c0b300caecb70002007800cbecb70087
:10e9880080c0b300ccecb70001007800cdecb70034
:10e9980067ccbf00ceecb70068ccbf00cfecb700a7
:10e9a8008000fd00d0ecb700d1ecb7008000fd007e
:10e9b80002007800d2ecb70020c0b300d3ecb70057
:10e9c80000c4b300d4ecb70001007800d5ecb70060
:10e9d800b1ab2a008f00370069ccbf00c2ecb7008a
:10e9e8006accbf000042b000c3ecb700e0c0b3007f
:10e9f800c4ecb7008040eb0001007800c5ecb7001c
:10ea0800a0c0b300c6ecb70001007800c7ecb7009f
:10ea180010c0b300c8ecb70001007800c9ecb7001b
:10ea280050c0b300caecb70062ccbf00cbecb70053
:10ea380060c0b300ccecb70001007800cdecb700a3
:10ea480067ccbf00ceecb70068ccbf00cfecb700f6
:10ea58008000fd00d0ecb700d1ecb700d2ecb700d5
:10ea6800d3ecb7008000fd0001ad2a0020c22000d1
:10ea7800dac60700220120006900370069ccbf0010
:10ea8800c2ecb7006accbf000042b000c3ecb700cc
:10ea980000c1b300c4ecb7008040eb00010078006f
:10eaa800c5ecb700c0c0b300c6ecb70001007800e1
:10eab800c7ecb70010c0b300c8ecb700010078007d
:10eac800c9ecb70030c0b300caecb70062ccbf00d5
:10ead800cbecb70080c0b300ccecb70001007800e5
:10eae800cdecb70010c7b300ceecb700010078003a
:10eaf800cfecb70065ccbf00d0ecb70066ccbf0048
:10eb0800d1ecb7008000fd00d2ecb700d3ecb70021
:10eb1800d4ecb700d5ecb7008000fd0060ae2a0049
:10eb2800c50e0700100720006c0f070080492a0057
:10eb3800c10e070031af2a0020c22000a7c6070077
:10eb48004201200021cc200020c22000b1fc070097
:10eb58000004e00075013a00700120000001370050
:10eb680069ccbf00c2ecb7006accbf000042b0005d
:10eb7800c3ecb70000c1b300c4ecb7008040eb00a1
:10eb880001007800c5ecb700c0c0b300c6ecb70000
:10eb980001007800c7ecb70013c0b3000300780089
:10eba800c8ecb70001007800c9ecb70040c0b3005a
:10ebb800caecb70022c0b30002007800cbecb70063
:10ebc80080c0b300ccecb70001007800cdecb700f2
:10ebd80065ccbf00ceecb70066ccbf00cfecb70069
:10ebe8008000fd00d0ecb700d1ecb7008000fd003c
:10ebf80003007800d2ecb70002007800d3ecb7002d
:10ec080000c4b300d4ecb70001007800d5ecb7001d
:10ec1800a1b02a0020c2200070c6070042012000cf
:10ec280021cc200020c220007afc07000004e0006c
:10ec38003e013a0000022000c900370069ccbf003d
:10ec4800c2ecb7006accbf000042b000c3ecb7000a
:10ec5800e0c0b300c4ecb7008040eb0001007800ce
:10ec6800c5ecb700a0c0b300c6ecb700010078003f
:10ec7800c7ecb70010c0b300c8ecb70001007800bb
:10ec8800c9ecb70050c0b300caecb70062ccbf00f3
:10ec9800cbecb70060c0b300ccecb7000100780043
:10eca800cdecb70065ccbf00ceecb70066ccbf009a
:10ecb800cfecb7008000fd00d0ecb700d1ecb70076
:10ecc800d2ecb700d3ecb7008000fd00f1b12a0008
:10ecd80020c2200041c607002201200021cc2000cc
:10ece80020c220004bfc07000004e0000f013a009e
:10ecf80090012000f9fc37002a0a0700811f7800dc
:10ed080091c6200011487800cf007800250a070036
:10ed1800a1c62000914078000142b000114098003f
:10ed2800200a070031c5b300214098001d0a0700da
:10ed38000044eb00384098001a0a0700f1c4b300f9
:10ed480041409800170a070058409800150a070024
:10ed580071c620009140780061409800110a0700b0
:10ed680082c6200012417800724098000d0a070000
:10ed780021c5b300014898000a0a070011c1b30071
:10ed880011489800070a070001c8b30021489800f5
:10ed9800040a070038489800020a070080c0eb0000
:10eda80041489800ff09070058489800fd090700e6
:10edb8006848980069ccbf00c2ecb7006accbf00b5
:10edc8000042b000c3ecb70060c0b300c4ecb700a9
:10edd80008007800c5ecb70021c0b3000100780036
:10ede800c6ecb70008007800c7ecb70067ccbf00d6
:10edf800c8ecb70068ccbf00c9ecb70030c4b3009a
:10ee0800caecb70001007800cbecb70051b32a0078
:10ee180020c22000f1c50700a20020004a003700e8
:10ee280069ccbf00c2ecb7006accbf000042b0009a
:10ee3800c3ecb700c0c0b300c4ecb7008040eb001f
:10ee480001007800c5ecb70080c0b300c6ecb7007d
:10ee580001007800c7ecb70010c0b300c8ecb700d9
:10ee680001007800c9ecb70070c0b300caecb70065
:10ee780062ccbf00cbecb70040c0b300ccecb7000d
:10ee880001007800cdecb70010c7b300ceecb70096
:10ee980001007800cfecb70065ccbf00d0ecb7001c
:10eea80066ccbf00d1ecb70061b52a00230037005b
:10eeb80069ccbf00c2ecb7006accbf000042b0000a
:10eec800c3ecb700c0c0b300c4ecb7008040eb008f
:10eed80001007800c5ecb70080c0b300c6ecb700ed
:10eee80001007800c7ecb70010c0b300c8ecb70049
:10eef80001007800c9ecb70070c0b300caecb700d5
:10ef080062ccbf00cbecb70040c0b300ccecb7007c
:10ef180001007800cdecb70000c7b300ceecb70015
:10ef280001007800cfecb70067ccbf00d0ecb70089
:10ef380068ccbf00d1ecb70031b72a0020c220004e
:10ef4800a6c507000201200021cc200020c2200015
:10ef5800b0fb07000004e00074003a00a0012000a4
:10ef6800606988007100370069ccbf00c2ecb70047
:10ef78006accbf000042b000c3ecb700c0c0b30009
:10ef8800c4ecb7008040eb0001007800c5ecb70086
:10ef980080c0b300c6ecb70001007800c7ecb7002a
:10efa80010c0b300c8ecb70001007800c9ecb70086
:10efb80060c0b300caecb70062ccbf00cbecb700ae
:10efc80040c0b300ccecb70001007800cdecb7002e
:10efd80065ccbf00ceecb70066ccbf00cfecb70065
:10efe80010c7b3001f00370069ccbf00c2ecb700e0
:10eff8006accbf000042b000c3ecb700c0c0b30089
:10f00800c4ecb7008040eb0001007800c5ecb70005
:10f0180080c0b300c6ecb70001007800c7ecb700a9
:10f0280010c0b300c8ecb70001007800c9ecb70005
:10f0380060c0b300caecb70062ccbf00cbecb7002d
:10f0480040c0b300ccecb70001007800cdecb700ad
:10f0580067ccbf00ceecb70068ccbf00cfecb700e0
:10f0680000c7b300d0ecb70001007800d1ecb700be
:10f0780001b92a0020c2200058c50700020120005b
:10f0880021cc200020c2200062fb07000004e00021
:10f0980026003a000002200010fc370060c0b300d0
:10f0a8006becb70040c0b3006cecb70030c0b300e5
:10f0b8006decb70069ccbf006eecb7006accbf003e
:10f0c8006fecb70030c1b30070ecb70081ba2a000a
:10f0d80020c2200041c5070062002000b1c6200000
:10f0e80020c220003cfb07000004e0000f003a00ab
:10f0f8000d00370030cdbf0072052000030020004e
:10f1080021cc20008f0b070030cdbf0072052000f6
:10f1180003002000b1c62000fe0a070003003700e4
:10f1280090bb2a00440d07003ef807004f04780002
:10f13800000006000600fa00881f780030cdbf00e6
:10f1480061e72000914078000104e10002003a00e4
:10f15800810eab0005003a000004e0000300320015
:10f1680030f807000000eb00c6090700506980006e
:10f17800e20f5000a600320005003e000000e0004b
:10f1880009003200e10f50002d013a00300037002d
:10f19800e40f5000f6003200ca003900e50f5000b5
:10f1a80027013a0019013700f0bc2a00220d070098
:10f1b80030cdbf008f87e8008040eb00e1ff9f0063
:10f1c80017c0b300b6c62000050120000002eb00fe
:10f1d800233120000741780011cab3003dec070035
:10f1e8008f87e9000004e00015013a0002003700ab
:10f1f80010be2a00100d070030cdbf00e681570071
:10f20800688157008040eb00a9ee07000000e0008d
:10f21800f7ff32001000200050698800262def000b
:10f2280007003700b0c62000614078000080fb006e
:10f23800aa0d070000c2b300f80c0700262dec0049
:10f2480031698000ef8f5000f6ff3400c6003700a8
:10f2580010c02a00f80c07001000200069c607003b
:10f268001fedb7004800de0020edb70020002000a9
:10f2780064c6070021edb7004800de0022edb700a4
:10f28800300020005fc607000081fb000001fd0080
:10f2980023edb7000001fd00c801de00030078007f
:10f2a80024edb70031c1b300010078006becb70062
:10f2b8001fcdbf006cecb70020cdbf006decb700d0
:10f2c80021cdbf006eecb70022cdbf006fecb700b8
:10f2d8000200780070ecb7000300780071ecb7000a
:10f2e80060c5b30072ecb70080ceb30073ecb70012
:10f2f80010c8b30074ecb70080c3b30075ecb70056
:10f3080080c0b30076ecb70060c0b30077ecb700fc
:10f3180010c5b30078ecb7007040500079ecb70026
:10f3280000ccb3007aecb700f0c7b3007becb700b1
:10f3380020c1b3007cecb700a0cab3007decb700d5
:10f3480090cdb3007eecb70060c6b3007fecb70089
:10f35800c0c3b30080ecb700e0ccb30081ecb700c9
:10f3680030cdbf008f87e8008043eb00e7ff9f00a8
:10f37800b6c62000750120000002eb0033312000e2
:10f3880092c0b300eec04000d2eb07008f87e900bf
:10f398000004e000030032000e00370010c32a000a
:10f3a800a50c070030cdbf00e681570068815700e3
:10f3b8008040eb003eee07000000e000f7ff32005f
:10f3c80020c52a009c0c07002000200050698800f6
:10f3d8000200370090c52a00970c0700262def0081
:10f3e80007003700b0c62000614078000080fb00ad
:10f3f8003a0d070000c2b300880c0700262dec0068
:10f4080031698000f68f5000f6ff3400560037004f
:10f4180000c72a00880c070040c1b3006becb70096
:10f4280020c0b3006cecb7008043eb008003fd0004
:10f438006decb7006eecb7006fecb70070ecb7007e
:10f4480071ecb7008003fd008003fd0072ecb7008b
:10f4580073ecb70074ecb70075ecb70076ecb70046
:10f468008003fd008003fd0077ecb70078ecb7005f
:10f4780079ecb7007aecb7007becb7008003fd00ad
:10f4880030cdbf008f87e800e7ff9f00b6c6200099
:10f49800150120000002eb004331200092c0b300a8
:10f4a80011c2b3008beb07008f87e9000004e0006e
:10f4b80063003a00300020005069880010c82a0014
:10f4c8005e003700f0bc2a005b0c070030cdbf009f
:10f4d8008f87e8008040eb00e1ff9f0017c0b30072
:10f4e800b6c62000050120000002eb0023312000f1
:10f4f8000741780011cab30076eb07008f87e9004f
:10f508000004e0004e003a000200370010be2a0056
:10f51800490c070030cdbf00e681570068815700cd
:10f528008040eb00e2ed07000000e000f7ff32004a
:10f538004000200050698800262def0007003700a2
:10f54800b0c62000614078000080fb00e30c070093
:10f5580000c2b300310c0700262dec003169800091
:10f56800ef8f5000f6ff340080492a00330037003f
:10f578000a08070051c0b3000148780007080700cf
:10f5880080c0eb0011409800040807000044eb001d
:10f59800284098000108070038409800d1e3070088
:10f5a8008841780008417800804078009000200069
:10f5b800fe07070008407800720807000840780036
:10f5c80069080700f50707008000780030cdbf0004
:10f5d8000202200003002000f2090700004478001e
:10f5e800c0c82a00140c07000804e00003003a0011
:10f5f8005000200050698800110037000880fb0087
:10f60800b60c070090c52a000c00370030cdbf00ab
:10f618007205200003002000b1c62000bd090700c4
:10f628000004e00006003200e24f500004003200ff
:10f638000080fb00a90c070050ca2a00fe0b070037
:10f6480000882300110020004bc807004f047800f1
:10f658000080fa0000000600406980000000e00019
:10f6680003003200e10f50000c003a00060037009a
:10f67800c60707008040eb005140980010002000aa
:10f68800406988000000060030cdbf00020220005b
:10f6980003002000b1c620009e09070000000600f4
:10f6a800881f780000072000808f50007d003200fe
:10f6b8000f003e0064005000808f5000710032003f
:10f6c80006003e0067005000808f50006b0032003b
:10f6d8007800390070f92f000d003700e00620008f
:10f6e800808f50006b0032006c003e0067003700ce
:10f6f80000192000808f50001800320008003e00da
:10f7080010072000808f500068003200c0f82f00da
:10f7180000804000e10f500066003e0063003700a3
:10f7280030192000808f50002500320004003e0070
:10f738000080e900808f50005e003a001a00370010
:10f7480040192000808f50003b003200f0ff270056
:10f75800808f500057003a0054003700e60f5200df
:10f76800e08f5a0053003a004240900030edb70055
:10f7780018002000786988000000eb0060698800a4
:10f7880050698800e0cb2a00ab0b070030cdbf00e2
:10f79800b40b070030cf2a00a70b070030cf2a0090
:10f7a800a50b07003300370060cf2a00a20b070023
:10f7b8009cf607000000eb00320807003b0037000a
:10f7c80076cebf00304de30038003a00810eab0022
:10f7d80036003200c0738000d1738000e00f500003
:10f7e800e08f580031003200060a0700e20f50008f
:10f7f8000b00320003003e00e10f50002b003a00de
:10f8080005003700e30f500007003200e40f5000f6
:10f8180026003a0006003700fcf6070023003700f0
:10f8280056f90700210037005af907001f00370072
:10f8380063f907001d00370076cebf00304de300a6
:10f848001a003a00810eab0018003200e073800005
:10f85800f1738000e00f5000e08f58001300320071
:10f86800e809070000047800e10f50000f003a0093
:10f878002af80700080078000f003700d0d12a00c6
:10f888000900370000d52a000700370040d82a00b1
:10f898000500370080db2a000300370070df2a00ec
:10f8a8000100370060e22a00630b07001000200007
:10f8b800010037000000eb004f047800000006004c
:10f8c800889fbe008a9fbe008c9fbe005ff607001f
:10f8d800e10f500005003200e0e42a00560b070053
:10f8e80030e52a00540b0700ffff37006000b8001e
:10f8f800b1ec0700e10f50000b003a00c0e72a0006
:10f908004d0b0700e0e42a004b0b0700d0e92a0062
:10f91800490b070020ea2a00470b0700ca42e20009
:10f928000600350009003700e0e42a00420b070012
:10f9380000ee2a00400b0700ffff370050f02a00b6
:10f948003d0b0700600c0700feff3700f6c50700f7
:10f95800ec6eef00a0f12a00370b07000000eb0067
:10f96800a8c40700710b070080492a00320b070062
:10f978000000eb00a3c40700d8122000880f500035
:10f988000d0032008000eb0010002000f7e20700b5
:10f998008000eb00080078004dc607000004e00076
:10f9a80008003a00a0f22a00230b070028db070012
:10f9b8000000fe00030037001fdb0700d0f32a0019
:10f9c8001d0b0700507780008de207009760a800a4
:10f9d800b1c0bf00f1c8b300014060000044a000fe
:10f9e800b1e0b700890907009680a800a8d90700e8
:10f9f8000046eb008c4678002e0c070032c2bf0090
:10fa08000008a30017003200b011800000447800fd
:10fa180040c5b300804f54000700320078404000d2
:10fa2800804f54000c003200fb4f54000b003a008a
:10fa38002de907000900370020c5b30080cf560024
:10fa480006003a000040e800804f560003003a00e4
:10fa58000000fe0001003700f7da07008c46780046
:10fa6800084678008dee070066090700e20f50008f
:10fa78000d00320003003e00e10f50000b003a0079
:10fa880005003700e30f500005003200e40f500076
:10fa980006003a00040037000bf90700030037009e
:10faa800edfe070001003700a2fd07006069800035
:10fab800fa0f50000600320050698000e50f500030
:10fac8000300320040698000e10f50007f003a00d7
:10fad800e4a2a9004b090700e10f500020003a00fa
:10fae800a20607009080fb00104090004800dd004f
:10faf80001007000c8122000880f50000c0036006a
:10fb08009a060700e04090008180fb00704090005a
:10fb18004800dd0001007000880f50000400360026
:10fb280070f52a00c40a0700d00120006069880027
:10fb3800d1da07000000e000090032004f07070093
:10fb480000047800ccda0700800f54000400360067
:10fb5800a0f62a00b80a0700d001200060698800d2
:10fb6800890a0700104078006240600003003200f4
:10fb7800850a0700604090000200370010188000d6
:10fb88004200de001fecb7007f0a07001040780033
:10fb980064406000030032007b0a07007040900058
:10fba80002003700201880004200de001eecb7007b
:10fbb8000018800072062000110009000280d80099
:10fbc800e8eeb70090698000e90f50005300360056
:10fbd800e4a2a800322def00180ce2002f003a0032
:10fbe8001fccbf00e70607001eccbf00de060700db
:10fbf800650a07001040780061406000100032007c
:10fc0800610a0700d04590005f0a07004045900050
:10fc18005d0a0700b04490005b0a0700204490008a
:10fc2800590a0700104090000b4278008a4178007a
:10fc38000941780088407800c4060700170037009b
:10fc48002ae20700ea0f500003003200eb0f5000d1
:10fc58000b003a000700370022e207008000780016
:10fc6800e8cebf000080fb008041eb000341780034
:10fc78000900370010002000c906070007003700f8
:10fc880018e207000004780018e207008041eb0042
:10fc98000341780088407800440607000000eb0024
:10fca800e80607000000eb00bd060700d5080700be
:10fcb800e10f500003003200d2080700e20f5000a5
:10fcc80016003a0064f8070014003700e4a2a900ff
:10fcd800550507002d06070000c8eb00c06080002e
:10fce800e10f500003003a00182cef00c0608000bc
:10fcf80086e207009169800060092000808f50002b
:10fd080001003a00e4a2a80091698000000a2000de
:10fd1800808f500001003600322def0000e82300ec
:10fd28000100200094c6070033ff37003600f800b2
:10fd3800809fbe00829fbe00849fbe00869fbe003b
:10fd4800881f78003400f80000002000a001880017
:10fd5800b2050700322dec000c0607001902070057
:10fd6800b6dc070032050700000607009080fb009c
:10fd7800104090004800dd0001007000c81220000b
:10fd8800880f50000a003600f805070080609000d0
:10fd98008180fb00106090004800dd0001007000c9
:10fda800880f50000200360010002000c060880054
:10fdb800c0608000e10f500004003a00c06080007d
:10fdc80052e20700c0608800020037006000b800f7
:10fdd8002bda070085a0a9002023a8008760a900c6
:10fde8003400f9004f0478004f03be004f02be00f4
:10fdf8004f01be004f00be003600f900004006006b
:10fe08003600f800809fbe00829fbe00849fbe001f
:10fe1800869fbe003400f80000002000a001880082
:10fe28001c003700b1608000c0032000808f5000a4
:10fe38000a003c00d4090700b2608000411280002b
:10fe480001717800d1050700b16080006140780039
:10fe58000080fb00401288000d003700b160800070
:10fe680070052000808f500005003c00c80907007d
:10fe7800160cb40030c097000080fb00010037006a
:10fe8800c00a200040128800401280001decb70014
:10fe9800162cec0040c2bf000018a30003003a0073
:10fea80040c2bf000058a300deff32008540a90011
:10feb8003400f9004f03be004f02be004f01be00e0
:10fec8004f00be003600f90000400600809fbe00cb
:10fed8003400f80000002000a00188004142e20040
:10fee8000300350012003700b00a200040128800d5
:10fef80040c2bf000018a300fbff3200d1c12000a0
:10ff0800914078000200370040128000804078005d
:10ff180040c2bf000058a300fbff32000100780078
:10ff28001decb700162cef0040c2a9008680a9007e
:10ff38003400f9004f00be00004006003600f8000b
:10ff4800809fbe00829fbe00849fbe00869fbe0029
:10ff58003400f80000002000a001880050c4b3005d
:10ff6800ae090700000000003400f9004f03be008e
:10ff78004f02be004f01be004f00be003600f90020
:10ff8800004006003600f800809fbe00829fbe0039
:10ff9800849fbe00869fbe003400f8000000200049
:10ffa800a0018800a0f72a00a30907000040060066
:10ffb8003400f9004f03be004f02be004f01be00df
:10ffc8004f00be003600f900004006003600f80079
:10ffd800809fbe00829fbe00849fbe00869fbe0099
:10ffe8003400f80000002000a001880050f82a0022
:10fff80091090700004006003400f9004f03be00d5
:020000040001f9
:100008004f02be004f01be004f00be003600f9008f
:10001800004006008000eb0063af2000d203200000
:10002800e0f178008100e800828f5000fcff3a0080
:100038000000060000037800814378008001780002
:1000480010407800e24f500083003200e34f500028
:10005800be003200e14f50004b013a00e7cf50009c
:1000680002003200edcf500047013a009340900063
:100078008180fb00234090004800dd0001007000f3
:1000880022002000110009000200d800f507200016
:1000980080824200f00f2000808f5200020034005e
:1000a80080027800030037000500e00001003d00f1
:1000b8008002eb00b34090008180fb004340900039
:1000c8004800dd0001007000220020001100090036
:1000d8000200d800f407200000024200f00f2000c0
:1000e800800f52000200340000027800030037003d
:1000f8000400e00001003d000002eb00d340900046
:100108008180fb00634090004800dd000100700022
:1001180022002000110009000200d800f007b000fa
:10012800f10f2000810f5000020034000100780018
:10013800030037000000e00001003d000000eb0074
:100148008002fd00f7eab7008002fd000002fd0012
:10015800f8eab7000002fd00f9eab700edcf530056
:1001680009013a0086027800f64090008180fb0081
:10017800064890004800dd000100700022002000c1
:10018800110009000200d800f40720000002420014
:10019800f00f2000800f52000200340000027800a7
:1001a800030037000400e00001003d000002eb00fe
:1001b800954890008180fb00254890004800dd00ac
:1001c8000100700022002000110009000200d80080
:1001d800f307200080814100f00f2000808f51003c
:1001e8000200340080017800030037000300e000bb
:1001f80001003d008001eb00b54890008180fb00c4
:10020800454890004800dd000100700022002000f1
:10021800110009000200d800f007b000f10f20001b
:10022800810f5000020034000100780003003700fd
:100238000000e00001003d000000eb000002fd00ae
:10024800faeab7000002fd008001fd00feeab700ef
:100258008001fd003b003700964090008180fb0044
:10026800264090004800dd000100700022002000b8
:10027800110009000200d800f50720008082420022
:10028800f00f2000808f52000200340080027800b6
:10029800030037000500e00001003d008002eb008c
:1002a800b34090008180fb00434090004800dd008f
:1002b8000100700022002000110009000200d8008f
:1002c800f407200000024200f00f2000800f5200c7
:1002d8000200340000027800030037000400e00048
:1002e80001003d000002eb00d34090008180fb003c
:1002f800634090004800dd000100700022002000eb
:10030800110009000200d800f007b000f10f20002a
:10031800810f50000200340001007800030037000c
:100328000000e00001003d000000eb008002fd003d
:10033800faeab7008002fd000002fd00feeab700fd
:100348000002fd00ffeab70000000600e2cf5000ff
:100358008d003600164090000068a30008003200a7
:10036800fbcabf00ef4060000104a00002cfb30049
:100378000240600001407000fbeab700010037004e
:10038800fb0aa900264090000018a30008003200cc
:10039800fbcabf00ef4060000114a00002cfb30009
:1003a8000240600001407000fbeab700010037001e
:1003b800fb2aa900164090000004e00008003d0058
:1003c800fbcabf00ef4060000124a00002cfb300c9
:1003d8000240600001407000fbeab70001003700ee
:1003e800fb4aa900264090000008a300080032003c
:1003f800fbcabf00ef4060000134a00002cfb30089
:100408000240600001407000fbeab70001003700bd
:10041800fb6aa900164090004200de0061006000ff
:100428004700dd00b1af2000914078000174a100c1
:1004380080c0700001007800fbeab7001640900009
:100448004400de00610060004600dd00f2cbb3002e
:1004580082c0600080c0700001007800fbeab7002d
:10046800164090004500de00610060004500dd0098
:10047800f4cdb30084c0600080c070000100780033
:10048800fbeab700164090004300de006100600000
:100498004400dd00f3ceb30083c0600080c070006c
:1004a80001007800fbeab700164090006140600048
:1004b800e5cfb300c1af20009140780085c060004f
:1004c80080c0700001007800fceab7001640900078
:1004d8000000d10061006000004040000114a1004c
:1004e80080c0700001007800fceab7002640900048
:1004f8004400de00610060004600dd0082c060004c
:1005080080c0700001007800fceab7002640900027
:100518004500de00610060004700dd000174a100b5
:1005280080c0700001007800fceab7002640900007
:100538004200de00610060004500dd0084c060000c
:1005480080c0700001007800fceab70026409000e7
:100558004300de00610060004400dd0083c06000ed
:1005680080c0700001007800fceab700a640900047
:10057800c608de00e1806000fdcabf0005406000db
:1005880001407000fdeab70000000600f068900026
:10059800314098000072900044409800907090009c
:1005a800014898008000eb0063af2000d2032000d0
:1005b800e0f178008100e800828f5000fcff3a00eb
:1005c800000006004f0bb000889fbe008a9fbe0047
:1005d8008c9fbe008e1f78000006780000f42f0064
:1005e8000f00400041b32000750009003158780021
:1005f8006007b1009f819700f3b79f000f809700b5
:10060800e0b79f00df8097004809de006f80970001
:100618004800dd0002017000d2b79f004f809700ac
:100628004800de00c808dd0000807000c0b79f00e9
:10063800bf809700b1b79f002f819700a2b79f0096
:10064800ff39970093b79f006f38970080b79f00d6
:100658008f489700e1df9f004f919700e2af9f001e
:10066800bf919700d3af9f008f9897004809de008d
:100678009f9997004818dd0002017000c2af9f00e3
:100688007f9097004800de00c808dd0000807000f9
:10069800b0af9f006f909700a0af9f00df909700ca
:1006a80091af9f002f91970082af9f001f909700f6
:1006b800f0a79f00ef689700c1cf9f00c819de0020
:1006c8002f9897004800dd0003077000af88970057
:1006d8004809de00bf8997004818dd000201700054
:1006e800d2a79f001f8a97004820de00c808dd00b7
:1006f80000807000c0a79f007f899700b2a79f0065
:100708006f889700a0a79f00cf8897004809de0050
:100718005f8897004800dd0002017000c29f9f00bb
:10072800c819de00c808dd0083817000b39f9f00f0
:100738008f8897004808de004822dd00000072001c
:1007480090a79f007f8097004800de00c808dd0062
:100758000080700080a79f00bf589700e17f9f002e
:100768000f919700e29f9f00dc4090008180fb0082
:100778004708de00c02f9f004608de0061006000c9
:10078800d02f9f004508de0061006000e02f9f0029
:10079800c408de00e1806000f12f9f001906070001
:1007a800e30f50000b003a005c4090006f006000bf
:1007b800e1006000c1279f00e2006000d1279f0090
:1007c800e4006000e1279f0068006000f0279f00b8
:1007d8001d0037005c409000ef406000e7cf5000fc
:1007e800050032000104e000030032000000eb00c5
:1007f800e1cf500001003a0010002000c0279f0000
:100808000001eb000140e900e24f500001003e000a
:1008180012002000d2279f000001eb0063c05000a7
:10082800e24f500001003e0012002000e2279f0026
:100838000001eb0065c05000e24f500001003e008f
:1008480012002000f2279f006c4190008280fb007c
:100858004608de006100600090279f004708de0020
:10086800a0279f004508de0061006000b0279f00b8
:100878004408de006100600080279f004208de0017
:1008880061006000802f9f004308de006100600067
:10089800902f9f0061016100a22f9f008100d1006d
:1008a800e1806000b12f9f007c409000e100600073
:1008b80081379f000000d1006100600090379f00e1
:1008c8001c4090000080fb00a0379f002c40900047
:1008d8000080fb00b0379f003c4090000080fb0088
:1008e800c0379f004c4090000080fb00d0379f002d
:1008f8000c4890000080fb00e0379f001c489000e7
:100908000080fb00f0379f006c5890006f4060003b
:10091800a07f9f001c5190000281fb002c5090008a
:100928004800dd0002007000a80020001100090046
:100938000800d800cf80de0092558000a3558000c3
:100948000000410081804900423d20000300200052
:100958001cbf07003c5290000482fb004c519000e1
:100968004811dd00040171007e11b900000041004a
:1009780081804900823e200003002000f2be07006b
:100988000005be0090558800a15588005c4990007c
:100998000281fb006c4890004800dd0002007000f6
:1009a800110009000800d800cf80de0072558000d1
:1009b800835580000000410081804900423d2000ad
:1009c80003002000ffbe07007c5290000482fb0059
:1009d8000c5990004811dd00040171007e11b90026
:1009e8000200500083805800823e2000030020004f
:1009f800d5be07000004be007055880081558800e8
:100a080042062000030020000a00be00cebe0700f8
:100a1800c03f9f0042062000030020000800be00df
:100a2800c9be0700d03f9f003c61900001c8b300d9
:100a380081416100090032007c6090000140600043
:100a480006003200e0cfb300c0cf9f000007eb00e4
:100a580080c0eb00e17f9f00ee9f9f000200fb003b
:100a68000080ea00cf05de00ef7897008184fb0064
:100a78003c6490000874a1000882fb00848f540035
:100a880001003a00eb9f9f004fc897000085fb00cc
:100a9800840f550001003a000b0778007c60900035
:100aa800804078000174a10081f79f008186fb00d7
:100ab8008d8f540004003a000000fb000080ea001b
:100ac8004f00de00e09f9f008d0f550005003a00a3
:100ad8000007eb007c6090000004e0000100350096
:100ae8001e0020000304e00087003a006fd9970039
:100af8000280fb00800f520015003200cc6090008d
:100b08008180fb005c6190000281fb006f00610046
:100b18004800dd0081007000a1b79f0000c42f00cd
:100b28000080400080b79f004411de006c60900098
:100b38000080fb004400dd0002017000b2b79f0096
:100b4800a0e22f000000410090b79f00e8df9f005f
:100b5800cc6090008180fb005c6190000281fb000a
:100b68006f0061004800dd00810370008fb09700be
:100b78000180530003c42f0003004000c0b79f004a
:100b88004411de006c6090000080fb004400dd0032
:100b9800020370001fb1970002005300a1e22f006a
:100ba80001004000d0b79f0087027800838143008e
:100bb80083b79f00860178008100430091b79f00aa
:100bc8002fb0970000805300e0b79f00bfb0970098
:100bd80081005300f1b79f00890f52001e003200b8
:100be8008a0f520030003200f03b2000808f530003
:100bf8000c003c0000ec2f000080430080a79f0001
:100c0800e87f9f000880fb00800f52000e00320032
:100c18001fb1970092a79f00b79f9f00c69f9f0094
:100c280021003700009c2f0000804300f0a79f00a0
:100c3800c8cf9f00a6af9f0097af9f009fb09700b7
:100c480081af9f0018003700b79f9f00c69f9f0085
:100c58009fb0970091a79f000fa1970002805300b3
:100c680002ec2f0002004000a0a79f001fa09700e1
:100c780080005300a0e22f0080804000b1a79f00b1
:100c88000281420082a79f00bf989700818052008e
:100c9800c1a79f004f99970002815100d2a79f00da
:100ca8001fb0970090a79f00cfc897000180fb0056
:100cb800800f520014003a007fa197000280530071
:100cc800029c2f0002004000b0af9f000fa89700c1
:100cd80080005300a0e22f0080804000c1af9f0039
:100ce80002814200f2a79f009fa8970081825200cc
:100cf800d5af9f002fa9970082815100e3af9f00d5
:100d08009fb1970083af9f007c6090000004e000d3
:100d18007c003500ef7897000180fb00808f56003b
:100d2800340032004fc997000280fb00808f5600c4
:100d3800500032008c6890008180fb001c68900095
:100d48008081fb006f8061004800dd0001017000b8
:100d5800f03b2000800f510013003c0000ec2f00f6
:100d68000000410080a79f00c418de002c68900096
:100d78000080fb004400dd0081007000c19f9f00df
:100d8800a0e22f000080400090a79f008ff19700fd
:100d9800e37f9f000380fb00808f56001400320021
:100da800b29f9f0057003700009c2f0000004100b1
:100db800f0a79f009c6890008180fb00c408de00bb
:100dc8002c6890000080fb004400dd00810070006a
:100dd800a1af9f00a0e22f000080400080af9f00dd
:100de8000ff09700c0cf9f0092af9f0021003700ff
:100df800b29f9f000c6890000080fb001c69900067
:100e08000281fb00ef006100c808dd0080807000ef
:100e18008fa197000380500004ec2f0004004000cd
:100e2800a0a79f004411de002c6890000080fb0002
:100e38004400dd00020070009fa1970003015000ec
:100e4800a3e22f0003014100b2a79f0004824000e3
:100e580084a79f008301400093a79f003f999700b4
:100e680082805000c1a79f00cf99970003005000cf
:100e7800d0a79f00cfc897000180fb00808f560045
:100e880020003a000c6890000080fb001c6990006c
:100e98000281fb00ef006100c808dd00808070005f
:100ea800ffa1970003805000049c2f00040040001d
:100eb800b0af9f004411de002c6890000080fb005a
:100ec8004400dd00020070008fa997000301500064
:100ed800a3e22f0003014100c2af9f00048240003b
:100ee800f4a79f008301400083af9f001fa99700cc
:100ef80082805000d1af9f00afa997000300500037
:100f0800e0af9f000b00e00004003a00fbb79f0031
:100f1800ebb79f00dbb79f00cbb79f006f98970098
:100f28000000e00004003a00d0a79f00c0a79f007f
:100f3800b0a79f00a0a79f000e00e00004003a00a1
:100f4800eeaf9f00deaf9f00ceaf9f00beaf9f0009
:100f5800ffb0970091879f006fb1970082879f002d
:100f6800f30f2000dfb097004808dd005f8197008d
:100f780003016100000171004808de000300600001
:100f880006f02f006f8297000602620000027200ce
:100f98004fb0970083006000c808dd004f809700bd
:100fa8000300600001007000c0879f00cfb0970069
:100fb8004808de00030060000601610000017100be
:100fc800d2879f003fb19700b2879f002fb097004c
:100fd800a0879f009fb09700f13f9f000fb1970037
:100fe800e23f9f006fd89700804f9f000380650005
:100ff8004800dd000302620000027200e4879f00df
:10100800efa89700c1979f005fa99700b2979f002c
:10101800cfa89700038060004800dd000f99970073
:1010280003016100000171004808de000300600050
:101038001f9a970006026200000272003fa89700fc
:1010480083006000c808dd007f90970003006000ff
:1010580001007000f0979f00bfa897004808de00c5
:10106800030060000601610000017100829f9f007b
:101078002fa99700e2979f001fa89700d0979f007d
:101088008fa89700a1979f007fa1970092979f0034
:101098004fc89700e06f9f00030067004800dd001d
:1010a8000302620000027200949f9f00c870de0075
:1010b800838060002f989700060060000100700090
:1010c800a09f9f00dfa09700038060004800dd001c
:1010d800af88970083806000808070005fa19700d0
:1010e8004810de00030060003f8a97000602620095
:1010f800000272004fa19700030061004800dd0064
:101108009f8a970083826200808272004810de0006
:10111800030060008680600080807000a18f9f00bf
:101128003fa09700f08f9f00afa09700e18f9f002e
:101138004f999700030061004800dd004f89970030
:1011480003016100000171004f989700c800de009c
:10115800838060005f8897000600600001007000cf
:10116800d08f9f00bf989700038060004800dd0083
:101178000302620000027200b48f9f004808de007c
:10118800030060000601610000017100c28f9f002a
:101198001fa19700030061004800dd008f889700b9
:1011a80083806000808070004810de0003006000cb
:1011b8008682620080827200958f9f000fa197003f
:1011c800030061004800dd00f0879f004810de0042
:1011d800030060008680600080807000818f9f001f
:1011e800ef799700b35f9f006f98970080979f00f3
:1011f800af789700d1779f0002f42f000f014100cc
:1012080043b3200075000900b25978006207b100a5
:101218004f0778004f06be004f05be004f04be00c2
:101228004f0bb10000000600ac2aef0000000600da
:10123800881f78000004eb008801780065ab200067
:1012480044b32000f60f20000380410085004000d1
:101258001181fb0091409000c808dd008280700079
:10126800040040001081fb00104090004800dd00a1
:1012780002007000808f500001003200180020002a
:1012880083804100048040001081fb0010409000e2
:101298004800dd0002007000858040000601600003
:1012a80091437800e0c86300914871004800de006f
:1012b80011419000904098008301e800f28f51009e
:1012c800e1ff3a008002eb0047b32000a6ad200002
:1012d8000581420040022000020040000702400051
:1012e8001480fb0094409000c808dd0080807000e6
:1012f800860141001381fb00134090004800dd0087
:1013080002007000808f5000070034001480fb003a
:1013180094409000c808dd00808070001381fb00b5
:10132800134090000a003700058042008600400004
:101338001181fb0091409000c808dd008280700098
:101348004002b000070040001081fb0010409000f0
:101358004800dd0002007000808050006a80520062
:10136800e10f500004003e00800c2000808f5000e8
:1013780003003c0003003700e58f500001003400f3
:101388001800200085804200400220000100400033
:10139800070040001081fb00104090004800dd006d
:1013a800020070008680400011417800e04861002a
:1013b800914870004800de0011419000904098006c
:1013c8008502e800ec8f5200c1ff3a00d1b7200037
:1013d800914078008180fb007ecbbf004800dd0093
:1013e8000100700002003a007fcbbf0080cbbf0035
:1013f8000800e00005003a0060558000e10f400059
:1014080003003200ac2aec000100370086ff070019
:10141800610014004f04780000000600889fbe0099
:101428008a1f78000002eb0045b32000aaba20000a
:10143800f90f20000044eb0027bf2000e6bc200085
:1014480004014200050041009080fb00104090001c
:101458004800dd00010070000e0032008a004100e3
:101468001181fb00114090004800dd00020070006f
:101478000000e8000901600091417800e0c86100bf
:10148800914871004800de0011419000904098009a
:1014980006003700040042000a004000904078002f
:1014a80060c8600090409000184098000401420015
:1014b800050041009080fb00104090004800dd00ce
:1014c800010070000d003200070041009080fb0011
:1014d800104090004800dd008101700007003a00cc
:1014e800060041009040780060c860001004a00029
:1014f8009040900013409800060037000400420016
:10150800060040009041780060c86100904090005b
:101518001840980084004200058040001081fb00bc
:10152800104090004800dd000200700087804000f5
:101538000901600091417800e0c86100914871009c
:101548004800de0011419000904098000402e80035
:10155800f20f5200baff3a004f0578004f04be0060
:101568000000060040b3200000000600a0ba2000da
:1015780000000600e0bc20000000060080b5200046
:101588000000060000b720000000060060af200041
:1015980000000600606f800000000600706f800089
:1015a8000000060040d920000000060081427800b3
:1015b80083407800e9cf520001003600a5c0b3008f
:1015c800646f800042529800515298000100200038
:1015d800e90f5000e08f580057003e0000600100fe
:1015e80010003700150037001b00370021003700b6
:1015f800270037002e00370003003700330037007c
:101608003c003700450037000040eb0010529800be
:10161800205298000540780042c1b3000440bc0045
:10162800430037000540780042c1b3000440bc00c5
:10163800125298000040eb00410037000540780046
:10164800f2c0b3000440bc001252980052c0b3006c
:101658000440bc000400370005407800a2c0b30075
:101668000440bc0012529800225298000040eb003f
:10167800340037000540780052c0b3000440bc0075
:1016880012529800f2c0b3000440bc00f6ff3700c5
:101698008040eb00115298000540780042c1b30029
:1016a8000440bc0022529800315298000000060005
:1016b8000040eb001052980005407800f2c0b300db
:1016c8000440bc0022529800110037000540780001
:1016d80052c0b3000440bc00125298000040eb0016
:1016e8002052980005407800f2c0b3000440bc00c6
:1016f8000f00370005407800f2c0b3000440bc007a
:10170800125298000040eb002052980005407800e3
:1017180052c0b3000440bc00050037000540780003
:1017280052c0b3000440bc001252980022529800e4
:1017380032529800000006000040eb00105298005a
:10174800205298003052980000000600656f800013
:1017580090529800a1529800b2529800c352980033
:10176800d45298000000060080407800e94f5000ed
:1017780001003e008040eb00606f800071489800d7
:101788000000060080407800e94f500001003e004c
:101798008040eb00606f8000015098000000060058
:1017a8000001780041b52000914078008180fb005d
:1017b80055cbbf004800dd0001007000e10f50006c
:1017c80002003200e10f510002003a00a0002000a0
:1017d80090578800f20ae20019003200a9cbbf0036
:1017e800e34f5000060036003edb07008041eb0067
:1017f8000341780080407800400020000e00370048
:10180800a9cbbf00e14f50000600360035db0700ca
:101818008041eb00034178008040780020002000e0
:10182800050037002fdb07008041eb0003417800fb
:10183800804078000000eb005cff0700f22aed0012
:10184800000006000000e00003003200a0578800f6
:1018580000c0eb00c4ff3700f40ae20006003200c3
:1018680000c0eb00c0ff0700f40aed00a057880095
:1018780001003a00bcff0700000006006055800028
:041888000000060056
:020000040000fa
:1009c800881f780028042000184478000884fb0059
:1009d8004544de0091028000ff3ffc0000ceb300da
:1009e8004260b700910288004e0307009102800020
:1009f800ff3ffc004544dd0042c0bf007f4060006f
:100a08000840700042e0b700910288004f04780067
:100a180000000600889fbe000244780022032000e0
:100a2800124178008284fb0006c0200007002000e5
:100a38000080fb008180fb004b02dd0004024300c4
:100a4800e0824b004a09dd0002014200e0814a00d1
:100a58004019de000001fd0032e0b7000001fd0092
:100a680000004000010040004a00dd000600400090
:100a780028030700f34f540008003200f44f5400d5
:100a8800090032008040eb00f24f540008003a00a1
:100a980064006000c200de000500370068006000e6
:100aa800c300de000200370070006000c400de00f2
:100ab8000900780032e0b7000180fb004f04be0057
:100ac80000000600881f78002803200018447800da
:100ad80006c02000070020000080fb008180fb008a
:100ae8004b02dd0004024300e0824b004a09dd00ae
:100af80002014200e0814a004019de000001fd00c9
:100b080032e0b7000001fd0022042400023b880007
:100b180000004000010040004a00dd0006004000df
:100b28008000780010030700a5ff07000800780080
:100b380032e0b7004f04780000000600889fbe002e
:100b48008a1f78008044780032c0bf000085fb000f
:100b58000004eb00030037000804e800e20f54002b
:100b68000600320032c1b30088407800094078009e
:100b7800a8ff0700e10f5000f7ff320006c0200071
:100b8800070020000982fb004b21dd000201430021
:100b9800e0814b004a40dd0000004100e080490050
:100ba8004008de0032e0b7000402420008024200ba
:100bb8004a22dd00060442008004eb008984e80034
:100bc8000884e80008007800d20207008040780016
:100bd80000402000808f540002003a008004eb009f
:100be80002003700e1cf4000f4ff3a000a00780025
:100bf80032e0b700090078004f0578004f04be00c6
:100c080000000600889fbe008a9fbe00800478000e
:100c1800e00f2000808f540002003600ecaea800e0
:100c280016003700f20f2000110009008284d80056
:100c3800000178008245780032c0bf000085fb00c3
:100c48000004eb00030037000804e800e20f54003a
:100c58000700320032c1b300884078000b407800aa
:100c68006cff0700e10f5000f7ff32000500370066
:100c78000a00780032e0b700eccea8000080eb0054
:100c88002800370004c02000050020004b59dd0073
:100c9800ca41dd0002004200e0804a000300400033
:100ca800e08048004008de0032e0b700040141005f
:100cb80003014100e13f200082804000f20f200044
:100cc80081057800110009008284d8008105fd00a3
:100cd8000920200001047800010078008d02070037
:100ce8008880e9008904e900030032008b0f500076
:100cf80007003200f7ff3700ec0ea8000a00780062
:100d080032e0b700c0032b004b460700dbff37007b
:100d180008007800810207000005fd0032e0b700f6
:100d28000005fd004f05be004f04be000000060090
:100d3800f4874700889fbe008a9fbe008c9fbe0034
:100d48008e1f780080f79f0032c0bf000080fb0034
:100d580090b79f008006eb00030037008d06e8007f
:100d6800e28f56000700320032c1b3008d40780090
:100d78000ff0970027ff0700e10f5000f7ff320040
:100d8800050037002fe0970032e0b700ec6ea800ae
:100d980030002000de0037000d06e800e20f5600a4
:100da80008003a000006eb00060037000c06e800d1
:100db800e20f560001003a000006eb008d0f5600c6
:100dc800c200320042c1b3008c4078000ff0970097
:100dd80010ff07000000e000f4ff320004c020000c
:100de800050020008ff097000181fb004b10dd000b
:100df8006103b800e6b79f00f7b79f004a60dd00bf
:100e08006103b800c6b79f00d7b79f006fb39700bc
:100e1800ffb397000400430085804b004fb3970051
:100e2800dfb397000000430081804b004008de00dc
:100e380032e0b70002014100b2b79f000c00410048
:100e48004a07dd00040447000ff097003bff070046
:100e58000000e00001003200ec4ea800eccebf001c
:100e680080e79f00ec0ea90010002400003b8800da
:100e7800880078000080eb003b02070088007800bb
:100e8800f00f2000340207000884e8008ff0970074
:100e98000180fb00f20f20000280b900a0b79f007c
:100ea800190020008045eb000b85fb002fb297004e
:100eb8000a00420053ff0700ec0eab0002003200ac
:100ec800ec0ea9000700370088007800260207000a
:100ed800880078000a0078001f0207000884e800ec
:100ee8008904e8008b45e800e1cf45000e003a0090
:100ef80008003700880078000080eb001a0207001d
:100f080088007800f00f2000130207000884e8002a
:100f18008904e800f0032000808f5400f5ff3400b6
:100f280080c5eb0003003700f0032000808f5400d9
:100f3800ddff3400a2fe07008004eb00e1cf45008e
:100f4800d9ff3a000fe09700eceeb70002c020008e
:100f5800030020006fb29700ffb297000200420022
:100f680083804a004fb39700dfb397000000430027
:100f780081804b004008de0032e0b70002054700e0
:100f88000a84e80008007800e2010700804478003d
:100f98008885e800630045000c0037000980fb00e5
:100fa800afb397000080430016ff0700880f50007a
:100fb8004b003a000b04e8000b007800d50107004d
:100fc800804478008b85e80008007800d30107008a
:100fd80000047800e1cf4400f0ff3a0002c020008e
:100fe80003002000bfb097000d8040004a00dd00dc
:100ff80002044000020547006fb29700ffb2970055
:101008000201420083814a004a68dd000000410075
:10101800e08049004008de0032e0b70008007800b0
:10102800be0107008004780008007800b9010700b5
:10103800004178000c00e00001003a008904e80053
:10104800e38f440002003600ec2ea8000244a10001
:1010580000c02000010020006fb39700ffb3970085
:101068000000430081804b004fb29700dfb2970029
:101078000000420081804a004008de0032e0b700ec
:101088000284fb008a00780008007800b20107009b
:101098008a00780009007800b301070030002400b6
:1010a800003b880046fe07000a0078009901070007
:1010b800800f54000a003a000a00780097010700e0
:1010c800808f54000b003200050037002fe0970096
:1010d80032e0b700ec2ea800100020000c0037000a
:1010e8002fe0970032e0b700eceea8007000200077
:1010f800070037008d4078000ff0970071fe070059
:101108002fe0970032e0b700ec0ed50061006000d8
:101118004f0778004f06be004f05be004f04be00c3
:101128004f01b10000000600889fbe008a1f7800aa
:1011380032c0bf000085fb0000c020000100200075
:101148004008de0032e0b7000004eb00030037007f
:101158000804e800e20f54000700320042c1b3005f
:10116800884078000040eb002afe07000000e000fd
:10117800f7ff3200050037000a00780032e0b700b8
:10118800ec2ea800100020004e0037000044eb00b1
:101198008004eb0032c1b300894078000040eb00c6
:1011a8001cfe07000000e00001003a000844e800c7
:1011b8008904e800e28f5400f6ff3a000804e000d2
:1011c80012003a0088407800084078003dfe070089
:1011d80008c02000090020004048de00010020006f
:1011e80032e0b70030002400003b88008800780017
:1011f8000000eb005c01070088007800300f200039
:1012080055010700eefd070026003700e14f5400a6
:1012180024003200e24f540026003a0032c1b300e5
:1012280011c0b3000040eb00fafd07000000e00029
:1012380005003a0032c1b30080407800f5fd070090
:101248000000e0000f0032000004eb00010037004e
:101258000804e8008844780032c1b3008840780068
:101268000040eb00ebfd0700e10f500002003a00e0
:10127800e20f5400f6ff3a008940e800e2cf500040
:1012880001003a008040eb000040eb000dfe070033
:101298000040eb0029fe07000000e00001003a00d2
:1012a800a3fe07000a00780032e0b7000000eb0058
:1012b800040037000a00780032e0b700eccea8003e
:1012c800600020004f0578004f04be0000000600b3
:1012d800e4874700889fbe008a9fbe008c9fbe009f
:1012e8008e1f78008006780081057800e00f2000c6
:1012f800808f500003003600ecaea800500020009c
:1013080077003700f20f2000110009008280d80012
:101318000004780032c0bf000085fb0030002400c4
:10132800003b88008004eb00030037008904e800d4
:10133800e28f5400080032000847780032c1b30039
:101348008940780008407800b2fd0700e10f50009e
:10135800f6ff3200050037000a00780032e0b700d7
:10136800eccea800600020005d00370004c020001b
:10137800050020004b41dd0002014200e0814a00e7
:101388004a48dd0000004100e08049004008de00d6
:1013980032e0b70008004400090040004a00dd00c0
:1013a80084044000c8ee2000184478000b00780040
:1013b80014fe07008d0f50000a003a006077800085
:1013c8006100600007003a000005fd0032e0b70048
:1013d8000005fd000004fd00eceeb7000004fd0070
:1013e8003f00370008007800eceeb7000e407800a8
:1013f800d2fd0700000678000000e00005003a0072
:101408000a00780032e0b700ec8ea8004000200007
:101418003300370080844400890078000d0078008c
:10142800d1000700f80f2000110009008885d800b6
:1014380081057800890078000b007800c600070055
:101448005ffd0700000000000000000009007800b0
:10145800b200070080f79f008ff097000180fb0023
:1014680008846600880f500010003a0009007800d0
:10147800a800070080f79f008ff097000180fb000d
:101488008b0f500009003a000900e800a30007008c
:101498004880de0080f79f000ff097008080fb00f7
:1014a8004868de00808f5000050032000a0078008e
:1014b80032e0b700eceea80070002000080037000a
:1014c800e03f2000800f560002003a000e407800ee
:1014d80017fe07000a00780032e0b7000000eb00b2
:1014e8004f0778004f06be004f05be004f04be00f0
:0814f8004f00b10000000600e6
:020000040000fa
:020000040001f9
:10188c003073880000000600e7eeb7000000060089
:10189c00e6eeb70000000600e5eeb700000006001b
:1018ac00e4eeb70000000600889fbe0000447800fc
:1018bc008144780010002000f1ff070010c8b3002d
:1018cc00f1ff070010c0b300f1ff070020c8b30000
:1018dc00f1ff070020c0b300f1ff07006000b80063
:1018ec00c0738800d1738800e0738800f17388009e
:1018fc00816eef000800780076eeb700027780006a
:10190c00824890008180fb009173880012489000ff
:10191c004800dd008080700091738800a248900020
:10192c008180fb00a1738800324890004800dd00e4
:10193c0080807000a17388000900780080eeb700e9
:10194c00810ea800640020000500200022e7200082
:10195c00011920000840780050f707001000200003
:10196c004f04be0000000600889fbe0000447800b3
:10197c008144780020002000c1ff070040c8b3005c
:10198c00c1ff070030c0b300c1ff07006000b80002
:10199c00c0738800d1738800e0738800f1738800ed
:1019ac00816eef000800780076eeb70002778000b9
:1019bc00824890008180fb0091738800124890004f
:1019cc004800dd008080700091738800a248900070
:1019dc008180fb00a1738800324890004800dd0034
:1019ec0080807000a17388000900780080eeb70039
:1019fc00810ea800640020000500200022e72000d2
:101a0c00011920000840780024f70700100020007e
:101a1c004f04be0000000600889fbe000044780002
:101a2c0081447800a0fe2a00020307003000200049
:101a3c0093ff070010c8b30093ff070020c0b3004a
:101a4c0093ff0700782eef007a2eef00816eef00e7
:101a5c000800780076eeb70002778000824890008c
:101a6c008180fb0091738800124890004800dd00d3
:101a7c008080700091738800a24890008180fb00e8
:101a8c00a1738800324890004800dd00808070000f
:101a9c00a17388000900780080eeb700810ea800c1
:101aac00640020000500200022e72000011920001e
:101abc0008407800f9f60700100020004f04be0023
:101acc0000000600889fbe00004478008144780026
:101adc00a0ff2a00d70207004000200068ff070083
:101aec0040c8b30068ff070030c0b30068ff0700b0
:101afc006000b800c0738800d1738800e073880060
:101b0c00f1738800816eef000800780076eeb70064
:101b1c0002778000824890008180fb0091738800de
:101b2c00124890004800dd0080807000917388009e
:101b3c00a24890008180fb00a1738800324890007d
:101b4c004800dd0080807000a173880009007800d7
:101b5c0080eeb700810ea800640020000500200074
:101b6c0022e720000119200008407800cbf607007e
:101b7c00100020004f04be00000006000400fa0014
:101b8c008041780076cebf00001ce1004a003a008c
:101b9c0010072000808f5000040032000000e80085
:101bac00808f500044003a000a00370014002000d7
:101bbc000500200062e72000111920000340780086
:101bcc00b6f607000040eb0081eeb70076eeb700ea
:101bdc00160037000200e00037003200ea0f520016
:101bec00e08f5a0034003a001202be00e4bf9f009e
:101bfc00f5bf9f00e2409000e7cebf000074a0004c
:101c0c0080cf50000b003a00816ea900c47388008d
:101c1c00d573880076cebf0044002000050020005c
:101c2c0064815700311920009cf607001000200039
:101c3c0022003700e5cebf000074a00080cf50001a
:101c4c0009003a00818ea900e4738800f5738800be
:101c5c0076cebf00440020000500200064815700b0
:101c6c0041192000f0ff3700e6cebf00000ce10068
:101c7c0007003a00812ea90076cebf004400200058
:101c8c00050020006481570021192000e6ff370071
:101c9c00e4cebf00000ce10007003a00814ea90021
:101cac0076cebf0044002000050020006481570060
:101cbc0051192000dcff37000000eb000080fa0017
:101ccc000000060000017800810eab000f0032000e
:101cdc0063e72000934178000304e0000b0032001e
:101cec000000e0000900320090738000920f100099
:101cfc0006003a0092009000a0738000808f500084
:101d0c0002003a0043419800100005000000050055
:101d1c000103780061e72000914078000104e100a4
:101d2c001c003a00017480000188a30019003200e5
:101d3c0001b8a30009003200680eec004073880063
:101d4c0021002000e50f500013003600816ea90021
:101d5c00682eef00210020000f003700816ea800d4
:101d6c00782eef007a2eef0071ee20009140780073
:101d7c000174a0000202be0006017800eee107002b
:101d8c000004e00001003200816ea9008080fb009d
:101d9c00010037001100200001007800000006004f
:101dac000103780061e72000914078000104e10014
:101dbc0019003a00017480000188a300160032005b
:101dcc000198a300090032006a0eec0050738800e1
:101ddc0021002000e50f500010003600812ea900d4
:101dec006a2eef00210020000c003700812ea80085
:101dfc0061ee2000914078000202be0006017800de
:101e0c0018e407000004e00001003200812ea90054
:101e1c008080fb00010037001100200001007800d9
:101e2c00000006008201780062e720001241780071
:101e3c000204e1001e003a00027480000288a30034
:101e4c001b0032000298a300090032006c0eec005b
:101e5c006073880021002000e50f5000150036004b
:101e6c00812ea9006c2eef002100200011003700fc
:101e7c008f87e8000041eb00e2ff9f00824378006f
:101e8c0001037800830278000002eb0084017800e3
:101e9c0011c2b3000ee107008f87e9000004e000d7
:101eac0001003200812ea9008080fb000100370068
:101ebc0011002000010078000000060001037800ea
:101ecc0061e72000914078000104e10019003a001c
:101edc00017480000188a3001600320001a8a30041
:101eec00090032006e0eec00707388002100200097
:101efc00e50f500010003600814ea9006e2eef0049
:101f0c00210020000c003700814ea80041ee20007b
:101f1c00914078000202be0006017800d1e3070070
:101f2c000004e00001003200814ea9008080fb001b
:101f3c0001003700110020000100780000000600ad
:101f4c000103780061e72000914078000104e10072
:101f5c001c003a00017480000188a30019003200b3
:101f6c0001c8a30009003200700eec0080738800d9
:101f7c0021002000e50f500013003600812ea9002f
:101f8c00702eef00210020000f003700818ea8007a
:101f9c007c2eef007e2eef0051ee20009140780059
:101fac000174a0000202be000601780062e1070085
:101fbc000004e00001003200818ea9008080fb004b
:101fcc00010037001100200001007800000006001d
:101fdc00e7cebf000080fb0000000600e6cebf008d
:101fec000080fb0000000600e5cebf000080fb0077
:101ffc0000000600e4cebf000080fb0000000600dd
:10200c003073800000000600a9c6bf0001ccb300ed
:10201c00014060000014a000a9e6b700a8c6bf00ec
:10202c00014060000024a000a8e6b700aac6bf00cb
:10203c0001406000c040b300aae6b700c3c6bf00b1
:10204c00014060007040b300c3e6b700d802a8009e
:10205c0081c6bf0001406000b040b30081e6b7000c
:10206c00aec0bf0081cfb300014060006040b30040
:10207c00aee0b7008220a9008680a90040c2bf0054
:10208c0031ceb300014060000024a00040e2b70054
:10209c000000eb00101288004322a90042e2a800c5
:1020ac0042a2a900201288004402a8000ad9070005
:1020bc00e10f50000a00320005003900e20f500019
:1020cc000b003200e30f500013003a000d003700f4
:1020dc0000f92a005701070042c2a9000700370087
:1020ec0010fa2a005301070042c2a9000800370069
:1020fc0020fb2a004f01070042c2a8004302a8009f
:10210c000700370030fc2a004a01070042c2a80031
:10211c004302a9000200370040fd2a0045010700d8
:10212c008540a900a9c0bf0081cfb3000140600069
:10213c006040b300a9e0b7009540a80041e2a800b8
:10214c00c10a2000010037004112880040c2bf00c4
:10215c000018a300fcff3200010037004012800081
:10216c0040c2bf000058a300fcff32000000060074
:10217c00889fbe000049900061416100e4cfb3002c
:10218c0081e020009140780084c0600082c0700023
:10219c008000fd0008eeb7008000fd002049900093
:1021ac006141610002414100d3cfb30083c06000a4
:1021bc0082c070008000fd0008eeb7008000fd00ba
:1021cc0040499000614161004211dd00b9cfb3007c
:1021dc0089c0600082c070008000fd0008eeb7006e
:1021ec008000fd0060499000614161004311dd00f9
:1021fc0078cfb30088c0600082c070008000fd0002
:10220c0008eeb7008000fd000059900061416100ac
:10221c004411dd00f7ceb30087c0600082c07000af
:10222c008000fd0008eeb7008000fd0020599000f2
:10223c00614161004511dd00f6cdb30086c0600040
:10224c0082c070008000fd0008eeb7008000fd0029
:10225c0040599000614161004611dd00f5cbb3009f
:10226c0085c0600082c070008000fd0008eeb700e1
:10227c008000fd00605990004711dd000174a10041
:10228c0082c070008000fd0008eeb7008000fd00e9
:10229c00405190006141610091e020009140780034
:1022ac0084c0600082c070008000fd0009eeb700a1
:1022bc008000fd00605190006141610002414100cd
:1022cc0083c0600082c070008000fd0009eeb70082
:1022dc008000fd0000519000614161004211dd0061
:1022ec0089c0600082c070008000fd0009eeb7005c
:1022fc008000fd0020519000614161004311dd0020
:10230c0088c0600082c070008000fd0009eeb7003c
:10231c008000fd0020419000614161004411dd000e
:10232c0087c0600082c070008000fd0009eeb7001d
:10233c008000fd0040419000614161004511dd00cd
:10234c0086c0600082c070008000fd0009eeb700fe
:10235c008000fd0010437800614163004611dd00f0
:10236c0085c0600082c070008000fd0009eeb700df
:10237c008000fd00604190004711dd000174a10058
:10238c0082c070008000fd0009eeb7008000fd00e7
:10239c002061900061416100a1e020009140780033
:1023ac0084c0600082c070008000fd000aeeb7009f
:1023bc008000fd0000609000614060000040400023
:1023cc0083c0600080c07000010078000aeeb70086
:1023dc004f04be0000000600900078000101d100ff
:1023ec000001fd00f0edb7000001fd00c908de00a2
:1023fc008000fd00f1edb7008000fd009000900022
:10240c000101d1000001fd00f2edb7000001fd005b
:10241c00c908de008000fd00f3edb7008000fd0070
:10242c00a00090000101d1000001fd00f4edb70007
:10243c000001fd00c908de008000fd00f5edb700cd
:10244c008000fd00b00090000101d1000001fd00f2
:10245c00f6edb7000001fd00c908de008000fd00ac
:10246c00f7edb7008000fd00c00090000101d10025
:10247c000001fd00f8edb7000001fd00c908de0009
:10248c008000fd00f9edb7008000fd00d000900049
:10249c000101d1000001fd00faedb7000001fd00c3
:1024ac00c908de008000fd00fbedb7008000fd00d8
:1024bc00e00090000101d1000001fd00fcedb7002f
:1024cc000001fd00c908de008000fd00fdedb70035
:1024dc008000fd00f00090000101d1000001fd0022
:1024ec00feedb7000001fd00c908de008000fd0014
:1024fc00ffedb7008000fd00800890000101d100c5
:10250c000001fd0000eeb7000001fd00c908de006f
:10251c008000fd0001eeb7008000fd0090089000e7
:10252c000101d1000001fd0002eeb7000001fd0029
:10253c00c908de008000fd0003eeb7008000fd003e
:10254c00a00890000101d1000001fd0004eeb700cd
:10255c000001fd00c908de008000fd0005eeb7009b
:10256c008000fd00300890008000d1008000fd004c
:10257c0006eeb7008000fd004900de0007eeb70054
:10258c0000000600c0e020000000060000df200074
:10259c00000006002000050087c0bf000068a300f3
:1025ac00fdff320032c2bf0080c0eb000008a30068
:1025bc0002003200b01180008040780087c0a90072
:1025cc000100fb000000060010022000c011880072
:1025dc000000eb00801188003062a8009011880088
:1025ec0031e2a8003342a80087c0a9000000060011
:1025fc0087c0bf000068a30004003a0032c2bf00cd
:10260c008000eb000008a300010032001100200044
:10261c0001007800000006000000fb00a0118800fb
:10262c000000000033c2bf000008a300fdff320011
:10263c0000000600881f78000004780002003700b4
:10264c0001407800f4ff07003840780080407800a3
:10265c000004e000faff3a004f0478000000060086
:10266c00889fbe008a9fbe008041780049c6b30097
:10267c000004e00008003a0000c3b300e6ff0700c6
:10268c001a0037000980fb00a2002000110009008d
:10269c000280d8008044780083cf5400f9ff3e00bc
:1026ac00834578000f0037000b84fb000985fb0085
:1026bc00110009000a84d8000004780001c3b3009b
:1026cc0001404400d4ff070009c4b90088c5550077
:1026dc00a2002000110009000285d8000005780036
:1026ec008a4478000904e000efff3a004f05be0071
:1026fc004f04be0000000600881f78000004e000b4
:10270c0004003d000044ea00d0c2b300c2ff070041
:10271c00010037000044780008407800d0ff070023
:10272c004f04780000000600889fbe008a9fbe0000
:10273c00800078000a7122000000e00009003a00d5
:10274c0000c3b300b4ff070018003700a20020003c
:10275c00811f7800110009000285d800000578005f
:10276c00cf007800810f5500f8ff3e0081057800fe
:10277c000c003700110009008a85d800000478008d
:10278c0001c3b30001404400a3ff07000ac4b90011
:10279c0088855500a2002000110009000285d80090
:1027ac00000578000a00e000f2ff3a004f05be0079
:1027bc004f04be0000000600881f78000000e000f7
:1027cc0004003d000004ea00d0c2b30092ff0700f1
:1027dc00010037000004780008007800d2ff0700e1
:1027ec004f04780000000600889fbe008a9fbe0040
:1027fc008c9fbe000004be000aa02c00abb92300c5
:10280c00e00f5000e08f580008003a0000c3b300fe
:10281c0081ff07001e003700a200200003002000eb
:10282c000a00be0056b707000005be00880f550011
:10283c00898f5d00f8ff3e000806be0011003700ce
:10284c000a01be000c00be004db707000004be001c
:10285c0001c3b300014044006fff07000a01be0032
:10286c000800be0056b707000006560081865e00c1
:10287c00a2002000030020000a00be0040b70700a1
:10288c000005be00e00f5500e08f5d00ecff3a0044
:10289c004f06be004f05be004f04be0000000600f0
:1028ac00889fbe00e00f5000e08f580005003d00ef
:1028bc0060041000e0841800d0c2b30056ff07007b
:1028cc00010037000004be000800be00c6ff070070
:1028dc004f04be0000000600889fbe0080047800f4
:1028ec004480de006f006000c8022b0060407c005a
:1028fc0049ff07006f80640060407c0046ff0700c2
:10290c004f04be0000000600889fbe0080047800c3
:10291c004c00de00c8022b0060407c003eff07002c
:10292c004848de006f00600060407c003aff070002
:10293c004448de006f00600060407c0036ff0700fa
:10294c006f80640060407c0033ff07004f04be00c2
:10295c0000000600889fbe008a1f78000004be009d
:10296c004c08de006f006000ca022b0060407d0046
:10297c0029ff07004848de00010020006f006000be
:10298c0060407d0024ff07004448de000100200069
:10299c006f00600060407d001fff07004048de00b4
:1029ac00010020006f00600060407d001aff0700ee
:1029bc004449dd004c40de0000007100cc48de00d4
:1029cc006f00600060407d0013ff07004849dd0088
:1029dc004840de0000007100c848de006f00600057
:1029ec0060407d000cff07004c49dd004440de00d8
:1029fc0000007100c448de006f00600060407d0084
:102a0c0005ff07006f04640068407d0002ff0700ab
:102a1c004f0578004f04be0000000600804078008f
:102a2c0060c6b30080cf500017003c0066405000d9
:102a3c0080cf50000200340090cab3000f00370062
:102a4c0060c4b30080cf50000f003c0066405000c3
:102a5c0080cf50000200340090ccb3000700370048
:102a6c0090c3b30080cf500007003c006a40500078
:102a7c0080cf50000400340000cdb30000c04000f3
:102a8c000000fb0000000600000005006f40600025
:102a9c00e94f5000030034007043b0000000fb000d
:102aac00000006000043b0000000fb000000060020
:102abc0032c2bf000018a300010032003222a9006c
:102acc0000000600881f780001003700f8ff07009f
:102adc00b1fe0700e24f5000fcff3a00aefe0700cb
:102aec008040780000cdb30000c44000e0002b0013
:102afc00d0fe070008407800d9fe0700a0012b008b
:102b0c00ccfe07007300a9000080eb004016880083
:102b1c0080168800c01688000017880040178800af
:102b2c00801788004016880080168800c016880020
:102b3c0000178800401788000000eb008017880001
:102b4c0060168800a0168800e01688002017880000
:102b5c0060178800a01788000880fb000100200087
:102b6c0042022000820f5000e08f580095003e007a
:102b7c0000600100240037002600370028003700d1
:102b8c002a0037002c0037002e00370030003700a9
:102b9c003200370034003700360037003800370079
:102bac003a0037003c0037003e0037004000370049
:102bbc004200370044003700460037004800370019
:102bcc004a0037004c0037004e00370050003700e9
:102bdc0052003700540037005600370058003700b9
:102bec005a0037005c0037005e0037006000370089
:102bfc006200370064003700660037006800370059
:102c0c006a0037006c003700f0c2a900f4c2a800bb
:102c1c006e003700f0e2a900f4e2a8006b00370068
:102c2c00f102a900f502a80068003700f122a90002
:102c3c00f522a80065003700c8a2a900cca2a80004
:102c4c0062003700c882a900cc82a8005f00370060
:102c5c00c842a900cc42a8005c003700c822a900d9
:102c6c00cc22a80059003700c802a900cc02a80049
:102c7c0056003700c902a900cd02a8005300370046
:102c8c00c982a900cd82a80050003700c9a2a900b2
:102c9c00cda2a8004d003700e862a900ec62a800a4
:102cac004a003700d1a2a900d5a2a80047003700de
:102cbc00d1c2a900d5c2a80044003700d822a9006f
:102ccc00dc22a80041003700d842a900dc42a80051
:102cdc003e003700d862a900dc62a8003b00370038
:102cec00d882a900dc82a80038003700d8a2a9003d
:102cfc00dca2a80035003700d8c2a900dcc2a800ad
:102d0c0032003700d8e2a900dce2a8002f0037001f
:102d1c00e802a900ec02a8002c003700e822a90068
:102d2c00ec22a80029003700e002a900e402a80068
:102d3c0026003700e022a900e422a8002300370077
:102d4c00e042a900e442a80020003700e062a9009c
:102d5c00e462a8001d003700e082a900e482a8000c
:102d6c001a003700c862a900cc62a800170037000f
:102d7c00d902a900dd02a80014003700d922a9004d
:102d8c00dd22a80011003700d942a900dd42a800bd
:102d9c000e003700d962a900dd62a8000b003700d5
:102dac00c922a900cd22a80008003700c942a900f9
:102dbc00cd42a80005003700c962a900cd62a80069
:102dcc0002003700d0012b001afe07004f047800d8
:042ddc0000000600ed
:020000040000fa
:10150000ec0e00000200000000000000e00e0000f1
:1015100004000000020000000000000000000000c5
:10152000820e00005e0000000000000000100000bd
:101530001000000000000000660e00001c0000000b
:1015400000000000e40e00000400000002000000a3
:101550000282010081000000e80e0000040000008b
:10156000020000000000cd000c000000160c00007e
:101570001e01000000000000340d000060000000ab
:1015800002000000e00101000000000002006d0008
:101590000426c60000020000006d040027c60000fb
:1015a000020000006f252e00c600020000006f0040
:1015b000252fc60000020000004f04007bb600008b
